:020000040800F2
:10000000A8B80020753B0008295C0308613B000884
:10001000613B0008613B0008613B0008613B000850
:10002000000000000000000000000000613C00082B
:10003000613B000800000000F93B000871AB0008BC
:10004000013E0008013E0008013E0008013E000894
:10005000013E0008013E0008013E0008013E000884
:10006000013E0008013E0008013E0008013E000874
:10007000013E0008013E0008013E0008013E000864
:10008000013E0008013E0008013E0008013E000854
:10009000013E0008013E0008013E0008013E000844
:1000A000013E0008013E0008013E0008013E000834
:1000B000013E0008013E0008013E0008013E000824
:1000C000013E0008013E0008013E0008013E000814
:1000D000013E0008013E0008013E0008013E000804
:1000E000013E0008013E0008013E0008013E0008F4
:1000F000013E0008013E0008013E0008013E0008E4
:10010000013E0008013E0008013E0008013E0008D3
:10011000013E0008013E0008013E0008013E0008C3
:10012000013E0008013E0008013E0008013E0008B3
:10013000013E0008013E0008013E0008013E0008A3
:10014000013E0008013E0008013E0008013E000893
:10015000013E0008013E0008013E0008013E000883
:10016000013E0008013E0008013E0008013E000873
:10017000013E0008013E0008013E0008013E000863
:08018000013E0008013E0008E9
:1001880081F0004102E000BF83F0004330B54FEA40
:1001980041044FEA430594EA050F08BF90EA020FAD
:1001A8001FBF54EA000C55EA020C7FEA645C7FEA40
:1001B800655C00F0E2804FEA5454D4EB5555B8BF63
:1001C8006D420CDD2C4480EA020281EA030382EAD4
:1001D800000083EA010180EA020281EA0303362D66
:1001E80088BF30BD11F0004F4FEA01314FF4801C39
:1001F8004CEA113102D0404261EB410113F0004F4B
:100208004FEA03334CEA133302D0524263EB430301
:1002180094EA050F00F0A780A4F10104D5F1200E9F
:100228000DDB02FA0EFC22FA05F2801841F10001FA
:1002380003FA0EF2801843FA05F359410EE0A5F1CE
:1002480020050EF1200E012A03FA0EFC28BF4CF0FF
:10025800020C43FA05F3C01851EBE37101F00045B5
:1002680007D54FF0000EDCF1000C7EEB00006EEBC2
:100278000101B1F5801F1BD3B1F5001F0CD349084C
:100288005FEA30004FEA3C0C04F101044FEA4452A3
:1002980012F5800F80F09A80BCF1004F08BF5FEA2A
:1002A800500C50F1000041EB045141EA050130BD0A
:1002B8005FEA4C0C404141EB0101013C28BFB1F51C
:1002C800801FE9D291F0000F04BF01460020B1FA67
:1002D80081F308BF2033A3F10B03B3F120020CDA3A
:1002E8000C3208DD02F1140CC2F10C0201FA0CF018
:1002F80021FA02F10CE002F11402D8BFC2F1200C7D
:1003080001FA02F120FA0CFCDCBF41EA0C01904032
:10031800E41AA2BF01EB0451294330BD6FEA04047B
:100328001F3C1CDA0C340EDC04F11404C4F1200266
:1003380020FA04F001FA02F340EA030021FA04F378
:1003480045EA030130BDC4F10C04C4F1200220FACF
:1003580002F001FA04F340EA0300294630BD21FA0D
:1003680004F0294630BD94F0000F83F4801306BFD3
:1003780081F480110134013D4EE77FEA645C18BFC7
:100388007FEA655C29D094EA050F08BF90EA020F5E
:1003980005D054EA000C04BF1946104630BD91EA56
:1003A800030F1EBF0021002030BD5FEA545C05D159
:1003B8004000494128BF41F0004130BD14F5800498
:1003C8003CBF01F5801130BD01F0004545F0FE410C
:1003D80041F470014FF0000030BD7FEA645C1ABF41
:1003E800194610467FEA655C1CBF0B46024650EA78
:1003F800013406BF52EA033591EA030F41F40021A4
:1004080030BD00BF90F0000F04BF0021704730B529
:100418004FF4806404F132044FF000054FF00001FE
:1004280050E700BF90F0000F04BF0021704730B5BF
:100438004FF4806404F1320410F0004548BF404294
:100448004FF000013EE700BF42004FEAE2014FEAE9
:1004580031014FEA02701FBF12F07F4393F07F4FC4
:1004680081F06051704732F07F4208BF704793F0C7
:100478007F4F04BF41F40021704730B54FF46074DA
:1004880001F0004521F000411CE700BF50EA0102DD
:1004980008BF704730B54FF000050AE050EA010286
:1004A80008BF704730B511F0004502D5404261EBF6
:1004B80041014FF4806404F132045FEA915C3FF437
:1004C800D8AE4FF003025FEADC0C18BF03325FEAD4
:1004D800DC0C18BF033202EBDC02C2F1200300FA85
:1004E80003FC20FA02F001FA03FE40EA0E0021FAAA
:1004F80002F11444BDE600BF70B54FF0FF0C4CF498
:10050800E06C1CEA11541DBF1CEA135594EA0C0F49
:1005180095EA0C0F00F0DEF82C4481EA030621EA84
:100528004C5123EA4C5350EA013518BF52EA0335BF
:1005380041F4801143F4801338D0A0FB02CE4FF071
:100548000005E1FB02E506F00042E0FB03E54FF0A1
:100558000006E1FB03569CF0000F18BF4EF0010E99
:10056800A4F1FF04B6F5007F64F5407404D25FEA95
:100578004E0E6D4146EB060642EAC62141EA555148
:100588004FEAC52040EA5E504FEACE2EB4F1FD0C8A
:1005980088BFBCF5E06F1ED8BEF1004F08BF5FEA08
:1005A800500E50F1000041EB045170BD06F00046BA
:1005B80046EA010140EA020081EA0301B4EB5C0467
:1005C800C2BFD4EB0C0541EA045170BD41F480115F
:1005D8004FF0000E013C00F3AB8014F1360FDEBF84
:1005E800002001F0004170BDC4F10004203C35DA60
:1005F8000C341BDC04F11404C4F1200500FA05F3E3
:1006080020FA04F001FA05F240EA020001F0004283
:1006180021F0004110EBD37021FA04F642EB0601F9
:100628005EEA430E08BF20EAD37070BDC4F10C0423
:10063800C4F1200500FA04F320FA05F001FA04F2E7
:1006480040EA020001F0004110EBD37041F10001D3
:100658005EEA430E08BF20EAD37070BDC4F12005DE
:1006680000FA05F24EEA020E20FA04F301FA05F246
:1006780043EA020321FA04F001F0004121FA04F2EE
:1006880020EA020000EBD3705EEA430E08BF20EABE
:10069800D37070BD94F0000F0FD101F000464000F8
:1006A80041EB010111F4801F08BF013CF7D041EA7A
:1006B800060195F0000F18BF704703F0004652007E
:1006C80043EB030313F4801F08BF013DF7D043EA4F
:1006D8000603704794EA0C0F0CEA135518BF95EA05
:1006E8000C0F0CD050EA410618BF52EA4306D1D18C
:1006F80081EA030101F000414FF0000070BD50EAAB
:10070800410606BF1046194652EA430619D094EA34
:100718000C0F02D150EA013613D195EA0C0F05D11E
:1007280052EA03361CBF104619460AD181EA030172
:1007380001F0004141F0FE4141F470014FF000002A
:1007480070BD41F0FE4141F4780170BD70B54FF0C5
:10075800FF0C4CF4E06C1CEA11541DBF1CEA135545
:1007680094EA0C0F95EA0C0F00F0A7F8A4EB050427
:1007780081EA030E52EA03354FEA013100F088801E
:100788004FEA03334FF0805545EA131343EA1263E7
:100798004FEA022245EA111545EA10654FEA00269C
:1007A8000EF000419D4208BF964244F1FD0404F555
:1007B800407402D25B084FEA3202B61A65EB0305B1
:1007C8005B084FEA32024FF480104FF4002CB6EB6E
:1007D800020E75EB030E22BFB61A754640EA0C00EE
:1007E8005B084FEA3202B6EB020E75EB030E22BF2E
:1007F800B61A754640EA5C005B084FEA3202B6EB6F
:10080800020E75EB030E22BFB61A754640EA9C002D
:100818005B084FEA3202B6EB020E75EB030E22BFFD
:10082800B61A754640EADC0055EA060E18D04FEABB
:10083800051545EA16754FEA06164FEAC30343EA5B
:1008480052734FEAC2025FEA1C1CC0D111F4801F28
:100858000BD141EA00014FF000004FF0004CB6E721
:1008680011F4801F04BF01430020B4F1FD0C88BFC0
:10087800BCF5E06F3FF6AFAEB5EB030C04BFB6EBCB
:10088800020C5FEA500C50F1000041EB045170BDBE
:100898000EF0004E4EEA113114EB5C04C2BFD4EBEB
:1008A8000C0541EA045170BD41F480114FF0000E6F
:1008B800013C90E645EA060E8DE60CEA135594EAEB
:1008C8000C0F08BF95EA0C0F3FF43BAF94EA0C0FEE
:1008D8000AD150EA01347FF434AF95EA0C0F7FF463
:1008E80025AF104619462CE795EA0C0F06D152EAB7
:1008F80003353FF4FDAE1046194622E750EA41069B
:1009080018BF52EA43067FF4C5AE50EA41047FF4AB
:100918000DAF52EA43057FF4EBAE12E74FF0FF3C10
:1009280006E000BF4FF0010C02E000BF4FF0010CE1
:100938004DF804CD4FEA410C7FEA6C5C4FEA430C5A
:1009480018BF7FEA6C5C1BD001B050EA410C0CBFA9
:1009580052EA430C91EA030F02BF90EA020F00200B
:10096800704710F1000F91EA030F58BF994208BF72
:1009780090422CBFD8176FEAE37040F0010070472F
:100988004FEA410C7FEA6C5C02D150EA013C07D186
:100998004FEA430C7FEA6C5CD6D152EA033CD3D0D1
:1009A8005DF8040B704700BF8446104662468C46CB
:1009B8001946634600E000BF01B5FFF7B7FF0028FE
:1009C80048BF10F1000F01BD4DF808EDFFF7F4FF27
:1009D8000CBF012000205DF808FB00BF4DF808EDB2
:1009E800FFF7EAFF34BF012000205DF808FB00BFD5
:1009F8004DF808EDFFF7E0FF94BF012000205DF8F7
:100A080008FB00BF4DF808EDFFF7CEFF94BF0120AB
:100A180000205DF808FB00BF4DF808EDFFF7C4FFA4
:100A280034BF012000205DF808FB00BF4FEA4102F7
:100A3800B2F1E04324BFB3F5001CDCF1FE5C0DD934
:100A480001F0004C4FEAC0024CEA5070B2F1004F7E
:100A580040EB830008BF20F00100704711F0804F81
:100A680021D113F13872BCBF01F00040704741F446
:100A780080114FEA5252C2F11802C2F1200C10FA4A
:100A88000CF320FA02F018BF40F001004FEAC1232E
:100A98004FEAD32303FA0CFC40EA0C0023FA02F3D2
:100AA8004FEA4303CCE77FEA625307D150EA0133A8
:100AB8001EBF4FF0FE4040F44000704701F0004078
:100AC80040F0FE4040F40000704700BF80F0004056
:100AD80002E000BF81F0004142001FBF5FEA41030E
:100AE80092EA030F7FEA226C7FEA236C6AD04FEA0E
:100AF8001262D2EB1363C1BFD21841404840414053
:100B0800B8BF5B42192B88BF704710F0004F40F404
:100B1800000020F07F4018BF404211F0004F41F420
:100B2800000121F07F4118BF494292EA030F3FD0EC
:100B3800A2F1010241FA03FC10EB0C00C3F12003FF
:100B480001FA03F100F0004302D5494260EB40008E
:100B5800B0F5000F13D3B0F1807F06D340084FEAF9
:100B6800310102F10102FE2A51D2B1F1004F40EBEE
:100B7800C25008BF20F0010040EA03007047490056
:100B880040EB0000013A28BFB0F5000FEDD2B0FAF3
:100B980080FCACF1080CB2EB0C0200FA0CF0AABF16
:100BA80000EBC25052421843BCBFD04018437047B4
:100BB80092F0000F81F4000106BF80F400000132BA
:100BC800013BB5E74FEA41037FEA226C18BF7FEA91
:100BD800236C21D092EA030F04D092F0000F08BFD3
:100BE8000846704790EA010F1CBF0020704712F0BA
:100BF8007F4F04D1400028BF40F00040704712F1F9
:100C080000723CBF00F50000704700F0004343F05D
:100C1800FE4040F4000070477FEA226216BF084693
:100C28007FEA23630146420206BF5FEA412390EA56
:100C3800010F40F4800070474FF0000304E000BF4C
:100C480010F0004348BF40425FEA000C08BF7047FD
:100C580043F0964301464FF000001CE050EA0102C1
:100C680008BF70474FF000030AE000BF50EA0102D6
:100C780008BF704711F0004302D5404261EB4101C3
:100C88005FEA010C02BF84460146002043F0B643E8
:100C980008BFA3F18053A3F50003BCFA8CF2083A0D
:100CA800A3EBC25310DB01FA02FC634400FA02FC16
:100CB800C2F12002BCF1004F20FA02F243EB02001D
:100CC80008BF20F00100704702F1200201FA02FC7F
:100CD800C2F1200250EA4C0021FA02F243EB020072
:100CE80008BF20EADC7070474FF0FF0C1CEAD052B6
:100CF8001EBF1CEAD15392EA0C0F93EA0C0F6FD077
:100D08001A4480EA010C400218BF5FEA41211ED054
:100D18004FF0006343EA501043EA5111A0FB013140
:100D28000CF00040B1F5000F3EBF490041EAD37115
:100D38005B0040EA010062F17F02FD2A1DD8B3F191
:100D4800004F40EBC25008BF20F00100704790F000
:100D5800000F0CF0004C08BF49024CEA502040EA52
:100D680051207F3AC2BFD2F1FF0340EAC250704718
:100D780040F400004FF00003013A5DDC12F1190F56
:100D8800DCBF00F000407047C2F10002410021FAC8
:100D980002F1C2F1200200FA02FC5FEA310040F1E0
:100DA800000053EA4C0308BF20EADC70704792F059
:100DB800000F00F0004C02BF400010F4000F013A91
:100DC800F9D040EA0C0093F0000F01F0004C02BF8C
:100DD800490011F4000F013BF9D041EA0C018FE7FB
:100DE8000CEAD15392EA0C0F18BF93EA0C0F0AD001
:100DF80030F0004C18BF31F0004CD8D180EA010027
:100E080000F00040704790F0000F17BF90F0004FBF
:100E1800084691F0000F91F0004F14D092EA0C0FA1
:100E280001D142020FD193EA0C0F03D14B0218BF34
:100E3800084608D180EA010000F0004040F0FE407A
:100E480040F40000704740F0FE4040F44000704716
:100E58004FF0FF0C1CEAD0521EBF1CEAD15392EA95
:100E68000C0F93EA0C0F69D0A2EB030280EA010C85
:100E780049024FEA402037D04FF0805343EA11111E
:100E880043EA10130CF000408B4238BF5B0042F17C
:100E98007D024FF4000C8B4224BF5B1A40EA0C0021
:100EA800B3EB510F24BFA3EB510340EA5C00B3EB53
:100EB800910F24BFA3EB910340EA9C00B3EBD10F41
:100EC80024BFA3EBD10340EADC001B0118BF5FEA93
:100ED8001C1CE0D1FD2A3FF650AF8B4240EBC250BC
:100EE80008BF20F0010070470CF0004C4CEA50207D
:100EF8007F32C2BFD2F1FF0340EAC250704740F4CC
:100F080000004FF00003013A37E792F0000F00F0BD
:100F1800004C02BF400010F4000F013AF9D040EA3B
:100F28000C0093F0000F01F0004C02BF490011F4CF
:100F3800000F013BF9D041EA0C0195E70CEAD153C7
:100F480092EA0C0F08D142027FF47DAF93EA0C0FAE
:100F58007FF470AF084676E793EA0C0F04D14B0292
:100F68003FF44CAF08466EE730F0004C18BF31F044
:100F7800004CCAD130F000427FF45CAF31F000433E
:100F88007FF43CAF5FE700BF4FF0FF3C06E000BFD7
:100F98004FF0010C02E000BF4FF0010C4DF804CDFA
:100FA8004FEA40024FEA41037FEA226C18BF7FEA0A
:100FB800236C11D001B052EA530C18BF90EA010F0C
:100FC80058BFB2EB030088BFC81738BF6FEAE1709B
:100FD80018BF40F0010070477FEA226C02D15FEA37
:100FE800402C05D17FEA236CE4D15FEA412CE1D0A3
:100FF8005DF8040B704700BF844608466146FFE76A
:101008000FB5FFF7C9FF002848BF10F1000F0FBD4B
:101018004DF808EDFFF7F4FF0CBF012000205DF844
:1010280008FB00BF4DF808EDFFF7EAFF34BF0120C9
:1010380000205DF808FB00BF4DF808EDFFF7E0FF62
:1010480094BF012000205DF808FB00BF4DF808EDB3
:10105800FFF7D2FF94BF012000205DF808FB00BF16
:101068004DF808EDFFF7C8FF34BF012000205DF8F8
:1010780008FB00BF4FEA40024FEA41037FEA226CB7
:1010880002D15FEA402C08D17FEA236C02D15FEAE3
:10109800412C02D14FF0000070474FF0010070471B
:1010A8004FEA4002B2F1FE4F0FD34FF09E03B3EB6D
:1010B80012620DD94FEA002343F0004310F0004FAD
:1010C80023FA02F018BF404270474FF00000704703
:1010D80012F1610F01D1420205D110F0004008BFA2
:1010E8006FF0004070474FF00000704742000ED28A
:1010F800B2F1FE4F0BD34FF09E03B3EB126209D44B
:101108004FEA002343F0004323FA02F070474FF000
:101118000000704712F1610F01D1420202D14FF075
:10112800FF3070474FF00000704700BF7BB972B9BD
:101138000029BEBF00204FF0004106E008BF00288C
:101148001CBF6FF000414FF0FF3000F077B8ADF1F1
:10115800080C6DE904CE002909DB002B1ADB00F02E
:10116800BCF8DDF804E0DDE9022304B07047404232
:1011780061EB4101002B1BDB00F0AFF8DDF804E068
:10118800DDE9022304B0404261EB4101524263EBC6
:1011980043037047524263EB430300F09EF8DDF8C7
:1011A80004E0DDE9022304B0404261EB41017047ED
:1011B800524263EB430300F090F8DDF804E0DDE908
:1011C800022304B0524263EB4303704753B94AB950
:1011D800002908BF00281CBF4FF0FF314FF0FF3037
:1011E80000F02CB8ADF1080C6DE904CE00F075F8EC
:1011F800DDF804E0DDE9022304B07047D0B5FFF75D
:1012080023F900220B4B06460F46FFF775F900F04D
:1012180017F80446FFF7F6F80022074BFFF76CF9BA
:1012280002460B4630463946FEF7AEFF00F008F896
:101238002146D0BD0000F03D0000F041704700BFDE
:101248004A0011D212F5001211D20DD56FF478733D
:10125800B3EB62520ED44FEAC12343F0004343EA92
:10126800505323FA02F070474FF00000704750EADD
:10127800013002D14FF0FF3070474FF00000704747
:1012880010F8012B11F8013B012A28BF9A42F7D028
:10129800D01A7047034611F8012B03F8012B002AD6
:1012A800F9D17047034613F8012B002AFBD1181A0D
:1012B80001387047430803F05533C01A00F0333340
:1012C800800800F0333018444FF0013300EB101061
:1012D80000F00F305843000E70472DE9F04786465E
:1012E8008C460846089E154674461946002B40F061
:1012F800C1808542B2FA82F245D94AB1C2F12003CF
:1013080000FA02FC954094402EFA03F343EA0C0CD1
:101318004FEA154EA8B2230CBCFBFEF80EFB18CC06
:1013280008FB00F943EA0C43994528D9EB1808F162
:10133800FF3704D2994502D9A8F102072B44A3EB41
:101348000903A4B2B3FBFEFC0EFB1C330CFB00F03C
:1013580044EA0344A04214D92C190CF1FF3304D2F7
:10136800A04202D9ACF102032C44241A43EA0740F4
:101378001EB1D440002334607360BDE8F08747464F
:10138800DDE76346F1E792BB431B01214FEA154EA7
:10139800AFB2200CB3FBFEFC0EFB1C330CFB07F8B2
:1013A80040EA0343984561D9EB180CF1FF3004D2A9
:1013B800984502D9ACF102002B44A3EB0803A4B270
:1013C800B3FBFEFC0EFB1C330CFB07F744EA03449B
:1013D800A7424DD92C190CF1FF3304D2A74202D9E8
:1013E800ACF102032C44E41B43EA0040C0E7C2F11D
:1013F80020039540944020FA03F12EFA03F34FEAB4
:10140800154E9040AFB20343B1FBFEFC0EFB1C101F
:10141800190C0CFB07F841EA0041884522D96918E4
:101428000CF1FF3004D2884502D9ACF102002944FE
:10143800A1EB08019BB2B1FBFEFC0EFB1C110CFBDF
:1014480007F743EA01439F420ED9EB180CF1FF312D
:1014580004D29F4202D9ACF102012B44DB1B41EAC2
:10146800004193E76046E3E76146F7E76046A4E793
:101478006346B8E7834206D916B9002108467CE7D7
:10148800C6E900E0F9E7B3FA83F78FB9834201D3DD
:10149800724508D8BEEB020460EB030301209C46AA
:1014A8001EB9002169E73846FAE7C6E9004CF8E7B3
:1014B800C7F1200CBB400EFA07F522FA0CF42EFAFD
:1014C8000CF1BA401C4320FA0CF3B8404FEA144917
:1014D80001431FFA84FEB3FBF9F809FB18300B0C23
:1014E80008FB0EFA43EA00439A4540D9E31808F18D
:1014F800FF3004D29A4502D9A8F102002344A3EB95
:101508000A0389B2B3FBF9F809FB183308FB0EFE8E
:1015180041EA03418E452CD9611808F1FF3304D202
:101528008E4502D9A8F10203214443EA0040A1EB09
:101538000E01A0FB02984145CE46434602D306D190
:101548004D4504D20138B9EB020E68EB0403002EB6
:10155800A7D0B5EB0E0261EB030101FA0CFC22FAED
:1015680007F3F9404CEA0303C6E9003199E740461E
:10157800C5E74346D9E700002DE9F04390F8A530C8
:1015880004460D4685B023B94FF07E50FFF7A2FA06
:101598000546D4F884202E4B9A4212D12846FEF7ED
:1015A80053FF29A3D3E90023FFF736FA011E18BF1A
:1015B800012104F184000FF0F1FB0120C4F89850D8
:1015C80005E0B4F89C30B3F5807F03D1002005B066
:1015D800BDE8F08304F15009484626F08DFE002846
:1015E800F4D01C492846FFF77FFBFFF77FFD94F8EE
:1015F8008080C3B294F89C60276E206DB8F1000F0C
:101608000DD08DF80D3002230122002100938DF8B2
:101618000C6003ABB847484643F05BFACDE78DF85A
:101628000B600126414632468DF80C3000960DF1CC
:101638000B03B847009642463146276E206D03AB30
:10164800E8E700BFAFF30080AE47E17A14AEEF3FA2
:10165800C81B050800007F4330F0004201462DE911
:10166800F84F034604D10120BDE8F84F32F010BD11
:10167800002803DABDE8F84F32F012BDB0F1FF4F91
:1016880003DBFFF729FABDE8F88FB0F5000F35DA6C
:101698004FF09841FFF728FB6FF018020346C3F399
:1016A8001604DE15764B4FF07E517F3E23441644D8
:1016B80003F4000006EBD35680F07E502043FFF77A
:1016C80009FA04F10F026F4B05461340002B3ED177
:1016D8000021FFF79DFC98B1002E00F0C88030462D
:1016E800FFF7AEFA68490546FFF7FEFA0446674970
:1016F8002846FFF7F9FA01462046C2E70022CEE75E
:101708005DA1D1E90001FFF791F92946FFF7ECFA4D
:1017180001464FF07C50FFF7DDF90446294628467C
:10172800FFF7E2FA01462046FFF7DEFA04460EB953
:1017380021466FE03046FFF783FA07465249FFF724
:10174800D3FA524906463846FFF7CEFA72E04FF010
:101758008041DFF83CB1FFF7BFF901462846A344B2
:10176800FFF776FB81463046FFF76AFA494680461E
:101778004846FFF7B9FA01468246FFF7B5FA4549E8
:101788000746FFF7B1FA4449FFF7A6F93946FFF7CC
:10179800ABFA4249FFF7A0F93946FFF7A5FA4049E5
:1017A800FFF79AF95146FFF79FFA3E4982463846B5
:1017B800FFF79AFA3C49FFF78FF93946FFF794FA91
:1017C8003A49FFF789F93946FFF78EFA014650463C
:1017D800FFF782F9C4F55713074603F5227343EA66
:1017E8000B03002B30DD4FF07C512846FFF77CFAC5
:1017F8002946FFF779FA014604463846FFF76CF99F
:101808004946FFF771FA074646B901462046FFF7F1
:1018180061F901462846FFF75DF934E71A49404661
:10182800FFF762FA194906464046FFF75DFA39465E
:10183800FFF752F901462046FFF74CF92946FFF712
:1018480049F901463046E6E701462846FFF742F9DE
:101858004946FFF749FA0446002E3FF469AF0A49A2
:101868004046FFF741FA0949064640466CE7002022
:1018780009E700BFAFF30080555555555555D53F7D
:1018880020FB4A00F0FF7F008071313FD1F7173706
:10189800305CCFFF9788173E25333A3E2549923E64
:1018A800ABAA2A3F4FD01C3E298E633ECDCCCC3EFE
:1018B80031F000432DE9F04F804687B00F4681464E
:1018C8000C460ED180F480094FEA490919F5000F3A
:1018D80040F2668239464046FFF7FEF807B0BDE899
:1018E800F08F20F00046B6F1FF4F02D8B3F1FF4F5A
:1018F80008D9B9F17E5FEDD184F48004640014F551
:10190800000FE5E7002832463DDAB3F1974F1BD3C5
:10191800B3F1FF4F3AD00225B4F17C5F4DD1B9F154
:10192800000F80F29780B6F1FF4F28F0004040F09A
:101938004F82A6F17E562E4340F0A080404607B065
:10194800BDE8F04F32F0ACBBB3F17E5F2ED3D915B2
:10195800C1F1960143FA01F505FA01F18B423BD139
:10196800B3F17E5F4AD1002C80F29380002140467B
:10197800FFF74EFB00284FD04FEAD97007B0BDE8FB
:10198800F04F32F085BBB3F1FF4F3CD1B6F17E5F2B
:1019980000F0068204D9002CC0F2058238469DE783
:1019A800002C80F2008207F1004097E7B1F1804FE8
:1019B80038D0B1F17C5F53D0002529F0404128F0A0
:1019C8000040B1F17E5F3BD1002C32DA01464FF086
:1019D8007E50FFF73DFA2CE0B3F17E5FC3D00025BF
:1019E800B4F1804FE9D1B6F1BF4F1DD2B6F1D05F47
:1019F80024D941464046FFF777F96FE705F001051E
:101A0800C5F10205ECE7B3F17E5FACD0B1F1804FD0
:101A18004FF00005E7D07FE741464FF07E50FFF7D3
:101A280017FA5BE70025DEE7B6F1FF4F28F0004024
:101A380031D1B9F1000FBFF651AF7AE728F0004075
:101A48004EBB002C22DAB9F1000F1DDA6B1E58428A
:101A5800584193E7404607B0BDE8F04F49F05AB8FF
:101A6800B6F1FF4F20F000403FF438AFB6F17E5F8B
:101A78003FF464AF002E3FF431AF5FE7012D7FF4F0
:101A88002DAF00F1004029E7304677E7012D7FF4BC
:101A980025AF404622E74FEAD9710139029129431F
:101AA8003FF44CAFB3F19A4F40F29F81604B9E4296
:101AB80007D8002C0ADA002007B0BDE8F04F32F052
:101AC800DFBA5C4B9E4207D9002CF4DC002007B03B
:101AD800BDE8F04F49F080B84FF07E51FEF7FAFFAD
:101AE80006465549FFF700F9544980463046FFF746
:101AF800FBF881464CA1D1E90001FEF797FF824629
:101B08004FF07A513046FFF7EFF801465046FEF79E
:101B1800E1FF3146FFF7E8F801464FF07C50FEF749
:101B2800D9FF824631463046FFF7DEF80146504677
:101B3800FFF7DAF84249FFF7D7F801464846FEF7BB
:101B4800C9FF014606464046FEF7C6FF20F47F6BF4
:101B580041462BF00F0B5846FEF7BCFF24F47F6478
:101B680001463046FEF7B6FF013D029B24F00F0404
:101B7800064638461D43214614BF4FF07E55314D69
:101B8800FEF7A8FF5946FFF7AFF8804639463046BA
:101B9800FFF7AAF801464046FEF79EFF0646214693
:101BA8005846FFF7A1F8014607463046FEF794FF6E
:101BB80000280446804620F0004320DDB3F1864F1C
:101BC8000BD900212846FFF72DFA003818BF01204D
:101BD80072E7002114E1012227E139D11A49304680
:101BE800FEF77AFF814639462046FEF773FF014625
:101BF8004846FFF735FA0028E3D186232DE0134A3B
:101C0800934207D900212846FFF70CFA003818BF7D
:101C180001205CE71CD13946FEF75CFF3146FFF72F
:101C280015FA0028E9D0EDE7E13D55555555D53F62
:101C3800F3FF7F3F0700803F00AAB83F70A5EC364E
:101C48003BAAB83F000080BF3CAA383300001643C7
:101C5800B3F17C5F40F2A080DB157E3B4FF40004BB
:101C68005249B8F1000F44FA03F438464444C4F327
:101C7800C753A3F17F0341FA03F1C3F1170301EA44
:101C88000401C4F3160444F4000444FA03F4B8BF8E
:101C98006442FEF71FFF074631463846FEF71CFF31
:101CA80020F47F68424928F00F084046FFF71CF8E7
:101CB800394681464046FEF70DFF01463046FEF79D
:101CC80009FF3C49FFF710F806463B494046FFF735
:101CD8000BF801463046FEF7FFFE07460146484628
:101CE800FEF7FAFE49460646FEF7F4FE0146384678
:101CF800FEF7F0FE314680463046FEF7F5FF2F49E5
:101D08000746FEF7F1FF2E49FEF7E4FE3946FEF7D7
:101D1800EBFF2C49FEF7E0FE3946FEF7E5FF2A49BE
:101D2800FEF7D8FE3946FEF7DFFF2849FEF7D4FE56
:101D38003946FEF7D9FF01463046FEF7CBFE074687
:101D480001463046FEF7D0FF81464FF080413846C5
:101D5800FEF7C0FE01464846FFF77AF841460746B7
:101D68003046FEF7C1FF4146FEF7B6FE014638464B
:101D7800FEF7B0FE3146FEF7ADFE01464FF07E504D
:101D8800FEF7A8FE00EBC453B3F5000F06DA2146B0
:101D980032F018F929462EE600247DE71846F9E7BF
:101DA8004FF07E509AE5002098E500BF000080FFC4
:101DB8000072313F1872313F8CBEBF354CBB313396
:101DC8000EEADD3555B38A38610B363BABAA2A3E9D
:101DD800B6F17E5F3FF4ADAD002E3FF457AE002D57
:101DE8003FF4ACAD00230225029319F0FF4F7FF4B6
:101DF800F0AE4FF09741FEF777FF6FF017010246FC
:101E0800D315C2F316027F3B42F07E560B44039370
:101E18007E4B9A4208DD7E4B9A427FF7DCAE039BED
:101E2800A6F500060133039300227A4B304604924C
:101E3800B24653F822B05946FEF74CFE3146814669
:101E48005846FEF749FE01464FF07E50FFF700F86E
:101E5800014605904846FEF747FF6F49019001EAA1
:101E68006606019B049A46F0005623F47F6806F53F
:101E7800800628F00F0806EB425641463046FEF72A
:101E880033FF01464846FEF725FE5946814630464F
:101E9800FEF720FE01465046FEF71CFE4146FEF7BF
:101EA80023FF01464846FEF715FE059B1946FEF737
:101EB8001BFF019983460846FEF716FF5749064659
:101EC800FEF712FF5649FEF707FE3146FEF70CFFF4
:101ED8005449FEF701FE3146FEF706FF5249FEF768
:101EE800FBFD3146FEF700FF5049FEF7F5FD314690
:101EF800FEF7FAFE4E49FEF7EFFD814631463046C1
:101F0800FEF7F2FE01464846FEF7EEFE414606465B
:101F18000198FEF7E1FD5946FEF7E6FE3146FEF769
:101F2800DBFD414681464046FEF7DEFE41498246DA
:101F3800FEF7D2FD4946FEF7CFFD20F47F66414605
:101F480026F00F063046FEF7CFFE3A498046304667
:101F5800FEF7C0FD5146FEF7BDFD01464846FEF7B7
:101F6800B9FD0199FEF7C0FE814631465846FEF795
:101F7800BBFE01464846FEF7AFFD82460146404695
:101F8800FEF7AAFD20F47F662B4926F00F0630469F
:101F9800FEF7AAFE414681463046FEF79BFD014604
:101FA8005046FEF797FD2549FEF79EFE80462449D8
:101FB8003046FEF799FE01464046FEF78DFD049A2D
:101FC800204B019253F82210FEF786FD064603982F
:101FD800FEF736FE1C4B019A80463146484653F8B8
:101FE80022A0FEF779FD5146FEF776FD4146FEF741
:101FF80073FD20F47F6B41462BF00F0B5846FEF71C
:1020080069FD5146FEF766FD4946A5E571C41C0009
:10201800D6B35D00C449050800F0FFDF42F1533E26
:1020280055326C3E05A38B3EABAAAA3EB76DDB3E8C
:102038009A99193F000040400040763F4F38763F5C
:10204800C623F6B8B4490508BC4905082DE9F04F80
:1020580091B0009302F004030293C2F3C203013368
:10206800840705460E46DDF868800392059340F024
:10207800BB81041D30B1072909D86FF01B0011B0CE
:10208800BDE8F08F01F007063444C6F10806009B4E
:102098004FF000094FF0040A591E4FF0FF334F4626
:1020A8000193CB465346CDF810900DB1009A2260AB
:1020B8000598002800F3E8809848009A824203D3E4
:1020C80097488242C0F0E080039AA4EB050E92077D
:1020D8004FEA9E0000F103810F2F00F2B180002D1E
:1020E80000F0058107F140020DEB020C019A0CF893
:1020F800200C0CF8102C049801300490E7E07A28A2
:102108005DD84B280ED8472859D829282DD82528F6
:1021180052D054D820287AD02338D0F1000B4BEB7A
:10212800000B74E04C382E2849D8DFE800F07048DE
:10213800484848484848484848484B484848484814
:1021480048484859484B4B595959704B6D48704845
:10215800184B184848827F4B48484B487F0000205E
:102168004FF0000B4FF0040A38E001222A38C0B2C1
:1021780002FA00F010EA0E0F49D110F0625C2FD17C
:1021880010EA020B43D06046013C5444B4FBFAF415
:102198000AFB04F4002D61D0A3EB050CA444B4455C
:1021A8003FF66BAF002868D1042B47D158F8043BA1
:1021B8002360042304342AE0019A013A01924FF083
:1021C800000B24E011F8010C6C2834D1002011F820
:1021D800023C83466C2BC5D14FF0080A5346D3E71F
:1021E80008F1070828F00708073424F00704F8E87E
:1021F80002AB35B106982044B0423FF63EAFC4E981
:1022080000AB4FF0000B08344FF0080A534611F8A2
:10221800010F002878D0BBF1000F7FF470AF25289C
:10222800F5D14FF0010B019B013301934FF0040AE4
:10223800ECE7584694E700208346A5E7082B02D030
:102248006FF015001BE708F1070828F00708F8E801
:102258000223C4E9002308230834D8E768B9042B0B
:1022680002D108F10408A4E7082BE9D108F107080E
:1022780028F0070808F10808EDE7059A013A0592E1
:1022880058F8042B009210E7039A900720D54FF0D6
:10229800010CA4EB050E4FEA9E00BEF5007FCFD2DD
:1022A8000F2FCDD8F5B107F140020DEB020E019AC0
:1022B800C0B20EF8200C0EF8102CBCF1000F3FF441
:1022C8001AAF60F07F000EF8200C09F10109013700
:1022D800C5F108024FF6DA7E0434069297E74FF00C
:1022E800000CDAE7BCF1000F01D00136EFE70298E5
:1022F80002360028EBD10098CDE90631FEF7D2FF6F
:10230800DDE906310644E2E7631BB3F5806F97D237
:1023180045B9A6F10804E018B1E600BF04AC04080A
:10232800A8D20508029A9B0828602B709DF81030E7
:10233800C2B1EB7085F80290B9F1000F05D0002208
:1023480008A8C5F1010C97420ED14FF0000AC5F15B
:1023580001030DF1200801930DF1300B574512D1FF
:10236800601B8CE66B70E5E710F8013B190608D591
:102378000CEB040EB64503F07F033FF67EAE04F87F
:10238800013B0132DFE7B9F1000F03D098F90020D3
:10239800002A17DB029BD3B11AF80B2004F8012B93
:1023A8000022019B18191044B0423FF666AE98F817
:1023B8000000009904F8010B2046039248F0CBFA7C
:1023C800039A14440AF1010A08F10108C6E798F8CB
:1023D800002055F822300093029B009845F82230DF
:1023E800FEF760FF421CDCE76FF00D0047E600BF18
:1023F8002DE9F04F97B000AFD7F880B03B62CBF330
:10240800C0030446894690F802A0FA62BB6141B94C
:10241800457800780AEB800020444D4517D8A0EB9A
:102428000409E378FB61BAF1000F02D01BF0010F39
:1024380016D1FB6953BBFB6A1BB1494620463A6A71
:1024480098474D4628465C37BD46BDE8F08F461C88
:102458003046FEF727FF0130304409F10109DCE777
:10246800626823787A62FA6A9900796104EB8301D9
:10247800002A40F001810E464FF000084D4601EB5E
:102488000A094E454CD101EB0A0610E01BF0020F79
:10249800D1D023789A007A61626804EB83017A626A
:1024A800FA6A002A77D14D46904601EB0A061BF0DE
:1024B800050F0CBF02230123FB62FB6906EB430AED
:1024C8000BF00203BB625645BCD016F8021B16F887
:1024D800013C54F82390994B994502D3984B994560
:1024E80036D3BB69002B40D0786A32F04DFE002805
:1024F8003BD0E9468AB06A46924B53617B6AC2E98F
:1025080006314FF4007313848F4B42F8103F0023B9
:102518004FF412518D4800F0A3FC023DCD46D2E79E
:1025280016F8013BF96254F82300FEF7BBFED7F812
:102538008430F96A01304BB1D7F8883098453EBFEE
:10254800D7F8843023F8180008F10108054498E703
:10255800BB6923B1786A32F017FE0028C9D11BF095
:10256800010F05D1FB6AED1AADE7BB6A002BAAD0B3
:102578004846FEF797FED7F8843053B1D7F888302D
:1025880098453FBFD7F88420431C22F8183008F13B
:102598000108054497E7BAF1000F73D01BF0040651
:1025A80073D0D046002607F1480052463B61B96215
:1025B80048F0D1F9B96A3B6901EB0A02BA62FA69D3
:1025C800F9695200FA60BA6A02EB41023A610BF00B
:1025D8000202BA603A69B96A8A4258D162781BF035
:1025E800020F18BF00217A6208BF4FEA5801B218DB
:1025F8001BF0010FD2B240F09F801BF0040F14BFF4
:1026080040460020BB616270A070E17020463A6AC3
:102618007969FB6A9847051EFFF614AFBB69414606
:1026280023707B6A3A6A6370FB6984F802A0E370DE
:1026380007F14800FB6A9847B0F10008C0F2BA8079
:102648007B69A9EB0A01C91AFB683A6AC91AD7E972
:102658000A0398470028C0F2AF804FF0000BA84447
:1026680008EB000507F1380AB34571D300213A6A2F
:102678000846FB6A9847E5E656464FF0000807F11A
:10268800380092E75646D04696E7B04694E7BA6ACD
:1026980012F8021B12F8015CBA6254F82500274AA6
:1026A800904202D3264A90421ED3BA6932B1786A60
:1026B8007B6032F069FD7B6800288BD1BA6802BB69
:1026C80008F1280207F1300C08F10100944407F1E1
:1026D800580208F1020852FA80F00CF8101C5FFA50
:1026E80088F800F8105C75E7BA693AB1786A7B60D7
:1026F80032F04AFD7B6800287FF46CAF1BF0010FB5
:1027080009D006F1280207F13000711C161806F8E6
:10271800205CCEB25EE71BF0040F3FF45BAF08F11C
:10272800280207F1300008F1010102EB000808F85F
:10273800105C5FFA81F84DE7002063E704AC0408F9
:10274800A8D20508A65305080400000198B004089B
:102758001BF80A3054F8239087F83730D7F88430BC
:102768002BB3D7F888309B4521D2D7F8843033F87B
:102778001B8001213A6AFB6A07F137009847002855
:102788001ADB0544B8F1000F06D14846FEF78AFD6A
:1027980000F101081FFA88F8414648463A6AFB6A80
:1027A8009847002808DB05440BF1010B5CE74FF064
:1027B8000008DEE7454645E6054643E6014B186056
:1027C800704700BF3802002080B505460E46174600
:1027D80098460BF0DBFA034601F020FB0446DFF8CD
:1027E8001890424649F8003039463046A84754F810
:1027F800090001F0E7F900BF08000000044608B529
:10280800EFF31183102383F31288BFF36F8F35F032
:1028180096FE204601F0C4F9024832F0DCFC33F0A1
:1028280021FAFCE75A540508054B00205A6822F0A3
:1028380002025A605A6822F004025A60704700BFC8
:10284800004004E010B5EFF31184102383F31288DD
:10285800BFF36F8F084803683BB9084A916A41F093
:1028680001019162916AC907FCD50133036084F3C1
:102878001188BFF36F8F10BD7C2500200008024629
:1028880010B5EFF31184102383F31288BFF36F8F11
:1028980011490B68A3B90122104BD3E8EF1F002997
:1028A80003D1C3E8E02F0028F7D104D102210C4A54
:1028B8000C4833F056F884F31188BFF36F8F10BDBE
:1028C800012B08BF084803F1FF3302BF826A22F0D8
:1028D800010282620B60EEE77C250020782500204B
:1028E8008E54050840B104080008024607B506F0F2
:1028F80055F80E4A136843F4807313600C4B0D4A65
:102908001A600D4BD3F8942042F00402C3F89420C7
:10291800D3F89430094A03F004030193019B9368A8
:1029280043F00203936003B05DF804FB002002400B
:10293800C80600200024F400000C024600080246E5
:102948002DE9F047044607464FF00109DFF85080AB
:1029580014B93846BDE8F08794FAA4F5B5FA85F5B8
:1029680009FA05F32E0108EB05156FEA030A24EAB4
:1029780003042B7B002BEBD058F806301B694BB9AE
:102988004644736802222846196807EA0A0732F0A3
:1029980078FFDDE7284698470028D9D1F0E700BF3F
:1029A800D0B1040830B5002289B00F490F4837F07C
:1029B80065F8002200230024CDE906230E230C4DE0
:1029C800CDE903344FF440722846CDE90144094B60
:1029D800094900940AF010FF0849284636F09DFE80
:1029E800204609B030BD00BF092A00086819002038
:1029F800C01400200D2D000888410020CF54050880
:102A080001480AF057BC00BF600F00202DE9F047CD
:102A1800804620480F4632F011FF0646002832D083
:102A280000252846BDE8F087237B83B12368DB684F
:102A38000BB120469847636883F8069023681B69A2
:102A4800CBB9636802222046196832F01AFF0136B2
:102A580010345445E8D3B8F1000FE2D0002DDFD090
:102A68002846FFF76DFF0546002FF7D000215020BC
:102A780036F007FFF2E7204698470028E1D009FA28
:102A880006F31D43E3E705464FF00109024CDFF862
:102A98000CA0DEE790250020D0B10408E0B10408BE
:102AA800014B53F82000704700B2040808B50346EC
:102AB80008462BB1044A136000F068FC002008BDEA
:102AC8006FF01500FBE700BF3C02002010B5044C76
:102AD800237813B903480AF0EDFB0123237010BDD6
:102AE8000E3E0020600F002010B50446094832F061
:102AF800A5FE3CB1084BD3E8EF1F0139C3E8E21F3C
:102B0800002AF8D1054836F0C5FFBDE81040044852
:102B18000AF0D0BB882500208C25002068190020E9
:102B2800600F002000200146034BD3E8EF0FC3E8F5
:102B3800E21F002AF9D170478825002070B5FFF7F9
:102B4800F1FF0546074C084EB44200D370BD6368D8
:102B58005B792BB123685B6813B1294620469847F7
:102B68001034F1E7D0B10408E0B1040810B5044C02
:102B78000449204632F041FC034B1C6010BD00BFE5
:102B8800780E0020ECB104088025002000230D4AAF
:102B980010B513700C4A4FF47A7113600B4A0C4845
:102BA8001360FFF783FFFFF7E1FF0A4B0A49184656
:102BB8008B4200D310BD1A1A5C68121101322271BF
:102BC8001033F5E70F3E0020882500208C250020D3
:102BD80057580308D0B10408E0B1040801460022A0
:102BE8000023014832F02ABC780E0020014832F058
:102BF800C3BC00BF780E0020024B0146186832F0B3
:102C080016BD00BF80250020014832F04BBD00BF33
:102C1800780E002070B5244B1878002843D0FFF7B1
:102C2800E5FF054600283BD1204B214C1B68002BB3
:102C380013DD36F0DBFED4E90032C00840EA41700B
:102C4800C01A40F2E9334FEAD10161EB0201984220
:102C580071F1000101D3FFF771FFD4E9003213F5D8
:102C68007A7342F10002C4E90032BDE87040FFF710
:102C7800CBBF63685B7923B12368294620461B686C
:102C880098471034B442F4D32846FFF7B5FF094BF0
:102C9800D3E8EF1F0139C3E8E21F002AC4D0F7E7E1
:102CA800054C064EEEE770BD0E3E0020882500203C
:102CB800601900208C250020D0B10408E0B1040878
:102CC80070B50D4D297861B90120FFF79FFE0B4CB7
:102CD8000B4EB44206D3FFF79DFF0028FBD101231A
:102CE8002B7070BD63685B791BB1236820469B68B5
:102CF80098471034EDE700BF0F3E0020D0B104081C
:102D0800E0B1040800212DE9F0470846FFF77EFEF0
:102D1800044658B34FF4C8784FF0000901F07EF824
:102D28001B4B1C4A1B58136033B11B4B1B68092BE8
:102D380002DD1A480AF0BEFA0025194FDFF85CA038
:102D480044B12046FFF7FCFD044618B94FF0FF38A0
:102D58004FF0FF39FFF75EFF064628B9B5B942467E
:102D68004B4650460AF0E0FA3546E9E74FF0FF389F
:102D78004FF0FF39D2E72B689B691BB10022284628
:102D8800114698471035BD42F5D3E8E7054DFAE7F7
:102D980008000000842500208C250020600F0020FA
:102DA800E0B10408D0B1040813B5184832F046FD64
:102DB800174B1B7873B1EFF31184102383F3128838
:102DC800BFF36F8FFFF726FF84F31188BFF36F8F70
:102DD80002B010BD0F4B1B68002BF9D050B9002270
:102DE80000230D48CDE900234FF4FA5200230BF0DD
:102DF800DDFAEDE70928EBD1074836F04BFE074826
:102E080002B0BDE810400AF055BA00BF8C2500207A
:102E18000F3E00208425002068190020600F002044
:102E280010B5064B04461B6898472146A060044825
:102E380032F083FBBDE81040FFF7B6BF3C0200202C
:102E4800780E0020044A054B9B1AB1EBD30F34BF10
:102E580052F831000020704780B00408D0B104084F
:102E68002DE9F04F8FB0C1F34A2804AF0D469146C3
:102E7800B8607B600C0DB8F1000F63D000264FF0EE
:102E8800040B4FF00A0A07F11403C7F80C80C7E9CE
:102E980007667E620193CDF808B0CDF800A007F16F
:102EA8001C0332464846F968FFF7A2FAB0F5006FEE
:102EB80003461CD36C468AB0D9F8041004AB2648E4
:102EC8001A46C3E9050140F2FF71D9614FF4007158
:102ED8001984224B42F8103F4FF4125133462048D0
:102EE800FFF7BEFFA5462C37BD46BDE8F08FC0F3FF
:102EF8000A0804F11700184420F0070080083B6016
:102F0800FFF76CFE68F35325044690B13B6800F167
:102F18001001C7E9083607F11403F961CDE900A3E8
:102F2800CDF808B048460F4AF96807F11C03FFF7C7
:102F38005FFA68F353252A4620467B68B96832F061
:102F4800C0FCD0E704F1170020F007008008FFF765
:102F580045FE0446EDE700BFE05405080400000103
:102F6800F0B004089D5803082DE9F04F87B00446D7
:102F7800DDE9105ADDE91279934698460391BFB10D
:102F88003B46524610210020CDF80090CDF8149011
:102F9800FFF75CF8B0F5006F06460AD340F2FF73FE
:102FA8000221174A174807B0BDE8F04F32F0E2BCDB
:102FB8003E4605F11700304420F007008008FFF76F
:102FC8000DFE04F007040BF0070BE40044EA8B1431
:102FD80044EA462444EA0554054640B13FB13B461D
:102FE80052463146CDF800901030FFF72FF843468F
:102FF80022462846039907B0BDE8F04F32F061BC7D
:103008001F550508F0B00408406820B1034BC01AEA
:1030180040F3CF0070474FF0FF30704780B004088E
:103028000EB403B503AB53F8042B014604480193CF
:1030380001F02CF902B05DF804EB03B0704700BF53
:10304800DF590308CA0605D48B064CBF0249034959
:10305800FFF7E6BF704700BF14B10508AF74050855
:103068002DE9F04F89B09B46149B9DF84CA0069320
:10307800159B04460593169B0D469046179E049390
:10308800BAF1000F00F09D8006F48073079332F0C8
:10309800F6FB06F00209024600283ED02046914978
:1030A800FFF7BEFF0746B9F1000F08D016F0440F2E
:1030B80035D12A4620468C49FFF7B2FF074406F06F
:1030C800010353B1894B204653F82A20884B89497C
:1030D800002A08BF1A46FFF7A3FF06F48073002BE7
:1030E80049D006F00803002B63D1B8F1000F66D071
:1030F800424620468049FFF793FF0546069B3D441C
:10310800002B6DD1049B002B73D1F30700F1E480F1
:1031180031462046FFF796FFD8E00746C3E7774BCE
:1031280018680028CAD0764B4FF47A791B684FF09C
:103138003C0CB5FBF3F5B5FBF0F14FF4616300FB14
:10314800115509FB05F5B1FBF3F2B5FBF0FE03FBE6
:10315800121100FB1E55B1FBFCF309FB05F5B5FB8D
:10316800F0F50CFB131120460091CDE901E5654906
:10317800FFF756FFA2E706F00803EBB1624B2046C3
:1031880053F82A206149FFF74BFF0546B8F1000FB5
:1031980005D0424620465849FFF742FF0544BBF197
:1031A800000FABD05A4620465949FFF739FF05446E
:1031B800A4E74FF0000BE1E706F00805E6E745460F
:1031C8009CE7BBF1010F069B06D1002B64D1049B41
:1031D800002B7BD000250CE0002BF8D04D485CE09C
:1031E8004D48069B22464D4931F09DFF049B002B1C
:1031F80068D0DFF82C81DFF82C91049F3146102F1E
:10320800204628BF10274FF0000BFFF71BFF5D4536
:1032180045DC059B494620461A78FFF701FF4FF029
:10322800010B1BF0070F03D141462046FFF7F8FEBC
:103238005F453BD9059B4946204613F80B20FFF70D
:10324800EFFE0BF1010BBBF1100FEAD14FF0000BB1
:1032580020463549FFF7E4FE5A46059B20469A5C0E
:10326800A2F120015F2928BF2E223049FFF7D8FE9E
:103278000BF1010BBBF1100F1DD01BF0070F03D191
:1032880041462046FFF7CCFE5F455A46E5D8414601
:103298002046FFF7C5FEEBE71F485546A1E7414624
:1032A8002046FFF7BDFE0BF1010BB0E72046204991
:1032B800FFF7B6FEC5E7059B3B440593049BDB1B64
:1032C80004939AD1BAF1000F7FF41FAF204609B0DA
:1032D800BDE8F04F32F072BB2046054A0549FFF7BA
:1032E8009FFE15E75C5505086055050810B20408EF
:1032F8005755050851B30508855505089825002038
:10330800942500206955050824B204088955050844
:103318008F5505080D5A0308DF5903089542000820
:103328001CC90508945505089A550508A9AF05084C
:103338001AC9050842F20F7373B58B4228BF0B46B2
:1033480005680446052168460D4A2FF0B9F9064676
:10335800636828460B225B680A4932F021FB6368E0
:103368003246694628465B6832F01AFB63681B22BE
:1033780028465B68044932F013FB02B070BD00BFF9
:10338800A5690508B85505089C55050800210123BD
:10339800064A904206D8064A01B901231360054B34
:1033A80018607047012140085B00F2E740420F00B7
:1033B8009425002098250020F8B50D460446064FB0
:1033C8004618B44201D12846F8BD14F8011BBB6861
:1033D80001485B689847F4E760AE0408014B036056
:1033E800012070476CB2040870B5104B0D461C687C
:1033F800B4B10F4B196800238B4202DB6FF0010058
:1034080070BD224612F8146B864202D0144601336E
:10341800F2E7E06835F0F2FE28B100202C60EFE713
:103428006FF00C00ECE76FF01200E9E748020020AB
:103438007CB204082DE9F8430646FDF733FF05463C
:10344800EFF31188102383F31288BFF36F8F114BAA
:103458001C68D3F804909C4208BF002434B988F350
:103468001188BFF36F8F2046BDE8F883A7683846F8
:10347800FDF718FFA84206D12A463946304647F0DC
:10348800B6FA0028EBD04C4501D02468E6E70024C2
:10349800E5E700BF4C0200202DE9F0410E46154635
:1034A800FFF7C8FF044628B3C3681BB35F690FB3AF
:1034B800062E07D0072E20D02A4631463B46BDE8C7
:1034C800F0411847838A3BB92A463146B84750B974
:1034D800A38A0133A38206E04FF6FF72934204D019
:1034E8000133A3820020BDE8F0810121114A12486E
:1034F80032F037FA6FF01500F5E745B12A7832B1A6
:103508000022828231462A465B699847EAE7A38A05
:10351800012B08D12A4607212046B8470028E2D1C6
:10352800A38A013BD6E70BB1013BDAE70221034A44
:10353800DDE700BF28560508A8B004084A56050864
:1035480010B5044608B1806838B9104A10480121FE
:1035580032F007FA6FF0150010BDFFF76BFF08B1E6
:103568000C4AF3E7A082EFF31181102383F312884A
:10357800BFF36F8F084B5A68C4E9003214605C606F
:1035880081F31188BFF36F8FE6E700BF685605081F
:10359800A8B00408815605084C02002008B5034865
:1035A800034A0021121A32F033FB08BD80110020B3
:1035B80088410020074808B5074A0849121A32F01E
:1035C80029FBBDE808400648064A0749121A32F0A6
:1035D80021BB00BF0000002044110020A8D205082C
:1035E8000000002000000020A8D205082DE9F047BF
:1035F80006460C4600AF002936D0D1E90012E9464C
:103608008AB06D46A3684FF0050AA8461F48C5E969
:103618000723C5E9050148F810AF002342464FF4D7
:1036280021511B48FFF71CFCD4E90312CD466369FE
:10363800AD461848C5E90723C5E90501C5F810A036
:10364800002342464FF421511148FFF709FCCD46AB
:10365800E3690121104A0E4832F08CF9A36901216F
:103668000E4A0B4832F086F9012E07D1EFF3058395
:103678000B4A31460648103B32F07CF92146304669
:1036880009F066FABD46BDE8F08700BFB0560508E8
:1036980020B10408DF5605080E5705081D57050810
:1036A8004B57050830BFFFF7FDBF00BF2DE9F041BC
:1036B80005460B4EDFF82C80324606EB0807CC1B7C
:1036C8002046094947F047F9A01942460021083C1D
:1036D80047F068F9C5F8904007F10800BDE8F081A7
:1036E8000000000008000000E0B10408054B5A691A
:1036F8009B689A421FBF044A536843F08053536043
:10370800704700BF5036002000ED00E070B52A4C2D
:1037180006460D4629482A4932F089FAA36ADB068B
:1037280047D52648274932F082FA1120A36A1C0798
:1037380004D52248244932F07AFA12201E4CA36A92
:10374800990712D521491D4832F071FA636BA26AB4
:10375800120609D501211E4A184832F00BF91EB18C
:10376800A36A23F08003A3621320134CA36ADE0725
:1037780004D51248174932F05AFA1420A36A9C0655
:1037880004D50E48144932F052FA15200A4B9A6AA9
:10379800D10658BF9A6A9A6A920642BF5A6A22F4B8
:1037A80000525A629A6A42F0FF029A6200232B7012
:1037B80070BD1020BAE700BF00ED00E020B104089A
:1037C8005E57050874570508A7570508BA5705082E
:1037D800D2570508E85705080758050810B5244CBE
:1037E8002449254832F023FAA36A99013ED5224894
:1037F800224932F01CFA1E20A36ADA0104D51E48B9
:103808001F4932F014FA1F20194CA36ADB0204D5B1
:1038180019481C4932F00BFA0220A36A1C0304D58C
:103828001548194932F003FA2120114CA36A5903AB
:1038380004D51148154932F0FAF92220A36A9A03EF
:1038480004D50D48124932F0F2F92320084CA36A36
:10385800DB0304D508480F4932F0E9F92420A36AAC
:103868006FEA03436FEA1343A36210BD1D20C3E749
:1038780000ED00E03658050820B104084E58050848
:10388800615805087B580508A5580508C358050858
:10389800E85805080259050870B5294C06460D4632
:1038A8002848294932F0C3F9A36AD9043CD52548E8
:1038B800264932F0BCF91720A36A1A0504D5214815
:1038C800234932F0B4F918201D4CA36A9B0512D580
:1038D8001C48204932F0ABF9A36BA26A100409D541
:1038E80001211D4A174832F045F81EB1A36A23F496
:1038F8000043A3621920124CA36A590504D5114844
:10390800164932F094F91A20A36ADA050ED50D4843
:10391800134932F08CF91B20094A936A43F47F4318
:10392800936200232B7070BD1620C5E7A36A9B0421
:10393800F2D504480B4932F07AF91C20ECE700BFB5
:1039480000ED00E020B104082D5905084359050889
:10395800A7570508545905086D59050882590508DF
:103968009D590508075805082DE9F0418AB0654BAF
:103978000446D3F80480002600AFC8F3080586F390
:103988001188BFF36F8F02F07F43B3F17F4F07D1E8
:1039980002F00C03082B12D15B495C4832F047F95E
:1039A800002634460023FB71EB1E092B00F28980A8
:1039B800DFE803F00A7F827B878787878785100780
:1039C8004CBF0C460126EDE75149504832F02FF91B
:1039D80000234C4DFB71EB6A9A0705D54D494B48BE
:1039E80032F025F9002331E0EB6A002B01DA4A496D
:1039F800F5E7EB6A5B00F5D54849444832F017F91A
:103A08006B69A26943F480736B61BFF34F8FBFF397
:103A18006F8F6B6932F8022C23F480736B61BFF3EC
:103A28004F8FBFF36F8F4DF602739A4207D0AB6A80
:103A3800DBB26BB30120F91DFFF768FE37E023689E
:103A48000121374A314831F095FF2368FA79DAB90C
:103A580007F1080504F1200C2A462068616808343B
:103A680003C264451546F7D17A6A002E45D0C2F3E1
:103A7800080121B96FEA52226FEA42227A62184697
:103A880007F10801FFF7B2FD2837BD46BDE8F08110
:103A9800AB6A13F47F4F04D00120F91DFFF7FCFE39
:103AA80005E0AB6AB3F5803F9CD3FFF797FE03466A
:103AB800CCE70020F91DBFE70020F91DEEE7194902
:103AC8008DE7194A18F4F87FE8468AB0174B18BFF3
:103AD80013466A461649103DC2E905134FF40073B0
:103AE8001384144BD56142F8103F00234FF4115151
:103AF8000648FFF7B5F9C54674E722F4FF7222F0CD
:103B08000102BBE700ED00E0E359050820B1040815
:103B18000E5A0508255A0508465A0508545A050834
:103B2800735A05088F5A0508CA590508B559050872
:103B3800B35A050804000001064B5A6942F0100206
:103B48005A615A6942F480625A615A6922F008023D
:103B58005A61704700ED00E0EFF30880EFF3098148
:103B680001B57246FFF700FF01BD00BF0A4880F3A8
:103B78000888102080F3118808484FF40061401825
:103B880080F30988EFF314800221084380F3148836
:103B9800BFF36F8F00F0C4F8A8B800208850002049
:103BA800BFF34F8F0549064BCA6802F4E06213431E
:103BB800CB60BFF34F8F00BFFDE700BF00ED00E013
:103BC8000400FA05084B9B6883420BD1EFF3058389
:103BD80043B1064B5A6842F080525A605A6A22F43E
:103BE80000425A620AF0D8B85036002000ED00E0D2
:103BF80016498A684FF030001044EFF3098C80E8CA
:103C0800F01F102080F31288BFF36F8F104F4FF012
:103C180000664A698A603E60D2F890000D4C2060C8
:103C2800D2F894000023C2F8943080F3118802F18E
:103C3800300090E8F01F8CF3098802F1000004B509
:103C480032F001F8BDE8044070470000503600200B
:103C580004ED00E0C82500201EF0040F0CBFEFF3B0
:103C68000880EFF30980816911F8021C0229FFD04E
:103C780001B5724631F0D0FF01BD00BF0028ACBFCE
:103C880000F16040064B4FEA0111C9B2ABBF00F525
:103C9800614000F00F0080F800131954704700BF0E
:103CA80014ED00E040B2002807DB01234109034A74
:103CB80000F01F00834042F82130704700E100E027
:103CC80040B200280CDB01220649430900F01F001E
:103CD8008240203341F82320BFF34F8FBFF36F8F0B
:103CE800704700BF00E100E0054B420953F822206D
:103CF800012300F01F0003FA00F01040704700BFD6
:103D080000E100E0044B054A23F07F039360BFF312
:103D18004F8FBFF36F8F70470000000800ED00E081
:103D280008B5FFF7EFFF0B4AD2F8883023F4700389
:103D3800C2F88830EFF3148323F0040383F3148864
:103D4800BFF36F8FFFF72AFCFFF734FC00F048F849
:103D580009F01EF800ED00E042F8203C009B0B49FA
:103D680042F81C3C019B21F0010142F8183C029BDF
:103D780042F8081C42F8143C4FF0807342F8043CA7
:103D88000023203A0265C0F894307047D127000814
:103D980000B50E4B15469860D0F890200C4B0E4697
:103DA8001A60D0F8803083F30B882C4686F3098894
:103DB8000020044B98472046002100220023024C93
:103DC800204700005F5C0308D12700085036002018
:103DD800C82500201022014B1A61704700ED00E051
:103DE800002310210348C2180133522B82F8001314
:103DF800F9D1704700E100E008B5EFF30583064A02
:103E0800103B02EBC30152F8330049688847BDE80C
:103E18000840FFF76BBC00BFC00B002001480068DA
:103E280070470000C82500201FB5094C094A2346E1
:103E38000121094800F012F900230393074B0121DF
:103E4800E41A01A80193029400F012F904B010BD1D
:103E58000000072000000020D0B2040880110020D4
:103E680010B50C7A0B6804F01F0223F01F031A43E5
:103E7800CB68640923F01F03054943EA440343F070
:103E88000103C1F89800C1F89C20C1F8A03010BD0A
:103E980000ED00E010B50A4BD3F89030C3F30723C8
:103EA800013B984208D901210346064A064831F0E9
:103EB80061FD6FF0150010BDFFF7D2FFFBE700BFF3
:103EC80000ED00E0CA5A050808B104082DE9F04FD2
:103ED8008946144606464FF00008514D85B0C8453E
:103EE80027DAD6F804A0BAF1000F44D0BAF11F0FB0
:103EF80017D91AF01F0F14D1D6F800B01BF01F0FF6
:103F08000FD1584631F0BBFE07460AEB0B000138CB
:103F180031F0B5FE874210D06FF01507414A3B4695
:103F280001E04346404A0121404831F023FD6FF04B
:103F38001504204605B0BDE8F08F17F1160FEDD037
:103F4800BC42EBDDC5F89870D5F89C10C5F89870A0
:103F5800D5F8A03021F01F0143F01F0BD6E900323D
:103F68001A44994202F1FF3A1DD1D34507D131468F
:103F7800F8B231F08DFE08F101080C36AFE7314692
:103F8800C5F89870D5F89C3022F01F0203F01F0383
:103F98001343C5F89C30E0B231F07AFE10F1160FE9
:103FA800C5D0441CE7E7C5F89870D5F8A020013BB8
:103FB80023F01F0302F01F021343D3453146E0B23A
:103FC800C5F8A030E8D031F063FE10F1160FAED07E
:103FD800C5F89870D5F89C209DF808300BF1FF3B88
:103FE80062F304038DF80830D5F8A0309DF8082056
:103FF8005B0863F347128DF80820D6E900321344B2
:10400800009323F01F035B44A3EB0A03013023F062
:104018001F036946C0B20393FFF73CFFBEE700BF2A
:1040280000ED00E0165B0508F05A050808B1040821
:104038000522044BC3F89420BFF34F8FBFF36F8F53
:10404800704700BF00ED00E0BFF35F8F0022024B16
:10405800C3F89420704700BF00ED00E010B5034C92
:104068002278FFF733FF207010BD00BF113E0020FB
:104078002DE9F74F294D8A4606464FF00008AB4612
:10408800274FD0451BDAD6F80490B9F1000F3FD07E
:1040980031680846019131F0F2FD0199044609EBB7
:1040A8000100013831F0EBFD84424FF014021D4B42
:1040B80008D002FB08F36FF015024BF8032003B099
:1040C800BDE8F08F14F1160F2C60F8D01978A142D2
:1040D800F5DD02FB08B0C7F89840C7F89840D7F854
:1040E8009C4000F10801007B64F304000871D7F8D4
:1040F800A0000C79400860F347140C71D7F89C10A5
:1041080021F01F016960D7F8A01021F01F01296173
:1041180008F1010814350C36B3E700BFCC250020A0
:1041280000ED00E0113E0020F0B55349534CD1F8A2
:1041380090302568C3F307239D4287B000F2998029
:104148000020FFF781FF4E4BC1F8C030854216D1E1
:104158004C4C01A82570FFF741F9002506464A4F47
:10416800AE4213D1002023784349D1F89020C2F3FE
:104178000722934277DBFFF75BFF002046E0616888
:1041880001EB0011FFF76CFE0130DFE70199280110
:1041980001EB0513DA683A40B2F1807F52D00AD8B1
:1041A800B2F5001F34D0B2F5800F3ED0B2F5801FB3
:1041B80012D00135D4E7B2F1006F43D0B2F1805F7D
:1041C800F7D15A689B680958013B22F01F00034445
:1041D80023F01F03012032E05A689B680958013B0D
:1041E80022F01F0003440120844623F01F0340EA05
:1041F8004C10CDE902218DF8100002A92078059312
:10420800FFF748FE00282ADA6FF0150007B0F0BD66
:104218005A689B680958013B22F01F0003444FF07D
:10422800020C012023F01F03E1E75A689B68095834
:10423800013B22F01F000344022023F01F034FF02C
:10424800000CD4E75A689B680958013B22F01F000C
:1042580003444FF0030C012023F01F03C7E7237822
:1042680001332370A5E7C1F89830C1F8A0000133E5
:104278007BE74FF0FF30C9E700ED00E0DCB204084F
:10428800AAFF4400113E00200000F0FFF0B587B0FF
:1042980007460E4614460021102268461D4646F081
:1042A80081FB02238DF80230054B2A4621466846D9
:1042B800CDE9047601932EF009FB07B0F0BD00BFED
:1042C800D15C030808B5024B1B689847002008BD5D
:1042D800E0250020034B044A1860937843F002035A
:1042E80093707047E02500205402002008B5054867
:1042F80030F071FF002383F31188BFF36F8F04231D
:10430800184602DF485B050808B50649064821F04B
:104318000701C1F1005202F5E02230F0ACFE0020A6
:1043280008BD00BF07D50020E42500204FF0FF326C
:104338004FF0FF33014808F0C7BE00BF64020020F9
:10434800014808F035BF00BF6402002038B50546B3
:10435800FFF7ECFF2A460821074830F0D8FD04464D
:1043680028B925B1FFF75AFD0C22044B1A50FFF764
:10437800E7FF204638BD00BFE42500200C00000000
:1043880038B504460D46FFF7D1FF21462B460822D3
:10439800074830F038FE044628B925B1FFF73EFD3E
:1043A8000C22044B1A50FFF7CBFF204638BD00BF44
:1043B800E42500200C00000010B50446FFF7B6FF06
:1043C8002146034830F042FDBDE81040FFF7B8BF72
:1043D800E425002070B541690446867A0A4D59B132
:1043E800437ADB0706D42C2303FB06535B6A1B685E
:1043F8009B689847002363612C20214606FB0050E8
:10440800BDE8704035F0EEB8B40F00202C22024B06
:1044180002FB0030704700BFB40F00202C21827AC5
:10442800054B01FB02339A6A1B7F801A1B3323F06A
:104438000303B0FBF3F07047B40F002038B52C2409
:10444800827A064B04FB02335B6AD3E901240C60D1
:104458001568FFF7E3FF04FB005038BDB40F0020D8
:104468002DE9F04385B00546684690461C46039101
:1044780035F0BEFADDE90067EFF31189102383F305
:104488001288BFF36F8F6B8B002B41D02A8B9A4217
:1044980025D900220023284608F0DAFE0446F0B1A8
:1044A80089F31188BFF36F8F039B002B41D03246ED
:1044B8003B46684635F0C1FA2C21A27A254B2046A6
:1044C80001FB02335B6A03A91B681D68DDE9002351
:1044D800A847606170BB2046FFF77CFF24E0698B2A
:1044E8004B1E6B8389F31188BFF36F8F2B7F2A8B49
:1044F800AC6A1B3323F00303521A02FB0344154B27
:10450800154AEB1A9B105343A3722B7FE372CBE738
:1045180089F31188BFF36F8F23464246284608F077
:1045280097FE04460028BFD10024204605B0BDE808
:10453800F0836361012300252381039B294663825D
:10454800E27A656004F1180046F02CFA6369258266
:10455800E360EAE7B40F0020A38B2EBA70B52C25D0
:104568000C4C00B970BD037A4668002BFAD0013BA9
:10457800DBB20372002BF5D1C3604360837A05FB7D
:1045880003431B6A13B198473046EAE7FFF722FF57
:10459800FAE700BFB40F0020F7B506460D461446EB
:1045A800124F384634F02AFEE0B1BB68314638462F
:1045B8001B68AAB29847002802DB002003B0F0BDB0
:1045C800002CFBD1AC42F8D22F1B042F28BF0427A4
:1045D80006F07EFB3A46019001A9301946F0BBF976
:1045E8003C44EFE76FF01200E8E700BF44AE040870
:1045F80038B5044609F0C0FA204631F0F1FBA0694D
:10460800C8B194F87030DB070DD50221144A15485B
:1046180031F0E4FB6FF07705201D31F0E8FB09F07D
:10462800BFFA284638BD34F0E9FD38B901210E4AF1
:104638000C4831F0D3FB6FF01205EDE7204601F08E
:104648002FF805460028E7D128220146A01846F091
:10465800A9F994F8703043F0010384F87030DBE76F
:10466800685B0508A0B10408925B050838B50546E3
:1046780009F082FA284631F0B3FB95F87030DA0772
:104688000DD40221184A194831F0A8FB4FF0FF3425
:10469800281D31F0ACFB09F083FA204638BD9B0792
:1046A80007D50221124A114831F098FB6FF07704C0
:1046B800EEE7A86932F0B1FD044628B101210D4AA0
:1046C8000A4831F08BFBE3E7284631F01AFD04462F
:1046D80018B1A86932F0CAFDDAE795F8703043F0EE
:1046E800020385F87030D3E7B55B0508A0B104086C
:1046F800DB5B0508015C050838B590F870300446A6
:104708009B0708D40221144A144831F067FB6FF064
:104718007705284638BD31F063FB0021204601F0BB
:104728005DF920B101210E4A0C4831F057FBA06910
:1047380032F09CFD054620B101210A4A074831F0B4
:104748004DFB94F87030201D6FF3410384F87030EE
:1047580031F04DFBDDE700BF1D5C0508A0B1040882
:10476800445C0508625C05082DE9F04385B00746FE
:10477800884614461E4631F03CFB05468EB1384645
:1047880031F03CFB012809D0FFF748FB6FF08502A8
:10479800334B1A50002005B0BDE8F083B5FA85F513
:1047A8006D09013429463846E2B231F0C6FC81462B
:1047B80030B9012123462B4A2B4831F0DBF8E3E7D7
:1047C80044684EB12068616801AB03C3227A01AC2A
:1047D8001A7007238DF8053008F10C06304631F0C1
:1047E800ECFA2278824203D9304631F0E6FA0246E2
:1047F8002146304631F0BFFAD9F80C90B9F1000FD4
:1048080009D1B8F81010FB8D9942C3D93046C91A9E
:1048180031F0CCFABEE7D9F8040083681B6B13B9F2
:10482800D9F80090EAE7294698470028F8D0041FED
:1048380054F8043F002BF3D01B78002BF0D03046FF
:1048480031F0BBFA23681A78824203D9304631F036
:10485800B4FA82B23046216831F08DFAE8E700BF39
:104868000C000000925C050880B104082DE9F041B5
:1048780090F82830044603F01F03012B0F4600F17F
:1048880028061BD0022B05D043BB90F8291031F025
:10489800C1FC03E0818DC9B201F0FCF90546E8B11D
:1048A800304631F0DDFB024668688368A2B99B6830
:1048B8004BB13A463146BDE8F0411847818DC9B23F
:1048C80031F08FFCEAE76FF08503FFF7A7FA0F4A8C
:1048D80013500020BDE8F081DB68E9E7204694F832
:1048E800291031F0D2FA02460028ECD0304631F0D7
:1048F800B7FB40B91369002BE5D03A46314620464C
:1049080098470346E1E7D368F5E700BF0C000000CD
:104918002DE9F04F95B00D46097E02AF00F128034E
:1049280031F0800804469146BB600BD00121A74AAC
:10493800A74831F0ABFB6FF0040840464C37BD4642
:10494800BDE8F08F6B7E03F00102B9F1000F17D0BC
:1049580019F10C0F14D0B2B919F1710F03D128460F
:10496800FFF7FCFDE9E79B4A0B4699480121CDF882
:10497800009031F009F82846FFF7F0FDC846DCE75B
:10498800002A00F0B284002940F072842B8A072B99
:104998000FD9EA681368A3625368E362D5F804A0E4
:1049A800E28DBAF1000F17D18B4A0121884831F006
:1049B8006DFB0121894A864831F068FB2846FFF7DC
:1049C800CDFDB86831F04CFB0346A069002B00F020
:1049D800A384802100F0A9BC04F1280031F040FB39
:1049E800E0B99AF8193032B198071DD46E4688B0EC
:1049F80002AA7B4B05E05E0716D46E4688B002AA71
:104A0800784BC2E9053A032342F8103F70480B4639
:104A18004FF4C251FEF724FAB546CAE70AB9724AFA
:104A2800C3E79AF81930DFE72946002031F08BF9FF
:104A3800054628B9684A0121654831F027FBC0E7D7
:104A4800FFF7ECF9002394F82820684E12F0600F65
:104A58008351C2F3411307D0032B40F0E981FFF7DC
:104A6800DDF96FF085033EE004F1280031F0F8FA33
:104A780094F82930002840F07781013B0A2BEED8C2
:104A880001A151F823F000BF534C0008674A000801
:104A9800D74C0008674A0008BD4A0008674A000862
:104AA800674A0008674A0008614B0008674A00081F
:104AB800054C0008A069618D03697F29D3F880300F
:104AC800CDD8A28D002ACAD1E28D002AC7D194F888
:104AD8002820D206C3D194F83420022A05D1FFF742
:104AE8009DF94FF0FF33335018E01A070BD5C9B2C0
:104AF80031F0EEFA804648B1638D01213C4A3448D2
:104B080030F038FF2BE7012384F83D3094F8343037
:104B1800012B1FD1638DEBB984F83430FFF77EF990
:104B28003358002B7FF44AAF0123B868236331F070
:104B380097FA002840F08983E38D002B00F08583E5
:104B48002946002031F0FFF80546002840F0798317
:104B5800284A70E70123DFE7204631F04AF9628DE1
:104B68000146FF2A3FF67BAFE38D002B7FF477AF3A
:104B780094F82830DB067FF472AF94F83430002BB9
:104B8800ADD02AB12046D2B231F0FDFA0028A6D025
:104B9800618D94F83C308B42C0D02046C9B200F0F9
:104BA8001DFF638D804630B101210090124A0848EC
:104BB80030F0EAFED3E61A1E14BF022301230521B2
:104BC800204684F8343031F04DFCA7E7B85C05087E
:104BD80080B10408D95C0508085D05086B5D050807
:104BE8002A5D0508395D05084A5D05080C000000C6
:104BF800825D05084C5E0508A45D050894F8283018
:104C080003F01F03012B7FF42AAFE38D002B7FF401
:104C180026AF628DFF2A3FF622AFA18DFF293FF60E
:104C28001EAF94F83430022B7FF459AF2046D2B22D
:104C3800C9B231F058FB10F1020F804640F04B81A9
:104C4800FFF7ECF846F8008068E7E38DA18D002BAC
:104C58007FF405AF94F83430002B3FF440AF012BBC
:104C680010D100297FF43BAF12F01F020DD1638DE4
:104C7800012B7FF453AF94F870306FF3C30384F8BB
:104C880070304BE712F01F0217D0022A7FF446AFAC
:104C9800B4F82A80B8F1000F7FF440AF5FFA81FAC8
:104CA8005146204601F05CF90346FFF7B7F8335048
:104CB800013306D14FF0FF3851E600297FF40FAFDA
:104CC800D5E742465146204631F0D0F926E7E38D34
:104CD800A18D002B7FF4C3AE638D5FFA81F8022BA0
:104CE80013D194F8283003F01F0358EA03037FF424
:104CF800B6AE0122A069090A31F0CAF900287FF48A
:104D0800AEAE012384F83D3008E794F8340000285B
:104D18003FF4E5AE01280DD100297FF4E0AE12F092
:104D28001F020AD1012B7FF4F9AE94F8703043F0DA
:104D38000803A4E712F01F0212D0022A7FF4EEAE95
:104D4800002B7FF4EBAE4146204601F0E7F803461E
:104D5800FFF764F833500133ACD001224146B2E783
:104D680000297FF4BCAEDDE70A2B3FF678AE01A13F
:104D780051F823F0A94D0008674A0008674A00085F
:104D8800674A0008674A0008674A0008294E000871
:104D9800674A0008E3510008674A000811520008F2
:104DA800E38DA18D022B7FF45AAE94F83430002B9A
:104DB8003FF495AE012B10D100297FF490AE12F08C
:104DC8001F020DD194F870304FEA930808F00208DA
:104DD800C3F3001348EA030806E012F01F0210D0DC
:104DE800022A12D04FF0000805F10C0A504630F0A4
:104DF800E4FFE38D98420ED2FFF710F86FF00B0333
:104E080071E600297FF46BAEDCE72046C9B231F0C9
:104E180008FB8046E8E74146504630F0BDFF7DE696
:104E280094F82810628DC8064FEA1223D2B204D033
:104E380029462046FFF71AFD4CE0013B0E2B3FF6B2
:104E48000EAE01A151F823F08D4E0008D34E000894
:104E5800ED4E0008674A0008674A000847500008F6
:104E6800E94E0008674A0008674A0008674A0008D0
:104E7800674A0008674A0008674A0008674A000846
:104E8800DF50000805F10C084046B4F82EA030F0B9
:104E980094FF82450AD2B4F82EA0204630F0A9FF2C
:104EA80048B101287FF4DBADA16F05E0404630F042
:104EB80084FF8246F1E7616F002900F0DC800A7800
:104EC800524528BF5246404630E000232946204636
:104ED800FFF74AFC8046B8F1000F7FF440AD1DE6AD
:104EE8000123F3E70321204631F00EF8824600281B
:104EF8003FF4B5AD31F0AFF8E38DF0B9BAF814204E
:104F080098463A85DAF8102005F10C0A12885046BE
:104F18007A8530F052FF80450BD2E08D97F8282033
:104F280007F12801824228BF0246504630F023FF8D
:104F3800F4E5504630F041FFF0E79B4600233B750F
:104F48009AF81530DAF808207B75C34B1340C34A2A
:104F5800934263D1102107F1180004F0DFFA00280A
:104F680042DB07F1280310289E4628BF1020DFF8EF
:104F7800F0C207F11802804503F102033DD3800017
:104F880002303875C7F80CE005F10C0A504630F0CD
:104F980014FF97F81480D84528BFD846404503D257
:104FA800504630F00AFF8046B8F1020FC34628BFCA
:104FB8004FF0020B50465A4607F1140130F0DBFE61
:104FC800A8EB0B08D7F80CB04FEA58030BEB5802C4
:104FD8005A452AD118F0010F3FF4A0AD5046FA689F
:104FE800D15C30F0D1FE99E558307FF438AD01211D
:104FF8009C4A9D4831F04AF831E512F8011B08F146
:1050080001084FEA111A01F00F011CF80AA01CF858
:10501800011003F802AC03F8011CACE79AF814304D
:105028003B75DAF81030FB60AEE750461BF8011B01
:10503800C7E9002330F0B0FED7E90023C8E72046CF
:1050480030F0D7FED4E91D83002808BF9846002316
:10505800C7F82A30C7F82E300A2387F828300623E5
:10506800204687F8293030F0C9FE01287FF4F7ACD4
:10507800B8F1000F02D16FF0150870E4B8F80230EB
:105088007B8598F8043087F82C3098F8053087F835
:105098002D3098F8063087F82E3098F8073087F8C2
:1050A8002F3098F8113005F10C0887F83030404659
:1050B800B4F82EA030F081FE824508D2E08D97F832
:1050C800282007F12801824228BF0246FBE6404615
:1050D80030F073FEF3E7204630F08BFE20B1012854
:1050E8007FF4BDACA36F00E0636F002BC3D05B8877
:1050F800B3F5007F7FF6B3AC5C4B04F15002BB62A2
:10510800002387F82C3004F15003FB60236D9A428A
:1051180060D105F10C0A504630F04FFEB7F82A80EE
:10512800E38D984528BF9846404503D2504630F055
:1051380044FE804697F828205046424528BF4246FC
:1051480007F1280130F017FEB8F1050F94BFA8EB5E
:105158000808A8F10508B8F1000F3FF4DFACD4F84F
:1051680050B0FB689B453FF4D9ACBBF1000F3FF44E
:10517800D5AC9BF815300F2B15D19BF81420504651
:10518800424528BF4246DBF8101030F0F4FD9BF88A
:105198001430434594BFA8EB0308A8EB0808B8F1FE
:1051A800000F3FF4BBAC636D5B453FF4B7ACDBF875
:1051B80000B0DAE75A7D0F2A08D11A7D798D0A44A2
:1051C8007A8597F82C20013287F82C20626D9A4254
:1051D8009FD01B68002BEDD19BE794F8343094F8EE
:1051E8003CA0002B3FF47BACE38D012B7FF437AC64
:1051F80005F10C08404630F0E0FDE38D9842FFF4DD
:10520800FBAD51464046ECE694F8283003F01F0306
:10521800012B7FF464AC204630F0A3FF00283FF454
:105228005EACA38D4268FF2B3FF619AC12799A4207
:10523800FFF415AC0F2B3FF612AC234493F83EA0B5
:10524800D2E76B7E59077FF57BAC2946204600F0F4
:105258001DFE8046FFF771BB00FF0200000302003D
:10526800695E0508C75D050880B10408050F0500DB
:105278005A077FF5A6AB80297FF4A3AB2846FFF732
:105288006DF9256B012D40D194F83D30002B3FF48A
:1052980054AB94F82930052B0CD1618DA069C9B2A3
:1052A80030F016FF804628B1638D234A29462348EB
:1052B80030F060FB94F82930032B11D1638D022B59
:1052C8000ED1A18D00220D0A2946A06930F0E0FE1A
:1052D800804628B101212B46194A184830F04AFB6C
:1052E800002384F83D30FFF728BB5B077FF569ABE7
:1052F8000029C0D1236B012B3FF431AB0221114AA5
:105308000E4830F0C3FEFFF72ABB02210E4A0B48B5
:1053180030F0BCFEFFF711BBE38D002B3FF459AB17
:1053280019F10C0118BF0121C90131F0ABFE0023AE
:1053380080462363FFF701BB825D050880B104083E
:105348000A5E0508E95D0508285E05080B7810B4B3
:10535800062B14D10369D3F89C20EFF31184102392
:1053680083F31288BFF36F8F00204B681860506A70
:1053780058B9C2E9083384F31188BFF36F8F00224C
:105388000023034810BC34F033B803605362F2E7DB
:10539800300F002030B589B0002200230024CDE969
:1053A80006236FF007034FF48062CDE90334CDE99B
:1053B8000144154B15490094154808F01DFA154984
:1053C800134834F0AAF9144B14498B4207D3002030
:1053D800134B14498B420CD3002009B030BD03F1A4
:1053E8001402D2E8EF0FC2E8E54F002DF9D11833C7
:1053F800EBE703F11402D2E8EF4FC2E8E50F002D06
:10540800F9D11833E6E700BF855400088844002026
:10541800A01900202A7C0508B4100020FC100020E8
:10542800FC1000204411002038B50D4630F099FEDC
:1054380030B90121BDE838400E4A0F4830F091BA22
:10544800C46804B938BD2B78032B07D0052B0CD0C2
:10545800022B08D1606883689B6902E060688368F2
:105468005B6903B198472468EBE760688368DB6988
:10547800F7E700BF835E050890B104082DE9F047FF
:10548800102684B0DFF8FC8100AF4FF0FF334FF0F7
:10549800FF324046391D07F0B3FDFB681B69D3F89E
:1054A8009C40236A73B1EFF3118386F31288BFF32C
:1054B8006F8FD4F820A0BAF1000F1BD183F31188A5
:1054C800BFF36F8F3B79062BDFD0072BDDD801A206
:1054D80052F823F073550008675500089B550008DB
:1054E80079550008D1550008BD55000893540008A7
:1054F8007B560008616ADAF800208A45226208BFF4
:10550800626283F31188BFF36F8F9AF8183051469F
:105518005D062046DAF81E201ED1FFF7F9F9054688
:105528000028BED0E9468AB06A469AF81830C2E91F
:10553800073A05235449C2E9051042F8103F0023F1
:105548004FF421515148FDF78BFC2A46CD460721DF
:10555800204630F087FFA4E730F053FEDFE7002253
:105568000121204630F07EFF8FE700221146F8E740
:1055780094F8703043F0040384F8703094F83430B1
:10558800022B03D12046391DFFF74EFF00220321CD
:10559800E7E794F870306FF3820384F8703094F87A
:1055A8003430022B03D12046391DFFF73DFF00227E
:1055B8000221D6E794F83430022B7FF466AF2046F8
:1055C800391DFFF731FF60E794F87030D4F8189070
:1055D8006FF3820384F87030D9F808A0D9F8103036
:1055E800A033D3E8AF3F9A071BD54846DAF83C30DA
:1055F8009847DAF824300021484698470546DAF8F3
:105608004030484698477DB1214A01211F4830F073
:10561800A8F900220421204630F024FF2A46072159
:105628009FE74FF0FF35EFE72946204600F0D6F90F
:10563800054608B1174AE8E78021204630F0EEFE1B
:1056480020B10121144A114830F08BF9A06931F0DA
:10565800CEFD0022831E5842584194F87030042130
:1056680023F0680343EA401384F8342084F8703048
:1056780077E70121094A054830F073F90621BA682D
:105688006FE700BF300F0020B25E050890B1040834
:10569800DC5E05080A5F0508365F0508535F0508E4
:1056A80038B5024605460C49806931F0FFFD0446CD
:1056B80030B10121094A0A4830F053F9204638BD73
:1056C80085F83C00284600F047F904460028F5D044
:1056D800A86931F01AFEF1E755530008635F050821
:1056E80090B104082DE9F8434FF0010805460C462F
:1056F80046462068002840D068F07F02D2B21146A2
:105708005FFA88F730F003FDE0B1D5F80090114654
:10571800484630F0FCFC48B9134619480121194A9B
:1057280030F028F96FF01500BDE8F88322F0800208
:10573800103206FA02F229EA02032B60236823EAF0
:10574800020323603946206830F0E1FC80B12A6802
:105758003946104630F0DBFC08B94346DDE706FA67
:1057680008F122EA01022A60236823EA0103236080
:1057780008F10108B8F1100FBBD10020D4E700BF31
:10578800B8B104088A5F05082DE9F04F00268FB0EC
:105798005368CDE90621D468099002930C960396C4
:1057A80074B9039B029A09339BB293701B0AD37096
:1057B800069B1671DC68002C40F0BC80A146A3E073
:1057C800002560680D9583681B6B002B00F0A38093
:1057D80007999847002800F09E80C4E9035535468C
:1057E800071F57F8043F0BB11A789AB9B54240F22F
:1057F8008F80E3680D9A1343E360606883689B6A4F
:10580800002B00F08A8098478146002800F08880A5
:105818004E4A75E05A780B2A08BF9D703B685A7843
:10582800042A10D1E2680D990A43E260DA78002A66
:1058380059D101229D702369AA4013430135236180
:10584800EDB200230D93D7F8008098F80130052BAE
:10585800C7D16FF012094FF0010B099B9B690893A0
:1058680098F8051098F804200C9B42EA0122ADF83C
:105878002E2098F902205FFA8BFA002AB8BF4AF066
:10588800800A51461846049330F041FC90BB0D9BAA
:1058980051461846059330F03AFC58BB98F8063044
:1058A80098F803205146009308980DF12E0331F023
:1058B80060FB8146F0B901231AF0800F1EBF2AF061
:1058C800800110318B400498059908BF03FA0AF348
:1058D800BDF82E2019431843CDE90C0188F802A021
:1058E800A8F804207DE76A1E9A700DA90CA8FFF796
:1058F800F9FEA6E70BF1010BBBF1100FB0D1144A6A
:105908000121144830F02DF848460FB0BDE8F08F5B
:105918006FF01509F3E735466FE76FF0850977E70C
:105928006068079930F03DFC039B2E4603442468C9
:10593800039335E7E36804F10C01A3600CA8FFF7B3
:10594800D1FE81460028DFD1246834E7CB5F050803
:10595800A75F0508B8B1040870B5836905461B69D7
:10596800426F93F88030C3F34113022B0CD0032B02
:105978000CD0012B0CBF10230823D3712E6E3EB917
:10598800AE6DBEB9344611E02023F6E74023F4E7B4
:10599800324601212846FFF7F7FE044640B17368F6
:1059A8005B790B4A01210B482FF0E4FF204670BDBC
:1059B8003668E4E7324600212846FFF7E5FE04464C
:1059C80018B173685B79044AECE73668D9E700BF19
:1059D800EF5F0508B8B10408126005082DE9F04129
:1059E80005460E4630F005FA95F83C30804633B34C
:1059F800284630F0B6FB0746F0B10146284630F09D
:105A080020FC10220446002105F13E0044F0CAFFA4
:105A1800002385F83C30FF683FB984B119491A481A
:105A280030F07EFB2046BDE8F081786883685B6AC9
:105A380003B198473F68EFE76FF03C04EEE71EB903
:105A480085F83C600024EDE732464146284630F0B0
:105A580074FB074690B10246284630F01CFC044609
:105A68000028DFD185F83C60FC68002CEAD060682B
:105A780083681B6A03B198472468F6E76FF03C0413
:105A8800D0E700BF445C050878B104082DE9F0416F
:105A9800054688461446576830F046FB95F870303E
:105AA800D8070BD54F49504830F03AFB6FF00F0834
:105AB800281D30F040FB4046BDE8F081B8F1010FE9
:105AC80015D1284630F09AF930B94849464830F09F
:105AD80027FB6FF08508EBE7FB7999061AD5AB69C8
:105AE8001B69D3F880309A070CD44149EEE7FB795B
:105AF8009B06F4D4B8F1000F0AD12B6E43BB05F115
:105B080058060BE0B8F1000FF7D0B8F1010F01D03B
:105B18003849DBE7AB6D83B905F1600600223368CD
:105B2800E3B96268B8F1000F3FD16B6F5B7C01335A
:105B3800DBB253716A6F537422E0A34206D12E4937
:105B4800294830F0EDFA6FF01508B1E71B68E2E775
:105B5800A34201D12949F3E71B68CFE79C4221D131
:105B68002368CAB972683360944200D17360002315
:105B7800236063685B790221214A1B482FF0FAFEF3
:105B8800A16819B3284630F0D9F98046D0B11D492B
:105B9800154830F0C5FA8BE7136073689C4208BF5C
:105BA8007260E4E71A461B68BAE7B8F1010F02D041
:105BB80001235371E4E7AB6F5B7C0133DBB25371B4
:105BC800AA6FB8E7A06830F046FAB87100232360DE
:105BD800736823B9C6E900444FF0000868E71C6001
:105BE8007460F9E76360050878B104088560050802
:105BF8003F600508A3600508C3600508E060050864
:105C0800FD6005081A610508F8B5054600AF21B31F
:105C180001290BD1184C194E2AE0636828461968E7
:105C2800FBF72EFBB0B11834B442F6D36C4688B0FB
:105C38006A46134BC2E905354FF400739383114B41
:105C480042F8103F00234FF4E2510F48FDF708F9DE
:105C5800A54600242046BD46F8BD0C4C0C4EE3E793
:105C6800636828461968FBF70BFB0028F2D0183444
:105C7800B442F5D3DAE700BFFC100020441100203D
:105C8800516105080300000188B10408B410002020
:105C9800FC10002070B5012501F07F0311F0800F82
:105CA80018BF10339D4090F834300446022B06D0BC
:105CB80001210C4A0C482FF054FE002070BD90F8CA
:105CC8003C6030F096F832460146204630F035FA0E
:105CD8000028F2D0C0680028EFD083681D42EDD1BB
:105CE8000068F8E76F61050888B104082DE9F843F2
:105CF80005460846114616469846FFF785FF0446AE
:105D0800002843D0284630F045FA95F87030DA0775
:105D180002D5204A012109E0D4F8049004F11407BF
:105D2800D7E8AF3FDB070CD502211B4A1B482FF0F1
:105D380018FE6FF00F04281D07F03AFA2046BDE858
:105D4800F883D9F804301BB1AB4201D0144AE1E71B
:105D580042463146284630F0F0F9A0B100232360CE
:105D680003696BB9C0E90344D7E8EF3F43F0010387
:105D7800C7E8E23F002AF7D10024C9F80450DAE75F
:105D88001C600461F0E76FF03C04D4E76FF0120484
:105D9800D4E700BF636005089461050888B104086A
:105DA800B66105082DE9F04F83B000AF7B6097F826
:105DB80030304C680E463B608146904630F019F80A
:105DC800A36801461B6B33B96FF0150420460C37E6
:105DD800BD46BDE8F08F204698470028F4D000243F
:105DE800051F06F10C0A55F8041F09B10B782BB9E9
:105DF800002C0CBF6FF03C040024E7E74B78042B21
:105E08000ED1002C3CD18B787A689342EBD1CB78B9
:105E18003A689342E7D10B79002BD7D00124E2E707
:105E2800052BE0D1002CDED0B8F1010F91F802B0BB
:105E380009D0B8F1020FF1D152465946D9F81800E5
:105E480030F0B7FA04E05246D9F8180030F095FA65
:105E580004460028E2D06D468AB06A46F368C2E973
:105E680007B3062307495062C2E9051842F8103FF4
:105E780000234FF441510448FCF7F2FFAD46A5E773
:105E88000024A3E7F6610508B0B104082DE9F04144
:105E98000B7E05465E060C4638D119062DD52FF027
:105EA800E8FF40B11B4801211B4A2FF05AFD4FF073
:105EB800FF30BDE8F0812846D5F87480268AEF8D3A
:105EC8002FF097FFF8B1421E534253419B01228A9B
:105ED8009AB1BE42324628BF3A46E98D91420CD962
:105EE800B2FBF3F103FB11223AB994F91830002BF5
:105EF800BEBF637E43F0080363762146A869BDE808
:105F0800F04131F01BB998F80730E0E76FF0150061
:105F1800CFE700BFA8B104083262050870B506468D
:105F280080690C4631F0AEF8054638B102212346A7
:105F3800094A0A482FF01EFD284670BD012214F0B8
:105F4800800F18BF24F08004B36B18BF1034A24030
:105F58001A43B263F0E700BF46620508A8B1040817
:105F680070B5054680690E4631F0B7F8044638B179
:105F780002213346054A06482FF0FCFC204670BD36
:105F8800314605F1380030F0EAF9F7E75D620508B7
:105F9800A8B1040870B50646EFF31181102282F308
:105FA8001288BFF36F8F1D4C236881F31188BFF3EC
:105FB8006F8F5B6893F87030DB0705D4BDE87040DD
:105FC8000822002307F0BCBBEFF3118382F3128889
:105FD800BFF36F8F256865B983F31188BFF36F8F9F
:105FE8002368D3B13046BDE870400022002307F093
:105FF80073BB61682A688D4208BF6260226083F3C0
:106008001188BFF36F8F686805F10801C369984765
:106018002946034833F089F9E2E770BDF0250020EE
:10602800BC0E002030B585B06C46054684E80600F5
:1060380000230022144803A906F044FF0246E8B9E9
:1060480094E80300039B5D60083383E80300EFF3E3
:106058001180102383F31288BFF36F8F039B1A609C
:106068000A4A516861B9C2E9003380F31188BFF365
:106078006F8F00220023064807F02EFB05B030BDC5
:106088000B605360F1E700BFBC0E0020F025002034
:106098000000002038B54B780469202B456820693A
:1060A80008D0222B19D0FDF7B9FE6FF08502104BEE
:1060B8001A5010E0CB88072BF5D1D3681A684260D4
:1060C8009A8802819B79837230F0F1F9224608217F
:1060D800284630F0D5F9002038BD4B880921C3F394
:1060E8004002838103F00103027643762246EFE7FC
:1060F8000C00000008B51346026910694A78212A85
:1061080012D133B9FDF78AFE6FF00B02094B1A5012
:1061180008E0CA88011D072A28BF072203F10C00DE
:106128002FF029FE002008BDFDF778FE6FF08502EC
:10613800004BECE70C00000038B5002405690E4957
:10614800EB6B05F14800C3E90144DC606B6BC3E904
:106158000144DC6033F0CFFA05F17800074933F0E9
:106168009EFA074905F1240033F099FA284630F0E1
:106178009EF9204638BD00BF9562000839640008C2
:10618800056500082DE9F341036906460D46D0F878
:1061980004801C690F7E002A32D00B8A713238487D
:1061A8000BBF02210121374A374A00933B462FF0A3
:1061B800EBFB30462F7E30F0EEF9874204D1042104
:1061C80004F1880030F068FA30462F7E30F0F1F99B
:1061D800874204D1052104F1880030F05DFA304689
:1061E8002F7E30F0CAF9874203D104F18C0007F002
:1061F800C1F82946404602B0BDE8F04130F00BB97D
:1062080030F0C9F9874214D12A8AE968606B2FF007
:10621800B1FA28B1E3691BB104F1240007F0ECF9E5
:1062280004F18800042130F037FA04F1780007F00F
:10623800E3F930462F7E30F0BCF9874215D1E36987
:106248001BB104F1240007F0D7F9052104F18800F7
:1062580030F022FAE36B5A89DB889A4205D0002293
:10626800002304F1480007F037FA30462F7E30F05B
:1062780084F98742BDD104F18C0007F01BF8B8E718
:1062880070B1040887620508AB6205082DE9F0477C
:1062980050F8483C00F140065B680746002130464C
:1062A800D3F8008030F063F9002854D0012130463B
:1062B80030F05DF900284ED1D6E8EF3F43F02002D8
:1062C800C6E8E12F0029F7D19B0644D4404630F0B8
:1062D80070F900220446002320482FF001FD0546EE
:1062E80050B93046052130F0D7F93846BDE8F047B7
:1062F8000822002307F0F0B98146047659F80C1FEC
:10630800428A57F80C0C2FF055FA044601464846C5
:106318002FF02BFD54B1D8F8040030F0B4F9B4FBD9
:10632800F0F303FB1044B4FA84F4640929464046A8
:1063380007F82D4C30F057F868B10121084A094890
:106348002FF00FFB2846FEF709F93046BDE8F04765
:10635800052130F0A1B9BDE8F08700BFB40F0020D7
:10636800CC62050870B1040838B503461B6940685B
:106378005D68AC68A37A84F8223094F82D3084F8EC
:106388002330696849B1237C3BB92FF0D7FD30B180
:106398000121054A05482FF0E4FA002038BD686855
:1063A8002FF059FE2074F8E7DE62050870B1040882
:1063B80073B5102504698DF80710EFF3118685F37E
:1063C8001288BFF36F8F0122E06B0DF107012FF0E8
:1063D800D1F986F31188BFF36F8F012814D033F0F9
:1063E80096F908B9A37EBBB901220E4BD3E8EF1F7B
:1063F800002903D1C3E8E02F0028F7D104D10221F6
:10640800094A0A482FF0ADFA0822002304F148008F
:1064180007F062F902B070BD0021082033F031FAAC
:10642800CBE700BFF82500200863050870B1040811
:1064380070B550F8782C00F110045268034600211A
:106448002046156830F093F800284DD001212046E9
:1064580030F08DF8002847D153F8442C68689388A9
:10646800918916695B1A9BB2F61A30F00CF9B042A2
:106478003AD8D4E8EF3F43F01002C4E8E12F0029EE
:10648800F7D1DB0606D5BDE870400221174A184847
:106498002FF067BA284630F07EF80022064600231F
:1064A80014482FF01DFC0446F0B10676686830F0F9
:1064B800EAF8638A984203D2686830F0E4F883B255
:1064C8002146284663822FF08EFF68B1284630F0B7
:1064D80062F8034606480121074A2FF04BFA204686
:1064E800BDE87040FEF73AB870BD00BF27630508E5
:1064F80070B10408B40F00204763050838B550F898
:10650800243C04465B681A6850F8083C33B9BDE877
:1065180038400121284A29482FF023BA002300F1E6
:106528006405838283830221284630F020F8B8B1BD
:1065380054E9023110699847637D1BB104F1540096
:1065480007F05AF80521284630F011F898B9637F0A
:106558006BB10022002304F1240007F0BDF80AE023
:106568000321284630F003F80028E1D1E4E714F8C5
:10657800093C002BEDD1022128462FF0F8FF38B155
:1065880023695A89DB889A4202D0204607F034F8FA
:10659800032128462FF0EBFF60B1A2699388918907
:1065A80012695B1A9BB29A4204D02046BDE8384073
:1065B80007F022B838BD00BF6C63050870B1040845
:1065C800D3B5002600270446CDE9006705482FF01B
:1065D8008BFB28B1230658BF0023047658BF0382DB
:1065E80002B0D0BDE00F00202DE9F04383B00023B6
:1065F8004FF0010805691C4C1C4E02AF28602B7730
:1066080085F8203005F12409B442234601D300203F
:1066180019E095F820201034CAB16C4688B01B6880
:1066280002AA1349C2E905134FF400739383114B6F
:1066380042F8103F104800234FF4E251FCF710FCD9
:106648006FF00B00A5460437BD46BDE8F08385F81A
:10665800208054F8043C4846009354F8101C54E930
:10666800032330F0B7FACFE7ECE30508FCE30508AD
:10667800F763050803000001C0B104081FB5002333
:106688000190CDE902334FF0FF324FF0FF3301A9FB
:10669800024832F0ADFE05B05DF804FB000F0020A3
:1066A80008B54B78FF2B07D14B882BB9CB881BB982
:1066B800FFF7E4FF002008BDFDF7B0FB6FF085028F
:1066C800014B1A50F6E700BF0C00000013B5144642
:1066D8004A780369FE2A14D14A8892B9CA8882B1D5
:1066E80093F820300BB1013BDBB201220DF1070119
:1066F80004F10C008DF807302FF03DFB002002B0AC
:1067080010BDFDF78BFB6FF08502014B1A50F5E7C2
:106718000C0000001FB5CDE9010103924FF0FF32D4
:106728004FF0FF3301A9034832F062FE002005B0A4
:106738005DF804FB000F00202DE9F04104461746E0
:106748000E46006830F0D1F831463A468046FFF7E9
:1067580037FFD4F87B300546DB1B0146C4F87B3095
:1067680020682FF040FE88B10B4A434601210B48B0
:106778002FF000F93146204630F05DF92846FDF744
:10678800EDFE2046BDE8F04130F021B9A37F01338A
:10679800A377BDE8F08100BF47630508C0B10408CE
:1067A8002DE9F74F0446006830F0B4F83027064664
:1067B8004FF02408E37F012B1FD82368D3F810A0DB
:1067C800D3F804909AF8611017FB01810AEB010BCA
:1067D800584630F025FA594602460190484630F0AE
:1067E800AFF89AF81F30054633B1019A5946121A84
:1067F800484630F0A5F8054615B903B0BDE8F08F56
:10680800204630F05AF82A46014681463046FFF7BE
:10681800D7FE0546014620682FF0E5FD88B10B4AF2
:10682800334601210A482FF0A5F82846FDF796FEC1
:106838004946204630F0FFF803B0BDE8F04F30F08D
:10684800C6B8E37F0133E377B4E700BF47630508C1
:10685800C0B104082DE9F04FDFF8EC9289B04FF091
:10686800FF324FF0FF33B94805A906F0C9FB059E72
:10687800069D3469002D40F09080257704F12406A8
:1068880094F820309D42C0F2828004F11803D3E8C6
:10689800EF2F22F00202C3E8E12F0029F7D1D3E855
:1068A800EF1F21F00401C3E8E21F002AF7D104F129
:1068B8001803D3E8AF3FDB07D1D5237F022B00F0C5
:1068C8009581032B00F08E8153BBDDF814A0DAF814
:1068D8001050EB7F23BB504630F01CF8804628460A
:1068E8002FF0EBFF4FF40072014606464046FFF7D3
:1068F80067FE0746014650462FF075FD002800F058
:106908006D8101214346924A92482FF033F8384668
:10691800FDF724FE3146284630F08DF830F057F860
:10692800A37F002B9BD1237F012B40F08481302350
:1069380004F1630694F86150304694F8621003FB42
:10694800054500F06BFA243502463146236928468E
:1069580000F082FA0646C4F88400284630F056F95A
:106968008046284630F057F90746284630F058F94F
:10697800E26D3044002A40F04281002840F03A811C
:10698800284630F074F9003818BF012033E130464A
:1069980030F033F90135303672E7079FD6F804A096
:1069A80095F8188047B32B8A71376A48009308BF57
:1069B8000221434616BF0121674A684A2EF0E4FFC8
:1069C80030462F7E2FF0A6FF874240F0F680E37F07
:1069D8005A1EE2776A680AB1023BE3772046696982
:1069E80030F029F86B6813B1596930F024F829465A
:1069F80050462FF010FD5AE730462FF08BFF8045A8
:106A080040F09480237FD5F80C80B5F810B0002BA7
:106A180049D1BBF11F0F42D1D8F800304B453ED1C8
:106A2800414604F1540308F11C0251F8040B914249
:106A380043F8040BF9D10A881A808A7842219A709F
:106A4800552384F87330532384F8743084F87630EF
:106A5800A36DE26DC4F877300023C4F8803094F851
:106A68006030C4F87B209A0684F875100FD194F82A
:106A7800612094F820309A4209D294F86230013BA0
:106A88000F2B04D8012384F87F30237798E72068F8
:106A98002FF036FF022384F87F300423F5E72046E1
:106AA8002FF095FF8CE7032B8AD1302394F861707F
:106AB80003FB0747D4F8803024375B44C4F88030A0
:106AC800BBF1000F16D0384630F0AAF890B1414615
:106AD8005A46384630F0B7F8804628B902215B4656
:106AE8001F4A1C482EF046FFD4F87B30A3EB08035E
:106AF800C4F87B30D4F88020E36D9A420DD2384632
:106B080030F08EF800287FF45BAFD4F88020E36D76
:106B18009A4202D220682FF009FF384630F0A7F8D1
:106B2800003818BF012084F87F00B6E7304695F892
:106B380018802FF0DAFE80457FF442AF237F2A8A3F
:106B4800052B0FD127773BE755534243000F002011
:106B580047630508C0B1040887620508AB620508E9
:106B68000E640508022B7FF42BAF4FF03008D4F8E1
:106B7800803094F861701344C4F880302368196930
:106B8800D3F804B091F8613008FB031124310846AA
:106B9800039130F045F80399024658462FF0D0FE8D
:106BA80000287FF40DAFD4F87B3013B120682FF0A4
:106BB800A7FE08FB07402430B0E730462F7E2FF0B1
:106BC80094FE87427FF40AAFA37F5A1EA2776A68B1
:106BD800002A3FF403AF023BA377FFE6EB7F0133C4
:106BE800EB779DE62046FFF7DBFD99E620462FF080
:106BF80032FF95E6022084F87F0004231AE094F916
:106C0800601040B90029206802DA2FF079FEB7E653
:106C18002FF08CFEB4E6002914DA904202D8B8F1BD
:106C2800000F06D120682FF06BFE022384F87F3016
:106C3800E3E702232377237F022B0CD120462FF092
:106C48000AFF0CE6904200D81FB920682FF06EFEAC
:106C5800EBE70323EEE7032B03D12046FFF7A0FD64
:106C6800FDE5042B7FF4FBADA37F2BB101211D4A69
:106C78001D482EF076FEF2E520682FF036FE074616
:106C880020462FF01AFE0546024604F1730304F16C
:106C98007F0153F8040B8B4242F8040BF9D11B789F
:106CA8002946137038460D22FFF78AFC064601462E
:106CB80020682FF098FB78B10C4A3B4601210A481E
:106CC8002EF058FE3046FDF749FC294620462FF0A5
:106CD800B2FE2FF07CFEC2E5A37F0133A377052324
:106CE8002377BCE534640508C0B104084763050888
:106CF800802938B50D46144621D083290DD019BBFB
:106D08008023537183230320117193710023E07052
:106D180023706570A370043038BD022313710123FA
:106D28005371002393710A23D37108224168A01874
:106D380043F06FFE064B0E201B882382E6E7044BC8
:106D480002201B889380E1E76FF08500E4E700BF2D
:106D58001BC905082DE9F0418769D0F82480BA429B
:106D680028BF3A46B2FBF8F50446C2692B460068CC
:106D78002EF037FF064648B9B7FBF8F7AF4207D001
:106D8800E3692B44E361606A684312E00025012649
:106D9800002205212068FCF77FFB60B10121094A28
:106DA80009482EF0DEFDE3692B44E3610020074B20
:106DB800A362BDE8F081E3692B44E361002EF5D1BD
:106DC800E1E700BF55640508C0B104080203000CE0
:106DD80081420B4607B509D302210D4A0D482EF012
:106DE800C9FD6FF0150003B05DF804FB6AB1013905
:106DF8001144814201D28B4207D9022100930548F0
:106E08001346054A2EF0C0FDEBE70020EBE700BF74
:106E18006C640508C0B10408836405080C2903469E
:106E2800084616D11B78252B12D009D8122B10D85A
:106E3800084A42FA03F313F0010F08BF062070470F
:106E480003F0FD02282A03D05A2B08BF0A207047F6
:106E58000A207047F6FFFBFF2DE9F0411E4690F827
:106E68002C30062A23F00C0380F82C304FF0000356
:106E7800C0E904338361044688460B7886B040F045
:106E88000C81D3B94D7915F0040540F0168290F8BD
:106E98002C309B070AD402234FF468521D4684F80D
:106EA800295084F82830002562853AE02FF014FE36
:106EB8000028F0D12B462A46F1E7032B35D14F792C
:106EC80017F0040740F0F98190F82C308DF807701E
:106ED80043F0040380F82C307023ADF8043090F8A8
:106EE80029300D7903F00F038DF806300A23122D8F
:106EF80028BF12258DF80B30438D2A465BBA3046E1
:106F080001A98DF808708DF809708DF80A7003973B
:106F1800ADF81030ADF81270ADF8147043F01BFDE9
:106F2800A762284606B0BDE8F081122B4BD14B79F9
:106F38005F0700F1C28190F82C3043F0040380F819
:106F48002C304B7813F0020723D113F0010F8B7804
:106F580019D0B1F8035032461946FFF7C9FE6DBA89
:106F6800ADB2854206DAB8F8030040BA80B2002311
:106F78001A4613E03246204698F80210FFF7B8FE8A
:106F88000028F4DA05E083B10221AB4AAB482EF0C1
:106F9800F1FC022305274FF410520020054684F81F
:106FA800283084F829706285BBE7B1F80350314670
:106FB8002FF0C8FD6DBAADB28542D4DB314620460C
:106FC8002FF0C0FDDCE71A2B27D14D7915F0040509
:106FD80040F0738190F82C3043F0040380F82C3093
:106FE8008B783F2B14D1CF7897B90D790323042DD3
:106FF80028BF042530462A4601A9019343F0ABFC7B
:107008003A463B4684F8282084F82970638588E747
:10701800022205274FF41053F4E71B2B23D14D7997
:1070280015F0040540F04981097990F82C200809E9
:10703800C2F340030AD18E0708D5C80711D402F05D
:107048000302032A00F03E81002301E0002BF6D062
:1070580094F82C2063F3410284F82C2000231A466C
:107068001DE70123F4E71E2B40F022814D7915F02E
:10707800040540F022810B7913F0030306D0012B9D
:10708800ECD190F82C3043F0010303E090F82C3059
:1070980065F3000384F82C30E0E70A2A40F0088101
:1070A800232B40D14B7A13F0040340F00681ADF84E
:1070B80004308DF80630082390F82C208DF807301E
:1070C80042F0040280F82C202FF006FD0028B5BFFE
:1070D8004FF0FF3302220322236A8DF80C20A8BF49
:1070E8001BBA0293636A30461BBAC3F307228DF8B2
:1070F8000D30C3F307438DF80F3094F82C308DF81A
:107108000E2043F0040384F82C30B8F8075001A986
:107118006DBAADB20C2D28BF0C252A4643F01BFCD6
:107128000023A362FDE6252B2ED14F7A17F0040722
:1071380040F0C38090F82C3043F00403990780F89E
:107148002C3006D402274FF46853002584F82870A1
:107158005AE72FF0C1FC0028F4D1236A93B1013B10
:107168001ABA22F07F421B0694F82C00616A1A436F
:1071780009BA40F0040084F82C0000230825326086
:107188007160E3E71A46EFE7282B2BD14D7A15F00B
:10719800040540F0928090F82C30D1F8027043F04A
:1071A80004039A07B1F8076080F82C307FF573AEB6
:1071B8002FF092FC00287FF46EAE76BA3FBAB6B2D2
:1071C80032463946206AFFF703FE20B1022305251F
:1071D8004FF4045263E61A4BE7612361636A734311
:1071E800A36167E62A2B2FD14D7A15F0040564D1E7
:1071F80090F82C30D1F8027043F00803B1F807601A
:1072080080F82C309B077FF546AE2FF065FC0028F0
:107218007FF441AE76BA3FBAB6B232463946206AF2
:10722800FFF7D6FD0028D1D1064BE7616361636A99
:107238007343A36112E700BFAD640508C0B1040839
:10724800AF6B03085D6D00085A2B31D14D7A15F0EC
:10725800040532D190F82C3043F0040380F82C3028
:107268008B783F2B19D1CF78E7B94FF4C063CDE9BC
:107278000135B1F8075030466DBAADB2082D28BFB8
:10728800082501A92A4643F066FB00231A4684F81C
:10729800283084F82970628543E6022305274FF4D5
:1072A8001052F4E7022305274FF410520025EEE7A9
:1072B8000121074A07482EF05DFB022305254FF4FC
:1072C8001052ECE50223052545F20232E7E500BF3E
:1072D800CA640508C0B1040807B56B46084A92E8B5
:1072E800030083E8030007488268126822B1194640
:1072F800904703B05DF804FB6FF05700F9E700BF53
:10730800E0B10408F4AC04081F2808B5034606D900
:1073180009480121094A2EF02DFB002008BD012053
:10732800074A00FA03F3D16833EA0101F6D012697B
:10733800934318BF0020F1E7B0B00408E5640508DE
:1073480000200246012100F01F021F2808B501FA9B
:1073580002F2034606D90648064A2EF00BFB6FF0E8
:10736800150008BD044B0020DA601A61F9E700BF78
:10737800B0B00408E5640508002002462DE9F04194
:10738800054600264FF001080E4F6B78F4B2A34271
:1073980001D8BDE8F0812B781C442046FFF7B4FFE4
:1073A80068B12046FFF7CEFF57F834303BB107EB02
:1073B800C40204F01F04516808FA04F09847013623
:1073C800E3E700BFFC310020014B1954704700BFB0
:1073D8005B0B0020034670B1B0FA80F2C2F11F02C5
:1073E800D2B206498856064AD2F880100B43C2F832
:1073F8008030FCF757BCFF22F3E700BF5B0B00208F
:1074080000200246034AD2F8803023EA0003C2F87B
:107418008030704700200246032921D8DFE801F0B8
:10742800020C10190F4B1A6822EA00021A605A68F7
:1074380022EA00025A6070470A4B1A680243F5E7CD
:10744800084B5A6802435A601A6822EA00021A6016
:107458007047044B1A6802431A605A681043586010
:10746800704700BF0020024630B5B0B1B0FA80F3D3
:10747800C3F11F03DBB20B4850F833408C4204D1F0
:1074880000EBC3056D68954205D044B940F8331048
:1074980000EBC3004260002030BDFF23EBE76FF034
:1074A8000F00F9E7FC31002060B1B0FA80F3C3F1B6
:1074B8001F03DBB20021044A42F8331002EBC30277
:1074C80051607047FF23F5E7FC310020C300074AED
:1074D800C0F38100183052F8202003F01800FF2371
:1074E8008340134023FA00F0704700BF0020024693
:1074F800F8B504690D4600AFA034D4E8AF3FC3F334
:107508008003994217D1164A164B6E4688B0002957
:1075180008BF13466A461449C2E905134FF40073BD
:107528009383124B42F8103F00234FF4E451104864
:10753800FBF796FCB5464DB1D4E8EF3F43F00403A2
:10754800C4E8E23F002AF7D1BD46F8BDD4E8EF3FD2
:1075580023F00403C4E8E23F002AF5D0F6E700BFB1
:107568004D650508456505085465050803000001D3
:1075780060B104082DE9F0470546894690461F4644
:10758800D0F808A02FF079FC0446D0B1067FF307A5
:107598000AD590F8203018480121184A2EF0EAF947
:1075A8006FF07700BDE8F0873B46424649462FF02A
:1075B80024FC48B994F820300121114A0E482EF0D5
:1075C800D9F96FF01200EDE79DF8203026F0060695
:1075D80084F82180678484F824302677DAF8183014
:1075E800214628469847B0FA80F3227F5B0963F367
:1075F80000022277D6E700BF60B104086665050877
:107608008065050870B5054686682FF036FC044687
:10761800D8B1037FDB0709D490F820300C4801214A
:107628000C4A2EF0A7F96FF0770070BD0146F36998
:107638002846984738B1237F03F00103227F63F37C
:1076480000022277F1E70346F8E76FF01200ECE753
:1076580060B10408A26505082DE9F3411746D0F882
:1076680008800546D8F83C300E469847002200238B
:1076780039460B48FCF7F4FE044670B901213B4635
:10768800084A094800962EF07FF92846D8F8403075
:107698009847204602B0BDE8F0810676F5E700BFBE
:1076A8000C100020BD65050860B1040870B50D46D2
:1076B8000C7E497E0669C907D6F88020D6F8A43022
:1076C8001FD56CBBEA68D48843B1012B03D1D6F827
:1076D800A800FCF743FF0023C6F8A430C6F8A8505A
:1076E80064B3EB681C78E4090134D6F8A4309C42F2
:1076F80004D10221144A15482EF033F9C6F8A440E3
:1077080070BD6CB9012B1BD0042B14D12B8A002B14
:10771800EBD002210E4A0D482EF023F90624E4E7A7
:10772800052B0FD0022B04D182F0040303F00404CC
:10773800DBE7032B06D00121064AECE70324D4E754
:107748000524D2E70024D0E71466050860B10408D0
:10775800E7650508F465050813B503690C46D3F811
:10776800AC0091F8201031F061F894F8203048B15D
:1077780001210090084A09482EF006F96FF004002C
:1077880002B010BD5B0601D10020F9E7237F43F06A
:1077980002032377F8E700BF2B66050868B10408E1
:1077A800F8B503694768D3F8AC4091F9203091F8EF
:1077B8002060002B01DB0020F8BD7306FBD0488C4D
:1077C800B7F84830C0F30A00834293BF033303304D
:1077D8008308C3F38D03402B98BF5B00D4F8E804FB
:1077E8009D008AB9A84224BF401BC4F8E80491F858
:1077F80020100022204601F07F0131F0B2F8002865
:10780800D9D06FF00400D7E7BA68121AAA4207D293
:107818000A4832460A492FF0A9FE6FF00B00CBE761
:1078280020469AB206F07F0131F09BF80028E8D193
:10783800D4F8E8342B44C4F8E834BCE768B1040849
:1078480052660508F7B5466803697468D3F8AC5002
:1078580064009834A1B20746A400284631F0A0F885
:10786800C5F8E844012410220021284631F079F8AF
:10787800D5F8E8344033C5F8E83473689C420ED331
:10788800284630F0E9FE054680B1024616491748F9
:107898002FF06CFE6FF00404204603B0F0BDE1B297
:1078A8000022284631F05DF80134E6E70246014639
:1078B800009040233846FFF75DFE044628B12A466B
:1078C8000B490A482FF052FEE6E702460090402393
:1078D80080213846FFF74EFE044608B18022EFE7C4
:1078E8003069FCF7DFF9D7E77566050868B1040861
:1078F8008A66050838B504460369D3F8AC5043686E
:107908001869FCF7DDF900212046FFF77BFE38B146
:107918000C490D482FF02FFE6FF00404204638BDA7
:1079280020468021FFF76EFE04460028F0D1284645
:1079380030F0A7FE02460028F0D0044902482FF094
:1079480015FEE9E7A466050868B10408C7660508D6
:1079580038B503690546D3F8AC40204630F0FBFF44
:10796800024630B10D490E482FF000FE6FF00400BA
:1079780038BD0021102031F084FF204630F0EEFFA2
:1079880004460028F2D101462846FFF7B1FD2246F9
:10799800022128462FF0C9FA2046E9E7DB660508E8
:1079A80068B1040870B5036945680446D3F8AC00AB
:1079B80030F03DFE024618B11A491B482FF0D6FD9B
:1079C8006668F069D8B1436898470446B8B102467A
:1079D800164915482FF0CAFD002C19DB00F09AFC57
:1079E800024618B1124910482FF0C0FD2869FCF76B
:1079F8007BF910B12869FCF763F9002070BD0D48C8
:107A0800716983685B6843B90B4907482FF0B3FD78
:107A18000A4905482FF0AFFDE0E798470028DDD078
:107A2800F2E700BFFC66050868B10408126705089C
:107A380065670508F4AC0408306705084C67050855
:107A48002DE9F04103690646D3F8AC50476800F0C9
:107A58002FFC044638B102462D492E482FF086FDEA
:107A68002046BDE8F08176682B4896F84A3071695F
:107A7800012BD0F8088012D9D8F81830083153B93A
:107A8800264924482FF077FD254922482FF073FD19
:107A98006FF00404E4E7224698470028F0D1D8F8AC
:107AA800003071690BB91F49EBE71B48984704463A
:107AB8000028F8D1F06950B103689847064630B1FC
:107AC8000246194913482FF051FD002EDCDB40F225
:107AD800E4420021284642F065FF3B6828462B60B7
:107AE8007B682B7140232B723B6B6B727B6BEB714A
:107AF80030F02DFD024620B10C4906482FF036FD26
:107B0800C6E7284630F0BDFD0028A9D0C0E700BF71
:107B18008367050868B10408F4AC0408A067050881
:107B2800FA670508C2670508DD67050812680508D1
:107B38002DE9F04F06464FF000084FF0280A4FF0A5
:107B4800400BD0F810904468D9F8AC708BB06368DB
:107B5800434559D84FF000084FF0280A4FF0400B22
:107B68006368434500F2908099F8803023F06E03F3
:107B780043F06A0389F88030636B2BB999F8803039
:107B880043F0010389F8803007F5B861082304221F
:107B9800C7F8E46407F5B26031F017FCD4E91012B5
:107BA80007F59E654FF000084FF000096FF00703D6
:107BB80001200027CDE90330CDE906892846CDE923
:107BC80001775D4B009605F017FE3168284631F0C5
:107BD800A4FDE36898473946A06909AA30F024FA59
:107BE800051E08DB099B3A461979186801F062FE00
:107BF800051E80F28480AB1C00F081802A464F4924
:107C08004F482FF0B3FC21E00AFB08F3E26B1A445B
:107C1800917E41F040019176E26BB8F1000F19D1E5
:107C2800917E41F001019176E26BA2F818B0E26B07
:107C380030461A4482F82080E16B19442FF02FF95E
:107C48000546F0B13F493E482FF095FC28460BB059
:107C5800BDE8F08F1A44917E41F004019176E26B01
:107C68001A44917E41F002019176E26B1A44917EAA
:107C780041F008019176E26BB4F848101A44118378
:107C8800D5E708F1010862E70AFB08F3A26B1A447A
:107C9800917E41F020019176A26BB8F1000F17D1C7
:107CA800917E41F001019176A26BA2F818B0A26B07
:107CB80068F07F011A4482F82010A16B30461944FD
:107CC8002FF0EDF805460028BCD108F1010847E778
:107CD8001A44917E41F004019176A26B1A44917E78
:107CE80041F002019176A26B1A44917E41F008019D
:107CF8009176A26BB4F848101A441183D7E7A06AAA
:107D080008B90025A2E7283431F078FA30B90E49CD
:107D18000B482FF030FC6FF0150597E74FF4B011C2
:107D280020462FF0AEFB0028EBD0084904482FF07E
:107D380022FC6FF0040589E72D7E000842680508DB
:107D480068B1040826680508606805087C680508A5
:107D580073B5D0F8AC6008460C4615462FF096F877
:107D6800B8B930466B8AEA6894F8201030F01EFDE6
:107D780058B194F8203001210090074A07482DF0A7
:107D880003FE6FF0040002B070BD012120462FF001
:107D980081F80020F7E700BF9968050868B1040872
:107DA8002DE9F3410369074608460C461546D3F802
:107DB800AC802FF06BF878BB94F820102B8A8029C0
:107DC8001E46EA6802D1402B28BF402691199B1B0A
:107DD8002B82E9603346404694F8201030F00CFDC1
:107DE800054660B194F82030012100900B4A0C48F8
:107DF8002DF0CAFD6FF0040002B0BDE8F08101214A
:107E080020462FF047F894F82030802B04D11EB17B
:107E1800294638462FF05CFB0020EDE7BF680508CF
:107E280068B104082DE9F74F0369A04FD3F8AC50A7
:107E3800DFF87C824FF0FF3201A94FF0FF3305F5E0
:107E4800B26005F0DDF89DF80410012900F0C78044
:107E580002294CD00029EDD1D5F8E44405F29C4A1A
:107E680020462FF00AF82FF035F808B1FCF776FB1A
:107E7800802120462FF001F82FF02CF808B1FCF7EC
:107E88006DFB0822002120462FF0A1F9064620B9F3
:107E9800384688492FF06FFBCCE72FF036F80822D8
:107EA800514606F10C002DF066FF20463146FFF7DB
:107EB800FDFB20462FF0C2FA68B1F3682046D98846
:107EC8002FF006FB10F10C0F0246B3D131462046C5
:107ED8002FF037F8AEE720462FF0B7FA18B1204652
:107EE8002FF060FAA6E720462FF082FAA2E79DF865
:107EF8000590D5F8E46449F0800B594630462EF0D9
:107F0800BCFF824600212EF0C5FF50462EF0F9FF37
:107F1800044600288ED019F07F0F18D1038A73B356
:107F2800402B28BF4023C268594628461E4630F0D9
:107F380063FC024620B1414638462FF017FB79E72B
:107F4800238A9B1B2382E3683344E36072E72EF0A5
:107F5800E3FF814678BB50462EF0B8FF4A462146DB
:107F680030462EF0EEFF50462EF0CBFF024600289A
:107F78003FF460AF51463046FFF712FF5AE72EF044
:107F8800CBFFC0B950462EF0A1FF30462FF06BFA58
:107F9800F8B1214630462FF04AFA30462146FFF71D
:107FA80085FB30462FF058FA00283FF443AF2046AF
:107FB800FCF7D4FA3EE720462EF0B2FFE268002331
:107FC8005946284630F018FC024600283FF432AFE4
:107FD800B1E730462FF04EFA0028DAD1DDE79DF8F8
:107FE8000590D5F8E46449463046BDF806B02EF051
:107FF80044FF04462EF085FF824648B938464A4673
:108008002D492FF0B3FA514620462EF043FF11E7D1
:1080180059460C302DF0A9FEB9F1000F3CD130467D
:108028002FF01AFAD8B120462EF050FF82460146AA
:108038003046FFF73BFB514630462FF0F8F9002158
:1080480020462EF027FF20462EF05BFF0246002830
:108058003FF4F0AE21463069FFF77AFEEAE6BAF857
:108068001020D5F8EC349A4209D2DAF80C104023E3
:108078000A44284694F8201030F098FBDAE62046A7
:108088002EF024FF824601463046FFF70FFB51468B
:1080980030462FF061F9D2E720462EF017FF002274
:1080A800014630462EF04DFFC9E700BF68B104080D
:1080B80003690508E668050822690508F7B591F817
:1080C8002150036905F00305D3F8AC706B1E022B31
:1080D8004FF001020C4688BF0025FFF761FB0646FA
:1080E80098B9628C2B46384694F82010C2F30A02DD
:1080F80030F0F5FA48B194F8203001210090044A94
:1081080004482DF041FC6FF00406304603B0F0BD82
:108118003B69050868B1040813B503690C46D3F830
:10812800AC0030F0C9FA40B1012100902346044860
:10813800044A2DF029FC6FF0040002B010BD00BF06
:1081480068B104085E69050837B5036905460C4639
:10815800D3F8AC0091F8201030F0FAFA024630B9A2
:108168002146284603B0BDE83040FFF719BB94F814
:10817800203001210090044A04482DF005FC6FF0DE
:10818800040003B030BD00BF8469050868B1040865
:1081980073B5036905460C46D3F8AC0091F8201076
:1081A80030F07BFB58B194F8203001210090154A3B
:1081B80015482DF0E9FB6FF0040002B070BD237F75
:1081C80060F34103237720462EF09BFE064608B94C
:1081D8000020F2E720462EF059FE94F92030002BBB
:1081E80007DA0028F4D1324621462846FFF7D8FDA1
:1081F800EEE70028ECD0324621462869FFF7A8FDB3
:10820800E6E700BFA869050868B1040837B50D4658
:10821800044630F0E9FA01238DF805508DF8043052
:10822800ADF806000022002301A904F5B26031F080
:10823800DFF818B1024903482FF09DF903B030BDAB
:10824800CF69050868B10408002307B5ADF8063002
:1082580002238DF805108DF804300022002301A9AF
:1082680000F5B26031F0C4F818B1034903482FF0A3
:1082780082F903B05DF804FBCF69050868B104080A
:10828800002307B501930022002301A900F5B2607D
:1082980031F0AEF8002803DA034904482FF06BF9EF
:1082A80003B05DF804FB00BFCF69050868B1040896
:1082B80010B54FF0FF324FF0FF33134805F034F894
:1082C8000446F8B9114A1368591C1160BBB9104B20
:1082D8001A6942F080521A61DA6822F40012DA60F0
:1082E800DA6842F40022DA60DA68D204FCD5DA6887
:1082F80042F48012DA60064AD3689B04FCD502482F
:1083080004F0D8FF204610BD900F00204C35002007
:108318000008024610B54FF0FF324FF0FF33134804
:1083280005F002F80446F8B9114A1368013B1360D6
:10833800BBB9104BDA6822F48012DA60DA6891046B
:10834800FCD4DA6822F40022DA60DA6842F4001217
:10835800DA60084BDA68D204FCD41A6922F0805239
:108368001A61024804F0A6FF204610BD900F0020B5
:108378004C350020000802468168044808318368AB
:108388005B6803B118476FF057007047F4AC0408F6
:1083980037B5184B8468D3F8A82042F00202C3F816
:1083A800A820D3F8A830206803F002030193019BAA
:1083B80002F0ACFC012002F09FFC63680E48012B20
:1083C800856807D82B6804F108016BB96FF057006E
:1083D80003B030BDAB6904F11001002BF6D00022C8
:1083E80098470028EED0F3E7034803B0BDE83040D3
:1083F800184700BF000C0246F4AC0408F8B54668FC
:1084080096F84530DB0609D40B799F0606D539491D
:1084180039482FF06DF96FF01500F8BD0B78092B6E
:1084280001D03649F4E74B78042B01D03449EFE703
:108438000C7949883268056904F01F04E9B143F6EC
:10844800FF73994222D08B0B032B05D02D492A4864
:108458002FF04EF92C49DBE70023DFF8B0C006F116
:108468002E0737F8020F40EA0C0080B2814205D08F
:108478000133082BF5D12649E9E70B4696F9411057
:10848800012905DC002933DB0020C6E70723F5E7CF
:1084980002292DD195F9B6104E1C01D099420ED162
:1084A8004FF4807085F8B6305169A04021EA000188
:1084B8005161516921F007010B435361E4E795F9D4
:1084C800B710481C01D0994210D14FF4807185F83B
:1084D800B73055690F48A140684001406940516173
:1084E800516921F0700141EA0313E6E70A49AEE752
:1084F8000A49ACE70E6A050880B004083E6A050818
:10850800536A05086D6A05081A6B050800C0FFFF65
:10851800956A050804FFFF03B86A0508E46A0508B8
:1085280038B5304C2368DA0605D510232E492F4874
:1085380023602FF0DDF823685B0743D5226C2C4CB1
:10854800D4F8A4302546991CC4F8A4101A8094F8CD
:10855800B53094F8B4200133DBB29A4284F8B530D0
:1085680030D1002384F8B530636F93B3D4F88C30DE
:10857800B4F898203BB11F4804F1740198470128CA
:1085880012D002281FD0B4F89830B4F894209A4238
:1085980019D90133A4F89830D4F888304BB9BDE81C
:1085A800384013482FF0B5B8D4F8A830C4F8A43030
:1085B800F2E7D5E8EF3F5A1EC5E8E12F0029F8D1C8
:1085C800012BECDC38BDD4F8883013B10A4831F0FF
:1085D80061FA4FF6FF73A4F8B6300848BDE8384092
:1085E80004F068BE00100246306B050880B004082D
:1085F8008001002098AE040888010020D8010020DE
:1086080073B504464668356828462FF0BDF860689B
:108618002FF072F896F845309B0602D560682FF067
:108628006BF80D48616883680831DB687BB90B49D2
:108638000B482FF05DF8019B1BB90A4908482FF039
:1086480057F8284602B0BDE870402FF084B801AA58
:1086580098470028EFDAEAE7F4AC0408A96B0508A4
:1086680080B00408C36B05084FF6FF732DE9F34784
:10867800DFF8F8A04768D0F81080DAF808903E686C
:10868800C8F8A000A8F8B6304468D9F80030054604
:1086980004F108013BB350469847024618BB94F8CA
:1086A8004530D80716D494F84530990708D5D9F835
:1086B800183004F11801B3B100222C48984790B93A
:1086C8002B4A216AD2F8083323F470130B43C2F8FB
:1086D800083308E0D9F8183004F110011BB15046EE
:1086E80098470028DFD00021786A01AA2FF09CFC67
:1086F800041E07DB019B00221979186801F0DAF8DB
:10870800041E0BDAA21C09D001212346194A1A4873
:108718002DF030F9204602B0BDE8F08797F94430D3
:1087280073B1B36823F0104323F0170343F0805369
:10873800B36097F94430022B02D13368DB04FCD5CF
:108748007B6803B198472846FFF75AFFF36830461D
:1087580023F45C63F3602FF017F8D8F848301BB99E
:1087680008F1400004F0A6FD0024D3E7F4AC0408A7
:1087780000100246D76B050880B004082DE9F347BE
:10878800036906460D4603F140084FF0FF324FF0EB
:10879800FF33404604F0C8FD73683469D3F800908D
:1087A800AB68C4F8A4306F683846C4F8B070F8F7FE
:1087B80081FD002384F8B40084F8B53067B97049A6
:1087C80070482EF095FF6FF01504404604F072FDD6
:1087D800204602B0BDE8F0871F46D6F804A0DAF8B4
:1087E80000009AF94020974202DB09D16649E7E781
:1087F800DAF82830297CDB5D994201D00137F2E7AD
:10880800DAF82C20C36852F8272003F00C039342AF
:108818000AD02EF0B9FFDAF82C20C36852F82720C6
:1088280023F00C031343C36033694FF0010CD3F8F2
:10883800B02000237068D2B990F942201AB90268B2
:10884800C3F31103936294F8B4202B68520013B158
:108858009B8903FB0222EB68934214D20121009208
:1088680048484A4A2DF090F86FF00B04ADE792FAA9
:10887800A2F1B1FA81F10CFA01F747EA81610B43E1
:1088880022EA0702D7E771686B7C0868002B4ED193
:10889800036923F001030361AB7C13B13046FFF792
:1088A800AFFE48462EF057FF10232F46C9F8003078
:1088B800D9F8043004F1740643F00403C9F804300D
:1088C8000FCF0FC63B683360002626672B68002B46
:1088D80052D00FCB04F1880585E80F006567A4F82E
:1088E8009860002848D0D4E8EF3FC4E8E26F002A37
:1088F800F9D1D4F888007D227C304FF0000346F18E
:108908000001F8F763FC0022CDE90001002304F11F
:10891800080005F04BFD4FF0FF324FF0FF3304F134
:10892800580004F001FD00B12067246F4DE7082BC3
:1089380020D8026942F00102026191F94320012A1C
:10894800AAD1134A52F82370124A52F823A0036995
:1089580003F01C039A4504D1036903F4F0739F42A2
:108968009AD02EF011FF036947EA0A0723F4FE7331
:108978003B4390E7084923E720462EF0CAFECAE7A2
:10898800F56B050880B004080A6C05081D6C05081D
:10899800E0B40408BCB40408426C0508074B1A6824
:1089A80022F004021A605A68D207FCD40222DA6064
:1089B8001A6842F001021A60704700BF00040340C1
:1089C800044B1A6822F001021A601A68D207FCD414
:1089D800704700BF0004034030B51E4B18680B8871
:1089E800C3F30B030C2B15D813B96FF0850010E0F7
:1089F800023B072B07D8DFE803F02304211F0606F4
:108A0800061D4FF4FA4010600B68B3F5805F1AD268
:108A1800002030BD882BF6D003F67473C3F30B0324
:108A28001C2BE2D801250C4C9D402C40002CEAD18F
:108A3800182BDAD14008E6E70848E4E70848E2E7F7
:108A48004FF40040DFE7C3F313330133B0FBF3F017
:108A58001060DDE7C8060020011111100024F400A1
:108A68000048E801044BDA6842F48032DA60DA68D8
:108A78001204FCD5704700BF0008024638B502F062
:108A8800A5F9434B43491A6A02F007028A5C20FAA7
:108A980002F51A6842F480321A601A689203FCD50B
:108AA8001A68540507D41A6842F480721A60384A62
:108AB80013685805FCD5364CF9F7C4FED4F8F030E5
:108AC80043F08063C4F8F030D4F8F0301901FBD5D6
:108AD800F9F7D6FEF9F7B6FED4F8F03023F018030C
:108AE80043F00803C4F8F030D4F8F03043F0010341
:108AF800C4F8F030264CD4F8F0309A07FBD5D4F8F7
:108B0800F03043F08003C4F8F030D4F8F0301B059F
:108B1800FBD5F9F7B5FEFFF7A5FF1F48A36A854205
:108B280023F00303A36201D202F086FF184B1A6AEE
:108B380022F007021A62D3F8002222F01002C3F8CA
:108B48000022DA6922F0030242F00202DA61DA69ED
:108B580002F00C02082AFAD10F4CA54202D3204693
:108B680002F06AFFFFF77EFF0C4B00201C60084BE9
:108B78001A6A22F070021A621A6A22F4E06242F457
:108B880080621A625A6A22F070025A6238BD00BFC7
:108B9800000C0246C97105080048E801C806002013
:108BA80008B5074830F02AFB38B10648FBF792FBB6
:108BB8000448F9F703FE002008BD6FF01200FBE738
:108BC80060AE0408D18B00080A2838B50446074D62
:108BD80004D1AB680D2128465B689847AB68034809
:108BE8005B68E1B29847204638BD00BF60AE040814
:108BF80037B5104C2268136823F0040313600E4B3A
:108C0800D3F88C309A0203D50C4B1B68DB070FD4C2
:108C180060680B4D83682968DB684BB101AA9847E7
:108C2800002805DB6068296883685B6803B198479A
:108C380003B030BDA4050020000C024600200C4201
:108C48001006002010B5094BD3E90040084B1968FD
:108C580083681B6803B19847236843F004032360C3
:108C6800236843F00803236010BD00BFA40500205B
:108C78001006002008B5EFF31181102383F3128842
:108C8800BFF36F8F0120084B93F8482083F8480002
:108C980081F31188BFF36F8F22B9FFF7D3FF3B2011
:108CA800FBF700F8002008BDA4050020F8B516461B
:108CB800837890F803C0EFF31182102484F31288AC
:108CC800BFF36F8F077890F801E0DB1B03EA0C0312
:108CD8009E4288BF9EB2BD190CEA05053C46057048
:108CE80082F31188BFF36F8F8A198A421AD17745A8
:108CF8000CD1EFF31182102181F31288BFF36F8F2B
:108D08000178417082F31188BFF36F8F02799B1B42
:108D18009A4205D330F0FBFC60B1084804F06CFCC3
:108D28003046F8BD05196D79013401F8015B04EA94
:108D38000C04DAE7FFF79EFFF2E700BFDC0500202E
:108D48002DE9F8430D461446124F07F1560807F16E
:108D5800180914B92046BDE8F8834FF0FF324FF0E8
:108D6800FF33384604F0E0FA224629464046FFF72A
:108D78009DFF064630B94FF0FF324FF0FF334846AB
:108D880004F0D2FA3846A41B04F094FAA4B235448D
:108D9800DFE700BFAC05002038B5456804693148F5
:108DA800836860601B68296803B198476068296810
:108DB800836808319B690BB100229847012204F1AE
:108DC8000800114630F01CFC0122002104F12000AB
:108DD80030F016FC244904F1380030F060FC072319
:108DE80084F86130042384F862300F23002284F869
:108DF8004C300C23114684F85E2084F85F2084F8F8
:108E0800602084F8492084F84A2084F84B2084F8AC
:108E18004D303B202CF00FFF144B1B681A68196962
:108E280022F07C42196822F07F0221EA0201104AEE
:108E38000A431A604AF6C7221A611A6822F0804269
:108E48001A601C6814F08044FBD11A6842F00402CE
:108E58001A601A6842F008021A60FFF70BFF2046F2
:108E680038BD00BFF4AC0408C5780308A405002089
:108E7800000F204810B51D4B01461B68EFF3118405
:108E8800102282F31288BFF36F8F5A68500605D4F8
:108E98005A68D2071DD46FF00A0015E01A6842F02C
:108EA80080421A601A6822F080421A600A22186802
:108EB800400005D45868400602D458684007E7D5F2
:108EC800013AF4D16FF0040084F31188BFF36F8F77
:108ED80010BD5A689207F5D4586810F04000F1D1D7
:108EE8009B680B60002BEFD1D5E700BFA4050020DD
:108EF8002DE9F347D8070F46144605D42E48FFF747
:108F0800D5FE02B0BDE8F087002A37D0EFF311850F
:108F1800102383F31288BFF36F8F3B20FAF7E4FE28
:108F280006463B20FAF7CCFE85F31188BFF36F8F16
:108F3800DFF88880FFF786FED8F800305A685107B6
:108F480014D45B685A0611D44FF0006A2546DFF83E
:108F58007090C9F884A1D8F800305B68DB070FD49B
:108F6800BFF34F8F20BF40BF20BFF4E701A8FFF732
:108F780081FF0024E6B13B20FAF794FE2046C0E7C3
:108F880001A8FFF777FF0028C9F884A1E3DB6A1E70
:108F9800291F019B17FA82F289B2013DADB202F88E
:108FA80001391B0A002DE5D08D42F6D10193D2E795
:108FB800FFF71EFEE2E700BFED050020A405002034
:108FC80000E100E02DE9F74301A8FFF753FF00286F
:108FD80044DB0021042788460846264C019A94F869
:108FE8004B3094F84CC094F84AE0A3EB0E053CEAE9
:108FF80005055FFA82F91ED194F8600094F85F6065
:1090080094F86150861B35EA06062AD109B184F81E
:109018004B30B8F1000F00D001923B20FAF750FE18
:10902800FFF7E6FD002384F84830134803B0BDE895
:10903800F04304F03FB9E11881F84E900121013363
:109048000CEA0303013F4FF001084FEA1222CCD18A
:1090580009B184F84B3001920028E6D103B0BDE88D
:10906800F08326180130054086F86390012084F8C3
:109078006050E7E7A4050020C405002000487047B9
:1090880004B50408044BB3F8A0379B020B60002317
:1090980018464B60704700BF0000FA0B07B503463F
:1090A800054A0091054801212CF06EFC6FF015006F
:1090B80003B05DF804FB00BF986C0508C0B0040855
:1090C80073B5064650220023684630F091FCDDE96E
:1090D800004533691B681A6A12F0FA0212D01A6A3C
:1090E80002F0FA021A626FF0040002B070BD224664
:1090F8002B46684630F0A1FCDDE9003213430CBF73
:109108000122002233691B68186A10F48030ECD001
:10911800002AECD00A230121024A03482CF02AFC39
:10912800E1E700BFC26C0508C0B0040870B5036968
:1091380006461D6849B1FFF7C3FF044650B13069C0
:10914800043004F0B7F8204670BDAB6A002B06DB8C
:109158000024F8E7AB6A43F00043AB62F8E7034B3F
:10916800AB6003F18833AB60F2E700BF23016745CA
:1091780073B5012306460D4614462EF05AFC50B925
:109188000A482B4601210A4A00942CF0FDFB6FF097
:10919800150002B070BD3CB122462946304602B0E7
:1091A800BDE870402EF0F7BB2046F2E7C0B00408D7
:1091B800D66C0508F7B51C46174601232246064615
:1091C8000D462EF036FC50B90B482B4601210B4AB0
:1091D80000942CF0D9FB6FF0150003B0F0BD44B13A
:1091E80023463A462946304603B0BDE8F0402EF003
:1091F800F7BB2046F1E700BFC0B00408016D0508C1
:109208002DE9F84F3F4B17461B680D46804603F083
:1092180001090026FFF7D4FB4FF6FF7B013FDFF87B
:10922800E8A02F44AF420CD3D8F810301C68A36ACA
:10923800002B0EDA0121354A35482CF092FB6FF0ED
:109248000406B9F1000F01D0FFF7A8FB3046BDE8CE
:10925800F88F4046FFF734FF061EF2DBBAF8A0206D
:10926800236C5A4503F4801307D1B5F5801F3AD211
:109278004BB1A36A43F4006308E0002AF5D0B5EBCC
:10928800422F2DD20BBBA36A23F40063A3626B0B9E
:10929800A26A404642F00202A262A26A22F47E72E8
:1092A800A262A26A42EAC303A362A36A43F48033B8
:1092B800A362A36AFFF704FFA36A061E23F0020352
:1092C800A362BEDB05F50055ACE7B5F5801FD0D32A
:1092D800A36A23F40063A362A5F580135B0BD7E7A9
:1092E800B5F5801F05D3002BF2D1A36A43F40063C0
:1092F800F1E701212B46074A05482CF03BFB6FF0AC
:1093080015069EE7000403400007FA0B526D050896
:10931800C8B004085F6D05082DE9F84F0024994688
:10932800304B06461B680D46174603F00108A34656
:10933800FFF746FBD9450DD93369D3F800A0DAF811
:109348002830002B0EDA0121274A28482CF009FB87
:109358006FF00404B8F1000F01D0FFF71FFB20469F
:10936800BDE8F88F3046FFF7ABFE041EF2DB05F1CF
:1093780000631A68013206D001212B461C4A1B489B
:109388002CF0F8FAE4E75A680132F5D19A6801320C
:10939800F2D1DA680132EFD1DAF828004FEAAB02ED
:1093A80040F00100CAF8280057F822202BF00301EA
:1093B800DAF8280039441A604A6830465A608A68E0
:1093C80010359A60CA68DA60FFF77AFEDAF8283052
:1093D800041E23F00103CAF82830BBDB0BF1100B85
:1093E800A8E700BF00040340526D0508C8B0040890
:1093F800786D050830B50F4C0F4D0C60236813B11C
:109408002B68136030BD03694FF6FD701B681B6C39
:109418000A4BB3F8A030591E89B281428CBF4FF471
:109428008073DB0823604FF40053636001232B60D3
:10943800E7E700BF54350020503500200007FA0B3D
:109448002DE9F843D0F8049090460746D9F808006B
:109458000D461E462DF0A1FCB8F5001F044616D196
:109468002846D9F80840FEF731F884420CD129463D
:109478002DF093FC0446FDF7C5FF2046FEF714F8CF
:1094880000212046FDF7C8FF0020BDE8F883B8F5A5
:10949800800F20D0B6F1806F19D0B6F1C06F18D008
:1094A800B6F1007F1AD102263A4620460E49FDF74A
:1094B800DBFFB0B92846D9F808102DF073FC204618
:1094C8003146FDF7A9FF2046FDF784FFDCE70126BA
:1094D800EAE70326E8E76FF08500D6E76FF01500A6
:1094E800D3E76FF00F00D0E7E57C030808B5094A19
:1094F800136943F000531361416807480C318368CE
:109508001B681BB1984700EAE07008BD6FF0570070
:10951800F9E700BF00080246F4AC04080C291FB59F
:1095280028BF0C210C460A4BD3F8082712BA01921F
:10953800D3F8042712BA0292D3F800370A461BBAA6
:1095480001A9039341F007FA204604B010BD00BFFB
:109558000000FA0B08B50121034A04482CF001FA6F
:109568006FF0040008BD00BF096E0508E8B00408E4
:1095780098B542680369D26800AF83F8621029B9C8
:10958800136823F440131360BD4698BD6C468AB037
:109598006A4603680848D161C2E905034FF40073BD
:1095A8001384064B42F8103F00234FF4115104482E
:1095B800F9F756FCA546E7E7276E05080400000101
:1095C800E8B00408F7B500224368044606691C4859
:1095D8000F46DD68596883680192DB684BB9012141
:1095E800184A19482CF0BDF96FF00404204603B05E
:1095F800F0BD01AA98470028F1DB376306F1180788
:109608004FF0FF324FF0FF33384603F08DFE2B68E2
:10961800204623F001032B6096F86210FFF7A8FF9D
:109628002046019900F0A0F896F8613004461BB175
:109638002B6843F001032B60384603F03BFED5E767
:10964800F4AC04083B6E0508E8B0040870B504469D
:10965800466805694FF0FF32002128462FF0D0FFF9
:10966800336820469847002385F8603085F86230D3
:10967800012205F1180011462FF0C2FF204600F024
:109688003FF83169184B994222D015D8174B9942A7
:1096980020D0174BCB1A594259418900204641F036
:1096A8001001FFF78FFF041E18DA0121114A124832
:1096B8002CF057F9204670BD104B99420CD003F599
:1096C800C31303F5206399420CBF0A210021E5E783
:1096D8000621E3E70221E1E70821DFE7012300246F
:1096E80085F86030E6E700BF40420F00A086010021
:1096F800801A0600696E0508E8B0040840E13300E6
:1097080037B545680021686901AA2EF08DFC041E52
:1097180007DB019B00221979186800F0CBF8041EBA
:1097280008DA012123460C4A0C482CF023F920467C
:1097380003B030BD0A48696883681B683BB90121DA
:10974800084A06482CF00DF96FF00404EFE7984733
:1097580004460028EBD0F2E79A6E0508D8B0040852
:10976800F4AC0408B86E05082DE9F74F446803699E
:1097780000200193E369E568DFF81481DFF81491AC
:10978800DFF814A1DFF814B10093009B8342019B1A
:109798001A6B0DD1C2F34202012A3BD0022A68D0CB
:1097A8003F4A404801212CF0DCF86FF015001FE01B
:1097B8000C2303FB00F7D4F818C0DFF8ECE00CEB3F
:1097C8000706736873451DD015D853451CD05B45F3
:1097D80014BF002301239B00C2F34202B2EB530FD4
:1097E80016D15CF807308B4212D1B36800202B6188
:1097F80003B0BDE8F08F434508D04B450CBF0A23A2
:109808000023E9E70623E7E70223E5E70823E3E780
:109818000130BAE741F25C2E4FF47A6C40F2E2472D
:109828004FF4FA760220214B421EB1FBF2F2B3FB51
:10983800F2F2BCFBF2F4013CFF2C23D8BEFBF2F899
:1098480008F1FF38B8F1FF0F1CD8B6FBF2F9B9F1EF
:109858000F0F17D8B7FBF2F2013A0F2A12D80238C5
:1098680048EA094343EA007343EA025343EA0423FC
:10987800BCE740F2145E4FF4167C4FF4FA7740F2DE
:109888007716CFE701301128CED1094A89E700BF02
:1098980040E13300404B4C00A0860100801A0600CE
:1098A800E86E0508E0B0040840420F0000CA9A3B81
:1098B800636F05082DE9F047044600251D4F00EBAE
:1098C800C106B44201D1002014E02068C30600F0AC
:1098D8001F0911D4656845F02005C0F3481AC0F384
:1098E8004420192823D857F82080B8F1000F0DD14B
:1098F8006FF01200BDE8F087B9F1100F04D0B9F18C
:10990800110FEAD16568E8E73025E6E740462FF011
:1099180075FC0028ECD04B462A4640460AF00F0159
:109928002EF0F2F9002804F10804CADAE2E76FF031
:109938001500DFE7E0B5040843681B6803F1080277
:1099480052E8002F42F0010203F1080040E800212C
:109958000029F3D1094A934203D0A2F574429342F5
:1099680003D15A6842F040025A6053E8002F42F48B
:10997800807243E800210029F7D170470038014080
:1099880043681B6803F1080252E8002F22F0010225
:1099980003F1080040E800210029F3D1094A934265
:1099A80003D0A2F57442934203D15A6822F04002D0
:1099B8005A6053E8002F22F4807243E800210029FE
:1099C800F7D17047003801402DE9F04182B0426874
:1099D80006460D46D2F8008000AF002945D05068F1
:1099E800116952698368012ADB6812D908316BB1A1
:1099F8003A1D9847041E16DA204A012120482BF008
:109A0800B0FF20460837BD46BDE8F0816FF0570427
:109A1800F2E72BB13A1D9847041E04DA194AECE71D
:109A28006FF05704FAE7D8F8003023F40043C8F879
:109A380000307B6803EB5503B3FBF5F30F2B17D806
:109A48006C468AB033686A460F49D561C2E9051386
:109A58004FF4007313840D4B42F8103F00234FF46A
:109A680011510748F9F7FCF9A5466FF01504C8E746
:109A78009BB20024C8F80C30C3E700BFA76F0508E5
:109A880058B104083B6E0508D56F050804000001AD
:109A9800F8B50C46036941681D682379012B15D078
:109AA8009F1E7E427E41B6026279022A96BF464FC9
:109AB8004FF4005737F81270A279022A09D0042A05
:109AC80030D0003B18BF01231B0306E04FF4C066EB
:109AD800EAE7B3FA83F35B091B07E2790968012A0D
:109AE80014BF4FF0000C4FF4407CA5421DD10A680A
:109AF80022F0805222F4B05232431A430A604B6873
:109B080023F440533B434B6043681A68936823F43B
:109B1800407343EA0C0393602968FFF755FF00EA96
:109B2800E070F8BD4FF48053D7E7D1F800E00EF4A9
:109B3800C06E76451FBFD1F800E02EF4C06E4EEA25
:109B480006060E6041680E68716801F440518F4244
:109B58001FBF716821F440513943716041680E6834
:109B6800316801F010218B421FBF316821F01021AC
:109B78000B433360436819688B6803F440739C4552
:109B88001FBF8B6823F4407343EA0C038B60436860
:109B98001B689968490405D5032A09D09A6822F4F4
:109BA800804204E0032A03D19A6842F480429A6012
:109BB80021682B68994205D0FFF706FF0028B0DB23
:109BC80023682B600020ACE79C4D0508F8B5436876
:109BD80002461C68036908791D6801280E4691F839
:109BE80005E08B7913D1BEF1020F54D9022B1F4621
:109BF8004FF4C0614FF4005C65D0042B5ED00028A0
:109C080066D0C31E012B5BD86FF08500F8BD022813
:109C18000AD1BEF1020F4AD9022B1F464FF48061C8
:109C28000BD04FF4005CE8E7BEF1020F42D9022BDB
:109C38001F4641D1002856D00021C31E012BE3D96D
:109C48000020022703239E45DED12EF038FAB842C1
:109C5800DAD1F3795BB1012B4DD1284B9C4206D068
:109C6800A3F574439C4202D0254B9C42CCD1236877
:109C7800314623F0010310462360FFF709FF00284F
:109C8800C2DB236843F00103236096E8030085E8FC
:109C980003000020BAE74FF4C0611A4F022B37F8CF
:109CA8001EC01F46A9D170B94FF0805010E04FF484
:109CB8008061F2E70021F0E70021B2E70028A3D194
:109CC8004FF4805004E0C31E012B9DD902270020C9
:109CD800BCF5805F0BD0BCF5405F0AD0BCF1000F2B
:109CE800B0D10123AFE701464FF08050AAE7002327
:109CF800A9E70223A7E7032BAFD085E70038014087
:109D0800002400469C4D05082DE9F04383B0D0F8A7
:109D180004800646D8F80400D8F81010836800AF0D
:109D28001B685BB9684A012168482BF01AFE6FF07E
:109D3800570420460C37BD46BDE8F08398470446D3
:109D480038B1614A012161482BF00BFE002CF0DB91
:109D580003E0D8F81430012B24D80021D8F82400C7
:109D68003A1D2EF061F9041EE3DB7B6800221979A5
:109D78001868FFF79FFD041EDBDB756833692C68E4
:109D8800D3F80090236823F001032360A8682FF01C
:109D980035FAB8B901214E4A4C482BF0E2FD6FF074
:109DA8001204C6E74B48D8F81010836808319B693D
:109DB8000BB9494AB7E72246984704460028CCD051
:109DC800454ABFE7D5E902018368DB6803B19847D4
:109DD80054E8003F43F00C0344E80032002AF7D16E
:109DE80049463046FFF754FE002802DA6FF01504A2
:109DF8009FE72B7E1BB1A36843F00803A3606B7E2B
:109E08001BB1636843F400436360AB7E1BB16368B6
:109E180043F480336360EB7E1BB1636843F4003323
:109E280063602B7F002B38D02C4B9C421BD0A3F5B2
:109E380074439C4217D02A4B9C4214D06C4688B07D
:109E48006A4633682749C2E905134FF400739383C0
:109E5800254B42F8103F00234FF4E2511B48F8F716
:109E6800FFFFA546C2E773681A68936843F4804306
:109E7800936023686A7F23F0787343EA4253236030
:109E88002368AA7F23F4F81343EA02432360EB7F95
:109E98001BB1A36843F40043A36095F820301BB1BD
:109EA800236843F000532360236843F001032360D1
:109EB800E3699A02FCD5E3695B02FCD53046D8F821
:109EC80028309847002434E7EC6F050858B1040897
:109ED8002F700508F4AC04080C7005080038014020
:109EE800002400464A7005080300000138B50B68D5
:109EF800054698882EF087FA04280C46D1E91812EE
:109F0800034618D002280DD194F87000012802D910
:109F1800E06E01280FD8288E80B209B102B10880FE
:109F280002250DE001281CD194F87000032813D9EC
:109F3800E06E032812D9286B09B102B10860042524
:109F4800626EB5FBF3F592B19542294617D91949C6
:109F580019482EF090FA0AE0012802D9E06E01288B
:109F6800D9D895F83000C0B229B112B901252846D0
:109F780038BD0870626E002AF8D001252946521AA9
:109F880062667AB9226D04F1540108322265626D65
:109F980004F15000013A626504F164022EF00FFAF0
:109FA8002066E4E7226E002AE1D001FB0322226644
:109FB800DDE700BF8770050830B1040838B50B68C5
:109FC800054698882EF01FFA04280C4603468A6D29
:109FD8001AD002280FD191F87010012902D9A16E68
:109FE800012911D8002A48D0E16D01B1118889B240
:109FF800298402250EE0012820D191F87010032948
:10A0080017D9A16E032916D98AB1E16D01B111687A
:10A0180029620425E26DB5FBF3F532B19542294674
:10A0280018D91B491B482EF026FA284638BD114678
:10A03800EEE7012902D9A16E0129D3D8FAB1E16D61
:10A0480001B11178C9B285F82010E26D0125002A06
:10A05800EBD02946521AE2659AB9A26C04F14C0178
:10A068000832A264E26C04F14800013AE26404F1A7
:10A078005C022EF0A4F9A065D7E71146B7E71146B0
:10A08800E0E7A26D002AD0D001FB0322A265CCE74D
:10A098008770050830B10408B0B50446406900AFC0
:10A0A80010F478701DD06D468AB06A460E4B536125
:10A0B8000E4BC2E906304FF4007313840C4B42F880
:10A0C800103F00230B484FF41151F8F7C9FE6FF009
:10A0D8000400AD4663695B0642BFA36943F04003D1
:10A0E800A361BD46B0BD00BFA5700508A0710508F5
:10A0F8000400000130B1040838B5436804465B69C0
:10A10800056998472B6923B96B6005F1080003F0CE
:10A11800D1F8012160682EF0DAF9002802DA10F18E
:10A12800860F14D16568002128462EF0D0F9041E48
:10A138000BDB0948A96883681B684BB1984704463C
:10A1480018B1064906482EF096F904EAE47038BDBD
:10A158006FF05704F5E700BFF4AC0408B0700508C9
:10A1680030B10408F8B5054647682C6938680369B2
:10A1780023F002030361036923F001030361036908
:10A1880023F020030361036923F04003036103699B
:10A1980023F080030361036923F480730361036977
:10A1A80023F40073036197F82530DA0707D50369AC
:10A1B80023F008030361036923F00403036143697F
:10A1C800DB0702D590F83030F9E7C3685E022BD57B
:10A1D800384E43689BB21BBB436913F4805F23D19D
:10A1E8000368DB0720D597F82530DA070BD42368F6
:10A1F8009B88C3F34513192B05D826FA03F3DA070E
:10A2080001D52EF0F2F80368C26803F4006302F483
:10A21800C0221343B3F5C02FDBD12EF0E6F8D8E700
:10A22800436913F0080FDAE743699B0542BF836966
:10A2380043F40073836197F825600368F607C268E2
:10A2480010D5836943F010038361836943F04003A9
:10A258008361836943F00803836143681B0C1B0413
:10A26800436007E003F4006302F4C0221343B3F52C
:10A27800C02FF2D023689B88DB0401D42EF0B5F8F8
:10A2880094F8443033B9A16304F12000BDE8F840E4
:10A2980003F010B8E36B13B12846226C9847236883
:10A2A8009B8813F4005303D1636004F10800EDE7C1
:10A2B800F8BD00BF000202022DE9F84347680646D0
:10A2C80097F825300569D807D7F8008004D5D8F85D
:10A2D8000030D90740F1FD804046FFF7DDFE01461A
:10A2E80020B13046BDE8F843FFF73CBFEB6D0BB932
:10A2F8006A6E42B32A683C689288D20700F1C2802D
:10A3080097F8253013F0010F2368E26800F09D806C
:10A3180003F4006302F4C022134342D163695B076C
:10A3280022D46369D80725D5EB6E1BB3294620468E
:10A338002EF0A5F863691B0747D43868FFF7ACFE11
:10A3480001460028CDD1D8F80030D8F80C2003F405
:10A35800006302F4C022134340F0B080EB6D002B81
:10A3680040F0B7806B6EADE0AB6E002BD9D0EB6ED2
:10A3780093B9636963699A07DCD5AB6E002BD9D0B2
:10A38800EA6E9342D6D1294620462EF08CF82369EE
:10A3980023F002032361CDE7294620462EF083F8F7
:10A3A800C4E7B3F5C12FE5D06269D10702D5EA6EDB
:10A3B800002ABBD1B3F5C02FBCD0DBE72946204625
:10A3C800FFF794FDEB6E1B1AEB66EB6E002BF5D1D5
:10A3D800EB6D6A6ECBB9C5E91A22002AADD0A36924
:10A3E800204643F01003A361A36943F00803A36167
:10A3F8002DF0FBFFAA6E3B6A9A420DD936493748C1
:10A408002EF039F86FF015016BE712B1934228BFAF
:10A418001346C5E91A33E2E7636829461B0C1B0497
:10A4280013436360236843F001032360236843F404
:10A4380000732360236943F004032361236943F015
:10A44800020323612EF02FF877E703F4006902F482
:10A45800C02349EA0309B9F5C02F07D13868436911
:10A46800D907FCD52946FFF741FD66E763699807D8
:10A47800FCD529462046FFF7A1FDB9F5C12F3FF4C9
:10A488005CAFEBE76269920713D593B12946204682
:10A49800FFF794FD6369DB077FF54FAF2B6E002B49
:10A4A8003FF44BAF6B6E002B3FF447AF2946204675
:10A4B800D9E7236923F002032361EBE7B3F5C12F42
:10A4C80003D1EB6D2BB900210BE7B3F5C02F3FF497
:10A4D80049AFBDE8F88300BFCB70050830B1040868
:10A4E8002DE9F04F87B000AF0E469A4693460569AE
:10A4F800F8601AB9BAF1000F00F0F382B388980433
:10A5080033D44FF0FF324FF0FF3305F1080002F06B
:10A518000BFF6E6097F8403085F844307B6CEB6336
:10A52800BB6C2B64FB68D3F81080D3F80490D8F880
:10A538000030D9F800409E4240F01981B3881905CF
:10A5480040F10D82BBF1000F16D020464FF4C12117
:10A558002DF026FFB0882DF056FF8046DBF800303E
:10A56800AB64A3B1DBF8043011E02B69002BC8D130
:10A578006B689E42C5D1CDE720464FF4C0212DF02F
:10A588000FFFB0882DF03FFF80460023AB64EB64DB
:10A5980005F15C02434605F14C0105F148002DF038
:10A5A8000EFFA865BAF1000F40F0F581C5F850A07C
:10A5B80000236B6505F16402434605F1540105F17A
:10A5C80050002DF0FCFE00232866AB632268E36888
:10A5D80002F4006803F4C02348EA030899F8253018
:10A5E800D80729D5FB68B2885B68D107BB601B68B0
:10A5F80022D41968D868FA6801F4006100F4C02010
:10A608000143126940F0D281D16D566E29B1002EF6
:10A6180000F0CA818E4228BF0E46002EC0F2BA80D2
:10A62800B968096AB142C0F0CF81C2E91A665A68AE
:10A63800120C120432435A60FB6859680B681A6896
:10A6480042F001021A60DA68520200F1C28191F800
:10A658002520D60700F1C6811A6942F020021A6146
:10A668001A6942F040021A611A6942F080021A61BE
:10A678001A6942F480721A611A6942F400721A6106
:10A68800BAF1000F03D01A6942F001021A614FF4BF
:10A69800FA5A1A6905F1200B42F002021A6195F87C
:10A6A8004430002B00F0A781B8F5C12FEB6D53D1D2
:10A6B800D9F80060002B47D16A6E002A00F00A82A0
:10A6C8002A689088C20715D41A46D5F854C062453E
:10A6D80040F0E4812DF097FE93FBF0F200FB12327C
:10A6E800002A40F0F481B3FBF0F37268120C1204F4
:10A6F8001343736030464FF4C0212DF051FE336888
:10A7080043F001033360F368580200F1CE8199F8F1
:10A718002530D90700F1D681336943F0200333612E
:10A72800336943F040033361336943F08003336195
:10A73800336943F480733361336943F400733361DD
:10A74800336943F0010333612368E26803F400636B
:10A7580002F4C02848EA0308EB6D1BB96E6E002EA0
:10A7680000F07B81B8F1000F99D1464675E1D9F820
:10A778001020B188022AC1F3451312D0032A13D03E
:10A78800012A2BD1043B1C2B8CBF002301237BB94E
:10A798006FF0850600236B6005F1080002F08AFD62
:10A7A80063E1043B0C2BEFE7082B01D0102BEFD112
:10A7B8000A0448BFE368AF4842BF23F4601343F478
:10A7C8000023E3608368D9F80810DB685BB9AA49FD
:10A7D800AA482DF050FE6FF00406DBE7A849A74809
:10A7E8002DF049FED4E707F1140298470028EEDB64
:10A7F80000227B69316823FA02F0884218D90132B5
:10A80800092AF8D16C468AB06A46D3611B0A1362DA
:10A8180005239C48C2E9050142F8103F00234FF484
:10A8280021519648F8F71CFBA5466FF01506B1E7CD
:10A838002368954923F001032360A36851F8222077
:10A8480023F070431343A36099F825309B0700F168
:10A858008F80B38813F0020FE36814BF43F00073CE
:10A8680023F00073E360B38813F0040FE36814BFA8
:10A8780043F0807323F08073E360B18811F40061C2
:10A8880004D0BBF1000F7AD04FF4C12120462DF03F
:10A8980087FDB38813F0100FE36814BF43F4000377
:10A8A80023F40003E360A36823F48003A360327DEC
:10A8B800B3881AB999F82520500763D5D90706D463
:10A8C800E368DA005EBF236843F480532360E368DB
:10A8D80023F0105343F08063E360B3886B4913F0AF
:10A8E800010FE36814BF23F4800343F48003E3609B
:10A8F800B288A368C2F34512043A51F8222023F023
:10A908001F031343A360E368D9F81C2023F00F0347
:10A918001343E360E368D9F8182023F0F00343EA0F
:10A928000213E36099F825305949DB0741BFB38822
:10A9380099F82420C3F34513073343BFDB085B00B2
:10A94800B2FBF3F3012388F87030A268013B51F899
:10A95800233022F4F0721343A360C8F80060B08873
:10A968002DF051FD8046BBF1000F7FF4F7AD0CE6EA
:10A97800D9F80020D36843F40043D36069E74FF463
:10A98800C02183E713F0010FE36823F0105308BFD9
:10A9980043F00053A0E7DAF800302B65002B3FF4B2
:10A9A80007AEDAF8043004E60E4636E6B1F5C12FF4
:10A9B80030460CBF59465146C7E900322DF039FDE3
:10A9C800D7E90032064628E632492C482DF053FDD7
:10A9D8002BE71A6842F400721A601A6890053FF56E
:10A9E80036AEFAE71A6942F008021A611A6942F0AB
:10A9F80004021A6130E61A46E86C82421BD1002232
:10AA080011466E6DB1421DD1934238BF13460AFB01
:10AA180003F22B681B68B2FBF3F2C832530FD20063
:10AA2800584602F081FCA0B11B4914482DF023FDC3
:10AA38006FF07306AEE6A96C01EBC20149680132FA
:10AA48000B44DAE7286D00EBC1004068013102448D
:10AA5800D8E7AE6B002E3FF427AE95F84430002BB4
:10AA68003FF498AE002EFFF695AE30461C37BD4633
:10AA7800BDE8F08FF4AC04081F71050830B1040874
:10AA8800F77005084B710508A8B604084CB7040808
:10AA98002CB70408CB7005087A710508296D01EBFD
:10AAA800C201496801320B4411E6336843F400736C
:10AAB800336033689A053FF52AAE73691B073FF583
:10AAC80026AEF6E7336943F00803336124E62368CA
:10AAD800E368AAE62268E36802F4006803F4C02386
:10AAE80038E65646C1E700BF4FF0E02310B50F49DE
:10AAF8009C691A6908689B690D4902F4803234B967
:10AB080093B903464AB90A681044C01A10BD002B0D
:10AB180008BF03460AB9A342F5D90A6802440A6085
:10AB28004FF0E0221269EEE70446F3E74C360020C6
:10AB3800403600201022094B002083F823204FF4D0
:10AB48007A62074B1A60074B40F69F7218604FF005
:10AB5800E0235A61072298611A61704700ED00E00E
:10AB68004C36002040360020684620F007018D460C
:10AB780001B5FFF7B9FF0D4B0D4A18681168084475
:10AB8800106000224FF47A611A600A4A1368C01AEA
:10AB9800B0FBF1F001FB0033136003F00FFBF8F793
:10ABA800A5FDBDE801408546704700BF403600203E
:10ABB8004836002044360020F8B5314F81B1421C98
:10ABC80009D14FF0E022136923F0010313614FF01C
:10ABD8007F433B60F8BD3D68012806DC00240AE09D
:10ABE800431C3D68F8D141F2610041F2620398428A
:10ABF800A8BF1846441EEFF31186102383F312886A
:10AC0800BFF36F8FFFF770FF4FF0E0230022DFF8EC
:10AC180074C09969DCF8003018441B4B1A601B4B50
:10AC28001A68831A28D44FF47A6E0EFB043404F69B
:10AC38009F74B4FBFEF4131A0EFB0433B3F5806F54
:10AC480038BF4FF48063124A934228BF13464FF02F
:10AC5800E0223B60013B946953610023A142936168
:10AC6800A1EB040338BF5B191844CCF8000086F345
:10AC78001188BFF36F8FADE74FF48063E7E700BF3C
:10AC88004C3600204836002040360020443600204C
:10AC9800A0EBFF0038B5EFF31185102383F312887A
:10ACA800BFF36F8F084B1C68084B1B68E41AFFF74B
:10ACB8001BFF85F31188BFF36F8F4FF47A6320442D
:10ACC800B0FBF3F038BD00BF483600204436002002
:10ACD80038B5EFF31185102383F31288BFF36F8F14
:10ACE800044B1C68FFF700FF85F31188BFF36F8FD3
:10ACF800204438BD48360020034A536F23F001032F
:10AD080003435367704700BF00040046034A536F6C
:10AD180023F03C0303435367704700BF0004004619
:10AD2800F8B51F4F786BC0F308000130F5F784FFC2
:10AD3800BC6A0546C4F302200130F5F77DFF0646DC
:10AD480014F0100018BFB86B04F0030418BFC0F368
:10AD5800CC00F5F771FF022C07461CD0032C1CD140
:10AD68000F4B10481B68C3F300531841F5F764FFF5
:10AD780004464FF064513846F5F7B6FF2946F5F713
:10AD8800ABFE314605462046F6F762F801462846EE
:10AD9800F5F7AAFFF8BD044CEBE70024E9E700BF8C
:10ADA800000C02460048E8010024744B10B5064B1D
:10ADB8005C6BFFF7B5FFF6F799F9C4F30664013445
:10ADC800B0FBF4F010BD00BF000C0246084AD3697E
:10ADD80013F00C0309D0082B05D113680548C3F3F9
:10ADE800005318417047FFF7E1BF0348704700BFA1
:10ADF800000C02460048E8010024F40008B5FFF7FB
:10AE0800E5FF054B054A1B6A03F00703D35CD840EE
:10AE1800034B186008BD00BF000C0246C971050845
:10AE2800C80600202DE9F04F066889B00446304670
:10AE38002EF06AF80390002840F06E8120682EF00A
:10AE480035F8002800F06881D6F808382068C3F380
:10AE58000D23C4F8D4342EF029F8870748BF226898
:10AE680006F5006542BF536903F002035361206889
:10AE78002EF01CF8C0062CD52268936923F0100325
:10AE88009361D6F82080C8F34343022B08F00F07DC
:10AE980040F0458147F6F07318EA030F14D02423D5
:10AEA80003FB0747C8F30A194A463046D7F8601229
:10AEB8002DF090FFD7F860324B44C7F86032D7F8CE
:10AEC80068324B44C7F868322268936943F010032C
:10AED800936120682DF0EAFF010300F132812068B8
:10AEE8002DF0E4FF42030DD520682DF0EBFF274637
:10AEF8004FF0000A049006F5106B049B2068002BA5
:10AF080040F0EA8120682DF0D1FF002813DA6B6841
:10AF180023F001036B6094F8CC34012B40F0848259
:10AF28000021204684F8CC142DF051FD2268536985
:10AF380003F00043536120682DF0B8FF01050AD5DE
:10AF4800AB68DA0702D520462CF085FB22685369E6
:10AF580003F40063536120682DF0A8FF030115D5A1
:10AF68002268536903F00063536194F8CC34002BD2
:10AF780040F05E820121236884F8CC145B6D204682
:10AF8800C3F38303C4F8D0342DF021FD20682DF0DD
:10AF98008DFFC70433D56B68102123F001036B6064
:10AFA80020682DF096FD4FF67F3106F51063227963
:10AFB8000398824200F24082EB6943F00113EB618F
:10AFC800E37B002B00F05682D5F8843043F00B0366
:10AFD800C5F884306B6C43F00B036B64D6F800380B
:10AFE80004F29C4223F4FE63C6F80038A179206875
:10AFF80000F0FCFC2268536903F480535361206815
:10B008002DF054FF800416D520682DF081FF2068AC
:10B018002DF0AAFDE0712768FFF7F0FEE2790146FE
:10B02800384600F06BFA20462CF0DDFA22685369A6
:10B0380003F40053536120682DF038FF010707D54A
:10B0480020462CF026FB2268536903F0080353615D
:10B0580020682DF02BFF020600F1178220682DF0E2
:10B0680025FFC3020CD5A046012706F512692379EE
:10B07800BB4200F228822268536903F480135361AB
:10B0880020682DF013FF870229D52346012206F5F3
:10B098003261207990421DD993F87C720868012F9B
:10B0A80040F02782002880F22482D4F8D4C48CEAA5
:10B0B8001040C00700F11D8283F87B72B06940F030
:10B0C8008000B0617069000600F113826B6843F478
:10B0D80000736B602268536903F40013536120689E
:10B0E8002DF0E4FE410007D520462CF0A8FA22688E
:10B0F800536903F08043536120682DF0D7FE42075F
:10B108000AD523685D686B0702D520462CF09DFAA6
:10B11800226853682B43536009B0BDE8F08F062BB3
:10B128007FF4D2AE0822304604F29C412DF052FE44
:10B13800242303FB0747D7F86832C8F30A184344A7
:10B14800C0E620682DF0B6FEA2460027049006F55A
:10B158003068049B2068002B3FF4C1AE049BDB07DA
:10B1680065D55FFA87FB59462DF0B4FE10F0010F44
:10B1780081461ED00123C8F80830206894F806C01C
:10B1880000F5306303EB4713BCF1010F016C9A68BB
:10B198007BD112F0080F07D0B448814209D91204B4
:10B1A80007D54FF4004203E012F0200F48D02022C8
:10B1B8009A6019F0080F0FD00823C8F808302368E0
:10B1C800AA49186C03F5306303EB471388429A6861
:10B1D80070D82046FDF754F819F0100F1CBF102343
:10B1E800C8F8083019F0020F14D073691A0642BF64
:10B1F8006B6843F480636B609AF85732012B06D171
:10B208000023594620468AF857322DF053FA022374
:10B21800C8F8083019F0200F1CBF2023C8F80830E0
:10B2280019F4005F1CBF4FF40053C8F80830049BA2
:10B2380001375B08049308F120080AF1240A88E71B
:10B2480012F0280FB5D1DFF824C2614501D91204E4
:10B25800A7D41A69DAF87432C2F312029B1ACAF830
:10B2680068326FB9D4F864222AB9012104F29C42E9
:10B2780000F0BCFB04E0D4F860221A44C4F8602251
:10B2880059462046FCF7C2FF93E7DFF8E4C1614561
:10B2980006D1110485D49006F2D520229A60EFE7F2
:10B2A800002FEDD1D4F86432002BE9D1394604F2ED
:10B2B8009C42DDE7110448BF4FF40042204648BFD6
:10B2C8009A60FCF7DDFFA179012985D1206804F295
:10B2D8009C4200F08BFB7FE7049BDB0740F19B80DF
:10B2E8005FFA8AF3194607932DF0FDFD10F0010F60
:10B2F800804620D001216B6B0AF00F0201FA02F29E
:10B3080023EA02036B63CBF80810A17901290DD158
:10B31800D7E9072313443B62BAF1000F06D1636AE9
:10B3280023B9206804F29C4200F060FB20465FFAD3
:10B338008AF1FCF789FF18F0080F1CBF0823CBF827
:10B34800083018F0100F1CBF1023CBF8083018F085
:10B35800400F1CBF4023CBF8083018F0020F10D064
:10B36800514630462DF0B5FBFB7D012B06D100235D
:10B378002046FB755FFA8AF12DF09DF90223CBF880
:10B388000830236818F0800F059344D0D7E90932B4
:10B398009A4240D8A3EB0208FB69984528BF984613
:10B3A800059B08F1030803F5106303EB4A134FEA02
:10B3B80098080693069B9969D7E9093289B24145ED
:10B3C80027D393420BD80121059B0AF00F00D3F82D
:10B3D8003428814022EA0102C3F834281BE0A3EB99
:10B3E8000209FB69079A994528BF9946A3790598E8
:10B3F8000093396A1FFA89F32DF0D9FC3B6A09F1E9
:10B4080003084B443B62BB6A4FEA98084B44BB6253
:10B41800D0E79342D7D9049B0AF1010A5B08049349
:10B4280024370BF1200B68E520462CF023F97DE545
:10B4380020462CF010F9A9E599601A68203322F407
:10B44800001243F8202CC3F8E811D3F8E02122F4C5
:10B458000012C3F8E021D3F8E02142F00062C3F8FB
:10B46800E021039A01320392A1E500BF0A30544F4C
:10B478000A31544F6B6943F4005343F02B036B615B
:10B488002B6943F00B032B61A8E501222427B3693C
:10B4980004F2572023F08003B36106F53263217963
:10B4A80091427FF6DBAD07FB02F1415C012907D130
:10B4B800196841F000611960196841F0804119600C
:10B4C80001322033EBE798F83C30D9F80020012B03
:10B4D80009D1002A07DA67F07F01204688F83B3057
:10B4E800C9B22DF00FFA013708F1240809F1200933
:10B4F800BDE5013224332031CBE500BF022A4AD111
:10B50800274B284A0B44934239D9274B274A0B44E7
:10B51800934236D9264AA1F57403A3F510539342F2
:10B5280031D9244AA1F18373A3F5E74393422CD37D
:10B53800214B224A0B44934229D9214B214A0B44DF
:10B54800934226D3204B214A0B44934223D3204ACB
:10B55800A1F1B773A3F5585393421ED31D4B1E4A4E
:10B568000B4493422CBF06230723C26822F470526F
:10B57800C260C26842EA8323C360002070470F2379
:10B58800F3E70E23F1E70D23EFE70C23EDE70B2399
:10B59800EBE70A23E9E70923E7E70823E5E700BF24
:10B5A800405327FFFF340C00401E1BFF3F420F0093
:10B5B8007F4F120020D6130060B6E5FE5FE3160049
:10B5C80000D3CEFE40771B00C05BB3FEC0912100C4
:10B5D80020753800E05459FEE09C410084B0F8B56D
:10B5E800044607A880E80E00002319469DF81C5061
:10B5F8009DF8266003F14002013304EB82020F2B11
:10B608005160F7D1A36B04F5006723F00073A363BF
:10B61800002E4BD17B6843F002037B60A36B43F0A1
:10B628008073A363A36B43F40003A3630023C4F8EC
:10B63800003E9DF82130032B42D19DF81F100029B0
:10B648003CD120462DF089FA102120462DF041FAF0
:10B65800014620462DF060FA00230843C0B20038A6
:10B668003B6118BF01207B6104F51062FB61002D6E
:10B678004FD0D4F80019994224DA4FF00061C4F889
:10B68800001900214FF67F3C01339D421161C2F839
:10B6980008C002F1200218D9D2F800E0BEF1000F6C
:10B6A80010DA4FF0904EC2F800E0EDE7A36B23F0FC
:10B6B8008073A363A36B23F40003B6E70121C0E7FB
:10B6C8000321BEE700211160DBE7D4F8002B04F565
:10B6D8003063002A19DA4FF00062C4F8002B002208
:10B6E80000214FF67F3C013295421961C3F808C02A
:10B6F80003F120030DD9D3F800E0BEF1000F05DAFD
:10B708004FF0904EC3F800E0EDE7002200211960E9
:10B71800E6E73B6923F480733B610023A3616FF084
:10B72800804363619DF81E301BB9A36943F0100381
:10B73800A361A2690A4B1343A3619DF822301BB190
:10B74800A36943F00803A361012E01BFA36943F075
:10B75800804343F00403A361BDE8F84004B0704798
:10B7680000383C8030B54A780B78012A00EB431347
:10B7780000F5006029D1D3F80029002A0BDAD3F8A4
:10B78800002942F00062C3F80029D3F8002942F0EA
:10B798008042C3F8002901240A78C56B02F00F0221
:10B7A80004FA02F225EA0202C2630978C26901F0CA
:10B7B8000F018C4022EA0402C261D3F80019174A2B
:10B7C8000A40C3F80029002030BDD3F8002B002A16
:10B7D8000BDAD3F8002B42F00062C3F8002BD3F841
:10B7E800002B42F08042C3F8002B01240A78C56B75
:10B7F80002F00F0204FA02F225EA0242C263097853
:10B80800C26901F00F018C4022EA0442C261D3F8F8
:10B81800001B034A0A40C3F8002BD4E7007833EC36
:10B828000078F3EFF7B54B780F78012B6C4EDFF803
:10B83800B4C100EB471440F089800D6904F510632A
:10B8480045BB1D6935401D611D6945F400251D6115
:10B858001D6905EA0C05012A1D614CD1CA6902B1AE
:10B868005A610B79012B0CD1D0F8083813F4807F7A
:10B87800D4F800390CBF43F0005343F08053C4F8A8
:10B888000039D4F8003943F00443C4F800390020E3
:10B8980003B0F0BD1D6905EA0C051D611D69354041
:10B8A8001D610D698E6867B9B54288BF0E611D6953
:10B8B80045F400251D610D691E69C5F31205354360
:10B8C800C9E73544013DB5FBF6F5474FD3F810C03D
:10B8D800AEB207EAC54545EA0C051D610D79012D93
:10B8E800E9D11D6925F0C0451D611F69750705F07F
:10B8F800C0453D43DEE7D4F8003943F00443C4F8BB
:10B9080000390B79012B0DD00B69002BBFD0012317
:10B918000A78D0F8344802F00F0293402343C0F865
:10B928003438B4E7D0F8083813F4807FD4F80039F5
:10B938000CBF43F0005343F08053C4F80039009221
:10B948000B8A0A78C9682DF032FAA0E7D4F8105BA0
:10B9580004F5306305EA0C051D611D6935401D615C
:10B968000E698D683FBB06B10D610D621E69C5F396
:10B97800120535431D611D6945F40025012A1D6125
:10B9880002D1CA6802B15A610B79012B0CD1D0F8E7
:10B99800083813F4807FD4F8003B0CBF43F0005301
:10B9A80043F08053C4F8003BD4F8003B43F0044311
:10B9B800C4F8003B6BE7002ED8D02E44013EB6FBFE
:10B9C800F5F6B6B275430D62074D1F6905EAC6451F
:10B9D8003D431D610D6A1E69C5F312053543CDE768
:10B9E800FFFF07E00000F8FF0000F81F30B5114C1A
:10B9F800056C00F53063A54203D9D0F8004B002C44
:10BA080016DB00241C611C69012944F400241C6114
:10BA18001C6944F018041C611C6944F0C0441C6192
:10BA280001BF5A61D0F8003B43F08023C0F8003BC7
:10BA3800002030BD0A30544FA0B1194BDB6813F415
:10BA4800803311D0174B184A0344934220D9174A20
:10BA5800174B02449A421DD3164A02449A421DD3F8
:10BA6800984219D901207047134A144902448A425E
:10BA780014D38842F6D812490A6822F00F021A43F2
:10BA88000A60086800F00F00C01A18BF012070474C
:10BA98000323F0E70223EEE70023ECE70123EAE7BC
:10BAA80000080246FF2747FAFF083D00FF6F2FFCFA
:10BAB8000048E801FFB717FEFFED85FF00127A0086
:10BAC8000020024010B50A46044619B1024B002175
:10BAD8001B68984710BD00BFCC0600200346002015
:10BAE800094AC3E900009A6002F18832DA6002F17B
:10BAF8002942A2F59612A2F68B621A61A2F1883247
:10BB08005A61024A9A61704701234567F0E1D2C33E
:10BB18002DE9F04F4B68AFB01BBA08930B69D1F809
:10BB280000E093FA83F84B698E6893FA83FA8B697D
:10BB3800CD681BBA0A93CB6901901BBA12930B6AA2
:10BB48009EFA8EFE93FA83FB4B6A36BA1BBA0B93A6
:10BB58008B6A2DBA1BBA0C93CB6A1BBA0D930B6B6D
:10BB68001BBA0E934B6B1BBA03938B6B1BBA0493D4
:10BB7800CB6B1BBA059383680F93C3680293036961
:10BB88000F9906934369029F10938369109A139340
:10BB9800069B83EA0200029B18405040DF4B139A31
:10BBA80003EBB7071A4402EBF16210440299069AB4
:10BBB800704482EAB1020F992F440A4006998EEA2E
:10BBC800060E4A4010998EEA0B0E19440A44089949
:10BBD8000A440F9902EBF0624FEAB10C02998CEA21
:10BBE800B104044084EAB1040699194431440C4470
:10BBF8008CEAB001114004EBF26481EA0C014FEACF
:10BC0800B202394482EAB00727409C4401EBF46150
:10BC1800C44482EAB40987EAB007674409EA01091B
:10BC28000AEB030C07EBF1670CEBB00C4FEAB10120
:10BC38000A9889EA0209E14481EAB40C0CEA070C83
:10BC4800184410448CEAB40C129A09EBF76984443E
:10BC580081EAB70000EA09001A4402EBB40248403E
:10BC680010444FEAB9020CEBF96C82EAB7040BEB0B
:10BC7800030904EA0C0484EAB704894404EB0901C3
:10BC8800DDF82C9000EBFC6082EABC040440994487
:10BC980001EBF06109EBB7094FEAB0000C9F544083
:10BCA8004C4480EABC0909EA01091F44174489EA9F
:10BCB800BC090D9A04EBF164B94480EAB107274046
:10BCC8001A4409EBF46902EBBC024FEAB404DDF84C
:10BCD80038C04740174484EAB10202EA09029C448A
:10BCE800844482EAB1026244DDF80CC007EBF967CC
:10BCF80084EAB90038409C4402EBF7620CEBB10CC3
:10BD08004FEAB70704996040604487EAB90C0CEA27
:10BD1800020C194421448CEAB90C059C00EBF26032
:10BD28008C4487EAB20101401C4404EBB904794011
:10BD38000CEBF06C214401EBFC6903994FEAB0006D
:10BD48008EEA010103EBF17E07910899BE4481EA6E
:10BD580005070B9980EAB2044F40049904EA0C04E1
:10BD6800794084EAB204744403EBF17E0EEBB20E20
:10BD78000C9A86EA080680EABC075640059A07EA44
:10BD8800090756404740774403EBF67E86440D98F2
:10BD980085EA0A054540079804EBF96485EAF070DE
:10BDA8001190119D08914FEAF0704FEAB90107EB25
:10BDB800F467159081EAB400384003EBF57303EBA0
:10BDC800BC03484018440A9B4FEAF67288EA030805
:10BDD8000E9B149288EA0308089B81EABC0288EA51
:10BDE800F3730993099D4E4B224082EABC0203EB90
:10BDF800F57C8C441299039D724402EBF7628AEA3F
:10BE080001014FEAB70787EAB409694081EAF67188
:10BE180089EA0209E14403EBF17C0CEBB40C0A9CBF
:10BE280000EBF26084EA0B08049C87EAB20A88EA0D
:10BE38000408119C8AEA000A88EAF478E24403EBD1
:10BE4800F87C129DBC440B9F09EBF06985EA070E4C
:10BE5800059D4FEAB0008EEA050E099D4FEAF87479
:10BE68008EEAF57E03EBFE7716944FEAFE7580EABC
:10BE7800B20407EBB2070C9A1295079D84EA0904ED
:10BE88008BEA02020AEBF96A644482EAF57280EAF4
:10BE9800B90C04EBFA6482EAF1728CEA0A0C4FEAF4
:10BEA800BA0A0A9203EBF27BBC440B9A8AEAB907F6
:10BEB8000D9D6740834407EB0B0082EA0507089A4B
:10BEC8000E9D87EAF27787EAF8720B9203EBF27B12
:10BED8000C9A0BEBB90B82EA050989EAF67686EA31
:10BEE800FE760CEBF46C8AEAB4074FEAF6750D9A05
:10BEF800179587EA0C07039D5F4403EBF67BD34451
:10BF080082EA050A119A00EBFC608AEAF2754FEAA8
:10BF1800BC0C0A9A8CEAB40904E000BF9979825AE9
:10BF2800A1EBD96E85EAF27589EA000907EBF0679B
:10BF38008CEAB00AD94403EBF57B4FEAF5728AEA3A
:10BF4800070A0BEBB40B0D920AEB0B040E9ADDF803
:10BF580010A009EBF76982EA0A0A099A4FEAB707BB
:10BF68008AEAF27A0B9A04EBF9648AEAF27203EB32
:10BF7800F27B87EAB00A8AEA090AE3440C920AEBE0
:10BF88000B0C039ADDF814A00CEBF46C82EA0A0A95
:10BF98008AEAF17A8AEAF67203EBF27B039287EA7D
:10BFA800B90A049A0BEBB00B07988AEA040ADA4438
:10BFB8004FEAB40B82EAF07484EAF87484EAF57400
:10BFC8008BEAB90003EBF4784FEAF47280EA0C00CC
:10BFD800B8440E9200EB0807059A08980AEBFC6A29
:10BFE80082EAF0700C9A80EAFE7080EAF2708BEABE
:10BFF800BC0E03EBF0784FEAF07208EBB9088EEA52
:10C008000A0E1192C644149ADDF81C8007EBFA67F1
:10C0180082EAF8780A9A4FEABA0A88EAF278039A22
:10C028000EEBF76E88EAF27203EBF2798AEABC0843
:10C03800D94488EA07080492C844159ADDF8209084
:10C0480008EBFE6882EAF9790B9A89EAF27989EABB
:10C05800F47203EBF27B8AEAB70989EA0E090BEB63
:10C06800BC0B059209EB0B0C149ADDF824904FEAEF
:10C07800BE0E82EAF97989EAF67989EAF0794FEA17
:10C08800F97214928EEAB706159A03EBF97B86EAE1
:10C098000806D34406EB0B0A82EAF176049A86EA8C
:10C0A800F57686EAF2764FEAF67203EBF67B15929E
:10C0B8000BEBB70B169A099F0CEBF86C82EAF77733
:10C0C8000C9A8EEAB80587EAF277059A85EA0C0594
:10C0D80087EAF27207925D4403EBF27B129A0AEB4D
:10C0E800FC6A82EAF1714FEABC0C039A8CEAB80741
:10C0F800F34481EAF27187EA0A075F4481EAF97B2F
:10C1080005EBFA658CEABA0E03EBFB7101EBB8019B
:10C118008EEA050E169A8E440A9907EBF56782EAAD
:10C12800F17181EAF47484EAF6744FEAF47203EB6D
:10C13800F4781692E044129ADDF82CC04FEAB5055F
:10C1480082EAFC7C079A8CEAF07080EAF2700EEBC7
:10C15800F76E85EAB70C03EBF0734FEAF07203EB66
:10C16800BA038CEA0E0C12929C440A9A179B85EA31
:10C17800BA0183EAF272049B794082EAF37282EA96
:10C18800FB730893089AE74B414401EBFE6103EB0C
:10C19800F272154441EABE020CEBF16C01EABE08EA
:10C1A80002EAB70205EBFC6542EA08022A44DDF818
:10C1B8002C800D9D85EAF875DDF8148085EAF87500
:10C1C80085EAF4754CEAB108099508EABE080CEA54
:10C1D800B10548EA0505DDF8248003EBF87808EB9B
:10C1E800B70805EB0807179DDDF8308007EBF26705
:10C1F80085EAF87888EAF97888EAF0784FEAF875F5
:10C208000B9503EBF87505EBBE0E42EABC0502EA96
:10C21800BC0905EAB10545EA09050EEBF76EAE441F
:10C22800DDF80C900D9D85EAF97585EAF676089D8E
:10C2380047EAB20986EAF5764FEAF6750D9509EAF6
:10C24800BC0907EAB20549EA050503EBF67909EBEB
:10C25800B1094D440E99DDF8309005EBFE6581EA91
:10C26800F971DDF81C9081EAF971DDF8249081EA12
:10C27800F9710A9103EBF17101EBBC0C4EEAB701BD
:10C288000EEAB70901EAB2010CEBF56C41EA0901C3
:10C298006144DDF80C90DDF844C08CEAF97C8CEA46
:10C2A800FB7C8CEAF87C45EABE09CDF80CC009EAAB
:10C2B800B70905EABE0C49EA0C0CDDF80C9003EB53
:10C2C800F97909EBB209CC440E9ADDF810900CEB21
:10C2D800F16C82EAF97282EAF47484EAF6744FEA3D
:10C2E800F4720E9203EBF47202EBB70741EAB5025F
:10C2F80001EAB50902EABE0242EA090207EBFC6755
:10C308001744DDF81490119A82EAF97282EAF07003
:10C318000A9A4CEAB10980EAF2704FEAF072119277
:10C3280009EAB5090CEAB10249EA020203EBF0791D
:10C3380009EBBE094A44DDF850E0DDF8109002EB45
:10C34800F7628EEAF97EDDF820908EEAF97EDDF854
:10C358000C908EEAF97E03EBFE7909EBB50947EA02
:10C36800BC05CDF810E005EAB10507EABC0E45EAC0
:10C378000E0509EBF269A944DDF814E0159D85EA7C
:10C38800FE75DDF824E085EAFE7585EAF475059505
:10C3980042EAB70505EABC0502EAB70E45EA0E0E01
:10C3A800059D03EBF57505EBB105AE441499079DA2
:10C3B8000EEBF96E81EAF57181EAF87888EAF0788F
:10C3C8004FEAF871149103EBF87101EBBC0C49EAE0
:10C3D800B20109EAB20501EAB70129430CEBFE6C88
:10C3E8008C4415990EEAB90581EAFB7A04998AEA20
:10C3F800F67A8AEAF17A4FEAFA7115914EEAB901AA
:10C4080001EAB2010D4303EBFA7101EBB701079E94
:10C418000D44169905EBFC6581EAF6710A9E81EADE
:10C42800F671059E81EAF67103EBF17707EBB20727
:10C438004CEABE02079102EAB9020CEABE010A43BD
:10C4480007EBF5671744129A05EABC0182EAFB7B01
:10C45800039A089E8BEAF27B45EABC028BEAF87BDA
:10C4680002EABE02114303EBFB7202EBB90211446C
:10C47800169A01EBF76182EAF67686EAF47686EA9E
:10C48800FA764FEAF672169203EBF67447EAB502AB
:10C4980004EBBE0402EABC0207EAB50E42EA0E0249
:10C4A80004EBF1641444DDF824E0129A82EAFE7287
:10C4B80082EAF070079A41EAB70E80EAF2720C92AB
:10C4C8000C984FEAF27212920EEAB50E01EAB70220
:10C4D8004EEA020203EBF07E0EEBBC0E089802EB6C
:10C4E8000E0C0B9A0CEBF46C82EAF072049804EAD6
:10C4F800B10E82EAF07282EAFB72089203EBF272E2
:10C5080002EBB50244EAB10505EAB70545EA0E05AE
:10C5180002EBFC622A440D98099D0CEAB40E80EAED
:10C52800F57501E0DCBC1B8F059885EAF07585EA96
:10C53800F6704CEAB40505EAB10545EA0E0E03EBC0
:10C54800F07505EBB7050990AE44DDE90A5080EABD
:10C55800F5750C9885EAF87585EAF0754FEAF57770
:10C56800179703EBF57707EBB10742EABC010EEB2F
:10C57800F26E02EABC0801EAB40141EA080107EBDD
:10C58800FE670F4403980D994EEAB20981EAF071EB
:10C59800089881EAFA7181EAF07109EABC090EEAA1
:10C5A800B20803EBF1734FEAF17049EA080803EBAC
:10C5B800B4030D9008EB03040A980E9B4FEABE0AD9
:10C5C80083EAF07307988AEAB20E83EAF07309984F
:10C5D8008EEA070E83EAF0730A930A98DF4B04EB9E
:10C5E800F76403EBF07808EBBC081198DDF80CC091
:10C5F800C64480EAFC7C8CEAFB7C8CEAF57003EB91
:10C60800F07C0B900CEBB20C04980E9A8AEAB708EF
:10C6180082EAF07989EAF67989EAF1790EEBF46E23
:10C628004FEAF97288EA04084FEAB4040E92E0442B
:10C6380003EBF97284EAB70C52448CEA0E0C0598A5
:10C648009444119A08EBFE6882EAF0760C9A0CEB97
:10C65800F86C86EAF2760A9A86EAF2764FEAF67279
:10C668000C9203EBF67084EABE0200EBB70082EA94
:10C678000802149F02444FEAB800DDF8108080EAEF
:10C68800BE0A87EAF877DDF820808AEA0C0A87EA8A
:10C69800F877DDF82C8002EBFC6287EAF8774FEA3E
:10C6A800F777039719971F442744BA44159C059FA9
:10C6B8000AEBF26A84EAF774099F84EAF77484EA59
:10C6C800F9744FEAF4740494049F1A941F4480EA9E
:10C6D800BC0407EBBE0754404FEAB20205923C4443
:10C6E800149A079F04EBFA6482EAF77888EAF578E7
:10C6F800059A88EAF6784FEAF87882EABC0508EBEA
:10C708000307159A074485EA0A053D4482EAFB7740
:10C7180087EAF1770399059A4F404FEAF77782EA5B
:10C72800BA00F91801EBBC016040169A0844079951
:10C7380005EBF46582EAF1710A9A4FEAB40481EADA
:10C74800F271049A84EABA0E51404FEAF171059ADF
:10C7580001EB030C94448EEA050E129AE644DDF8C8
:10C768002CC082EAFB7282EAFC7282EA08024FEA73
:10C77800F27200EBF56084EAB50C02EB030B0BEBED
:10C78800BA0B8CEA000CDDF858A0DC44DDF820B0C8
:10C798000EEBF06E8AEAFB7A8AEAF97A8AEA070AE5
:10C7A8004FEAB0004FEAFA79CDF81490CDF87C90B2
:10C7B80080EAB50A9944A1448AEA0E0A129CCA443E
:10C7C800DDF824900CEBFE6C84EAF97484EAF674C4
:10C7D8004C404FEAF4740794209480EABE061C4447
:10C7E80004EBB50486EA0C062644179C039D84EAEC
:10C7F800FB746C4054400AEBFC6A4FEAF4744FEA4D
:10C80800BC0C8CEABE09E518054489EA0A09CDF88A
:10C818006C801C971D911E92A9442194099D0D9826
:10C8280006EBFA6680EAF570049D09EBF669684044
:10C83800059D68404FEAF0708CEABA0500EB030BDF
:10C848000BEBBE0B7540DDF85CE05D44DDF828B00D
:10C858004FEAB6068EEAFB7E8EEA080EDDF81C80EB
:10C8680005EBF9658EEA080E4FEAFE7E0EEB030B28
:10C8780086EABA08E34488EA0908DDF834C0D844EF
:10C88800DDF82CB008EBF5688CEAFB7C8CEA070C29
:10C898008CEA040C4FEAFC7786EAB90407EB030C30
:10C8A8000CEBBA0C6C40DDF828A06444DDF838C005
:10C8B8004FEAB5058CEAFA7C8CEA010C8CEA000C8C
:10C8C8004FEAFC7101EB030CB4440C9E229086EAFB
:10C8D800FB76564086EA0E0685EAB9004FEAF676F8
:10C8E80004EBF864269685EAB80280EA08001E443C
:10C8F80006EBB9066044624000EBF460324402EB98
:10C90800F06C039E0E9A4FEAB4045640059A249799
:10C9180056407E404FEAF67627961E440C9A2E44DF
:10C92800049D84EAB8075540079A474055404D4052
:10C938004FEAB00018954FEAF5752591289584EAD5
:10C9480000011D4481EA0C01374405EBB80507EBEB
:10C95800FC674B190F994FEABC0201E0D6C162CAC5
:10C9680003EBF763CDF88CE02D942A972C9029934C
:10C978002B920B4401998B60029B1F44069BCF604E
:10C988001A44109B0A611844139B48611C448C612B
:10C9980018A85821FFF796F800202FB0BDE8F08FAF
:10C9A80003460846C1B9C3E910110D4A0D49DFF81D
:10C9B80038C0C3E912120D4A0D49C3E914C20D4A21
:10C9C800C3E916120C4A1A6602F17452A2F5230240
:10C9D800A2F692425A6670476FF07300704700BF24
:10C9E80085AE67BB67E6096A72F36E3C3AF54FA5F8
:10C9F8007F520E518C68059BABD9831F2DE9F04FF0
:10CA08000446CFB0039100F1480346AD00F1680633
:10CA18002A4618685968083303C2B3421546F7D145
:10CA2800DDE94883DDE94B96DDE946154FF0000C5A
:10CA380001933E4BDDF834B14A9804AA0293BCF145
:10CA48000F0F5BD8039B53F82C301BBA4FEAF02E1C
:10CA580086EA0907DDF808A08EEAB01E07408EEACC
:10CA6800706E774077445AF804EB936077443B4400
:10CA780045EA010E4FEA7137CDF808A087EAB107F9
:10CA88000EEA080E05EA010A4EEA0A0E87EAB157CD
:10CA980077440CF1010CDDF804E05B44BCF1400F75
:10CAA8009E44B3463B4402F10402CDF804801ED1F3
:10CAB800CDE94C96CDE94AE0CDE94858CDE9463173
:10CAC800CDE9043745A904F14403643453F8042F2D
:10CAD80051F8040FA34202441A60F7D104A84FF496
:10CAE8009471FEF7EFFF00204FB0BDE8F08FA84625
:10CAF8004E460D46814619467046A0E7136852F81F
:10CB080034AC4FEAF34E8EEA734E52F8387C8EEA14
:10CB1800932E52F8143C3B444FEABA4787EAFA1777
:10CB2800734487EADA073B4490E700BFC0B70408BC
:10CB380010B50446F6F7C4F803480121034A28F063
:10CB480010FF20462CF065FB20B10408D1710508C0
:10CB58002DE9F84304460D4600AFEFF31188102382
:10CB680083F31288BFF36F8F0428294A98BF294B93
:10CB7800E9468AB09668117C98BF53F820306A4617
:10CB880088BF254BC2E9073140F20133234893841B
:10CB9800234BC2E9050442F8103F00234FF43151FA
:10CBA8002048F6F75DF9CD4645B1EB69C3F30803B4
:10CBB80023B101211C4A1B4828F0D3FE2EB1304670
:10CBC8002CF0AEFD08B1037803B91848E9468AB0DD
:10CBD8006A46174BD061C2E9053640F20133138427
:10CBE800144B42F8103F00234FF411510D48F6F74B
:10CBF80037F92946CD462046FFF79AFF88F3118872
:10CC0800BFF36F8F3046F6F7DDFFBD46BDE8F8830A
:10CC180050360020C0B80408E0710508F671050810
:10CC28000500000120B104081E720508EE71050810
:10CC38003F7205080400000138B50A4B53F820403C
:10CC4800013053F82050A54200D838BD606830B193
:10CC5800037EDB0701D42CF0B9FA0834F3E7236824
:10CC68009847FAE7D4B80408012270B5294B032085
:10CC780086B01A70FFF7E0FF01F028FC0420FFF7E8
:10CC8800DBFF254C254D2646AE4204F1300410D377
:10CC980000F072FF204C224EAC4226D300F080FFF9
:10CCA80027F0CBFE1F4A938923F00103938106B036
:10CCB80070BD54F80C3C059354F8103C049354F898
:10CCC800143C039354F8183C029354F81C3C019309
:10CCD80054F8203C009354E90A2354E90C0100F06D
:10CCE80035FD54F8303C5E65CDE7D4E90A23B3F14D
:10CCF800FF3F08BFB2F1FF3F05D052EA03012068A9
:10CD080003D101F01FF83034C6E73146183001F07E
:10CD1800C5F9F8E7123E002008AF040838AF040848
:10CD28000998030860210020A02370B5134E012242
:10CD380003FB0066002386B0CDE904230F2201938C
:10CD4800CDE9023214234FF4A0720D4D0D4903FBB7
:10CD58000055044602FB00110B4B3046009500F0CD
:10CD6800F5FC337C2C7423F004033374074B013433
:10CD780003EBC423EE606B6006B070BDC0200020DA
:10CD88005036002088580020A393030888500020BC
:10CD9800BFB50020FFF750FF294B03F5006282F36F
:10CDA800088883F30A880024F023264D264F85F847
:10CDB8002230EC772C766C76AC7685F820406B6A5E
:10CDC80043F4E0236B62F6F7B7FEF7F703F84FF08A
:10CDD800FF33AB62EB62F7F7A7F9F7F725F8F5F73A
:10CDE800D5FE1A4800F034FD28F014FD0120FFF7A5
:10CDF80023FF0220164DFFF71FFF00F005FF154B1C
:10CE080015495D61154B45F6E062059301232846F7
:10CE1800CDE90343CDE901443B46009400F096FC7C
:10CE280006462A7C284622F004022A742CF0B4FC18
:10CE38002046FFF779FF3A4631462846F6F7A8FF1D
:10CE48008850002000ED00E071CC0008002200208E
:10CE58006021002050360020C8590020C65405081B
:10CE680038B5064C064DAC4201D3002038BD2046EB
:10CE7800D4E901122CF017FA1434F4E7D80E002084
:10CE8800EC0E002030B5054B85B0DDE9084502936E
:10CE9800CDE900452CF0C5F905B030BD174F0308A2
:10CEA800002038B5054C064DAC4200D338BD2046AD
:10CEB8002CF01DFA0028F9DB1C34F5E7BC0E002025
:10CEC800D80E002073B50C46EFF31181102585F3B9
:10CED8001288BFF36F8FC5685DB125602B68C3608A
:10CEE800836901338361002081F31188BFF36F8F59
:10CEF80011E052EA030603D16FF00B002560F3E757
:10CF0800CDE900230246083000F07CFD18B9034B38
:10CF18009B685B69236002B070BD00BF503600207B
:10CF28002DE9F34104460E469DF8200004F1080857
:10CF3800EFF31187102181F31288BFF36F8F256AF1
:10CF4800E1688D4247D22568AC4218D0BDB1284669
:10CF58002CF02EFA05F118002CF01CFD3146A268C1
:10CF680068693DF0F8FC00232846C5F898302CF095
:10CF780013FC4046394600F0D9FD002038E0A2688D
:10CF8800D8B13146E0693DF0E6FCE369A268134494
:10CF98006269E361934201D12369E361236A102145
:10CFA8000133236204F124002CF0D3FD0028E0D1E2
:10CFB80087F31188BFF36F8F1AE0A169236999423B
:10CFC80008BF6369314608BFA361A069801AA061E0
:10CFD8003DF0C1FCE2E752EA03010CD007494046A4
:10CFE80089684E61CDE900233946224600F00AFDE2
:10CFF80002B0BDE8F0816FF02200D9E7503600207A
:10D00800F7B50446084604F10807EFF31186102126
:10D0180081F31288BFF36F8F216A00293AD0A26882
:10D02800A1693DF098FCA369A26825681344626968
:10D03800A361934204BF2369A361236AAC4203F14D
:10D04800FF33236234D02846002D32D02CF0B0F9BB
:10D0580005F118002CF09EFCA2686969E0693DF0B2
:10D068007AFCE369A268284613446269E361934243
:10D0780004BF2369E361236A013323620024C5F8EE
:10D0880098402CF089FB3846314600F04FFD204689
:10D0980003B0F0BD52EA030110D00A49896848611B
:10D0A800CDE9002331462246384600F0ABFCEFE7D5
:10D0B800002086F31188BFF36F8FE9E76FF0220035
:10D0C800F7E700BF503600202DE9F3410446174624
:10D0D8001E46EFF31188102383F31288BFF36F8F76
:10D0E800C368314A7BB180689168884219D057EA91
:10D0F800060318D188F31188BFF36F8F6FF00F0004
:10D1080002B0BDE8F081916891F90E100133E36037
:10D1180093682161A36088F31188BFF36F8F0020A3
:10D12800EEE72169F2E790F90E3091F90E10994275
:10D13800A8BF19468B422DDD2CF0A4F905462246DE
:10D148004146CDE90076194800F05CFC0028E6D09D
:10D15800EFF31186102383F31288BFF36F8FA06853
:10D16800D0B1236821699C420AD04BB193F90E30A3
:10D178009942A8BF19466FF07F039942B8BF194674
:10D188002CF080F940B13146084800F0CFFC6FF030
:10D198000A00B5E70025D2E7002DF4D186F31188FF
:10D1A800BFF36F8FF3E700BF50360020133E002017
:10D1B800F8B583680546002B40D0234A926893420D
:10D1C8003FD1C368012B03D9013BC3600020F8BDE0
:10D1D800EFF31187102383F31288BFF36F8F016970
:10D1E80080682CF04FF92C68AC4207D10023C5E9C0
:10D1F800023387F31188BFF36F8FE7E7002CF5D070
:10D20800D4E90032002613605A60237CC4E9006622
:10D2180023F002032374A66004F118002CF0BAFB73
:10D22800AC6094F90E3020462B61C4F898602CF05D
:10D23800B3FA3946054800F079FCC7E76FF01500E6
:10D24800C5E74FF0FF30C2E750360020133E0020FC
:10D2580037B51146EFF31185102282F31288BFF318
:10D268006F8F04689CB12368426823F003039442DB
:10D27800036008BF4360012120462CF090F9044662
:10D2880085F31188BFF36F8F204603B030BD51EA94
:10D298000302F5D000F10802CDE900131046294633
:10D2A80000F0B0FB0028EFD1014B9B685C69EBE70D
:10D2B8005036002070B5EFF31186102383F31288DF
:10D2C800BFF36F8F0468A0421BD0D4B1D4E90032F9
:10D2D800002513605A60237CC4E9005523F002033B
:10D2E8002374A56004F118002CF054FB2046C4F800
:10D2F80098502CF051FA3146BDE87040094800F0CA
:10D3080015BCD0E902329A4218BF0133022183606A
:10D3180010302CF01EFC0028EDD186F31188BFF3E5
:10D328006F8F70BD133E002013B5EFF311811024E9
:10D3380084F31288BFF36F8F846844B1013C846022
:10D3480081F31188BFF36F8F002002B010BD52EA3D
:10D35800030406D181F31188BFF36F8F6FF00F00BC
:10D36800F3E7CDE900230246014800F04BFBECE768
:10D37800133E00202DE9F8430546EFF311881023EA
:10D3880083F31288BFF36F8F00266FF00A093746C0
:10D398002C68A54216D0ACB1D4E9003213605A60AB
:10D3A800237CC4E9007723F002032374A76004F107
:10D3B80018002CF0EFFA2046C4F898902CF0ECF9FD
:10D3C8000126E5E700230221AB6005F110002CF0EF
:10D3D800C0FB30B92EB988F31188BFF36F8FBDE851
:10D3E800F8834146BDE8F843014800F09FBB00BF01
:10D3F800133E00202DE9FF41044610274E4EEFF35F
:10D40800118887F31288BFF36F8FD4F8A450F5B949
:10D41800022104F1BC002CF003F9002868D004F1C3
:10D42800B4050022012128462CF049FA0028F8D139
:10D4380000234FF0FF3202934FF0FF334146CDE90E
:10D4480000233E4804F1AC0200F048FDD7E7D4F8C9
:10D45800A8202B689542C4F8A43008BFC4F8A830A7
:10D46800D4F8BC3043F00203C4F8BC30EB6823F0B6
:10D47800040343F00103EB606B6888F31188BFF382
:10D488006F8F28469847EFF3118887F31288BFF308
:10D498006F8FEB68D80623F0010236D4EA60EB6898
:10D4A8009A0716D5306823F00203EB6088B1002193
:10D4B800036870B14268954235D1036869BB7268E8
:10D4C8003360824200D17360002340F8083BFFF7C5
:10D4D800F1FED4F8BC3023F00203C4F8BC3088F362
:10D4E8001188BFF36F8FDB0589D400F0ABFB86E7AB
:10D4F800D4F8BC30D9069BD5C4F8BC0088F3118891
:10D50800BFF36F8F04B0BDE8F08123F01103EB6027
:10D5180005F11000FFF7CEFEC1E70B607368834288
:10D5280008BF7160D0E723B11A6801461846134650
:10D53800BFE71A46F9E700BF74360020133E002003
:10D54800F8B5C36804469A070F46C3F340062ED4BD
:10D558005B071CD40B680BB983680B60E368DD07B5
:10D5680042BFA36802263B603D6858BF0126002DD4
:10D578003CD0204B9A68D5F8A0309A420AD0D5F80A
:10D58800BC30D807C3F3800214D46FF0120600230E
:10D598003B6025E02CF0BBF8D5F8BC300028F0D172
:10D5A800D907C3F3C002F0D552B15B0708D46FF0B6
:10D5B8000F06ECE7002AFAD1C3F3C003002BF6D11B
:10D5C80000232360D5F8A83063B9C5E92944284663
:10D5D8002CF040F8E36843F00403E3603B68A36081
:10D5E8003046F8BD1C60C5F8A840F0E76FF0150696
:10D5F800CDE700BF50360020014601482CF06BB83B
:10D60800C0220020F0B50446002089B0C4E92900F2
:10D618000E9D04F1AC00C4E92B0004F1B400C4E988
:10D628002D0055B32879002840F2011008BF0120C9
:10D63800C4F8BC0000204FF0FF364FF0FF37CDE9AB
:10D648000330CDE90100CDE9066720460C4B009474
:10D6580000F0D2F855B1296811B120462CF05DF8D8
:10D668006B791BB1A38943F00103A381204600F025
:10D6780069FBC4F8A04009B0F0BD0120D8E700BF9D
:10D68800FDD3000837B501900846EFF31184102147
:10D6980081F31288BFF36F8FC16811F01E0F16D186
:10D6A80053EA020508D101A9FFF74AFF84F311885C
:10D6B800BFF36F8F03B030BD41F00801C16001991D
:10D6C80010308161034900F0E9FC0120EEE70020F9
:10D6D800ECE700BF6B96030801460148FFF7D2BF8D
:10D6E800C0220020F7B50C4616461D460190EFF300
:10D6F8001187102383F31288BFF36F8F08462BF02E
:10D708009AFF55EA060309D1204601A9FFF718FF39
:10D7180087F31188BFF36F8F03B0F0BDE36832461B
:10D7280043F00803E360019B0449A36204F110007D
:10D738002B4600F0B3FC0120EAE700BF6B96030814
:10D7480001460148FFF7CEBFC02200202DE9F04F67
:10D75800984685B000F15803C0E91633129B00269D
:10D7680083810423073222F0070A0374119B01EB1B
:10D778000A090F46C0E90666494686608373C67380
:10D788000446DDF838B0F5F791FF109BC51D25F06C
:10D798000705C4F88850C4E9207A02930F9BA9EBC7
:10D7A8000505CDE900B32A46434639462046F6F733
:10D7B800D3FA0F9BC4E91B8B6367109B6665A3674D
:10D7C800EFF31182102383F31288BFF36F8F094B95
:10D7D800196A1C62E16782F31188BFF36F8F9B6837
:10D7E8000BB1D3F88C302846C4F88C3005B0BDE8AE
:10D7F800F08F00BF50360020F0B5002587B00595A2
:10D80800109DDDE9127604950F9D044603950E9D43
:10D8180002950D9D01950C9D0095FFF797FFB6F1B8
:10D82800FF3F08BFB7F1FF3F05D056EA070305D110
:10D83800204600F087FA204607B0F0BD3A46334646
:10D8480004F11800014900F029FCF4E709980308DD
:10D858000123037483810023C0E92033C0F88C308E
:10D86800014B9860704700BF503600206FF00A01E6
:10D87800094A9368C3F898100849C3F894004B689C
:10D8880043F080534B60002383F31188BFF36F8FFD
:10D898009368D3F8980070475036002000ED00E0F8
:10D8A80070B590F91020037C002A36DBD90634D1F4
:10D8B8001B4C63F07F032246037452F8183FE1695A
:10D8C800934207D1C0E900210860E06111E0994264
:10D8D800F8D01B68002BF5D090F90E5093F90E6024
:10D8E800B542F4D0AE42F2DD5968C0E900310860B3
:10D8F8005860A569954200D005B9E568A3681A7C07
:10D90800D20604D1DA897F2A01D9AA6932B1AB4299
:10D9180002D0284600F024FB656170BD6361FCE716
:10D928005036002038B590F910200146002A037CB3
:10D9380004DA03F07F0303742BF0F4FE0D4D2A463E
:10D9480052F8184FAB68944200D004B9EC688B4287
:10D9580007D01A7CD20604D1DA897F2A01D9A269B4
:10D968002AB1A34202D0204600F0FAFA23466B619E
:10D9780038BD00BF50360020B3F1FF3F08BFB2F1F9
:10D98800FF3F03D00249183000F088BB704700BF42
:10D998000998030838B5194CA168E0690B688142F9
:10D9A80014BF1A46002249680B605960A368E169F0
:10D9B8002AB9134AC3E900210B60E3610CE093F92B
:10D9C8000E0092F90E50A84214D0854212DD51681B
:10D9D800C3E900210B605360A569094B9D4200D043
:10D9E80005B9E568A3689D4202D0284600F0B8FA58
:10D9F800656138BD9142DCD01268D9E75036002005
:10DA080068360020F8B5DDE906670D4B0C469868C6
:10DA180011460C4A1060EFF31182102282F312882B
:10DA2800BFF36F8F9D6828462BF08EFE284632463E
:10DA38003B46FFF7A1FF2046BDE8F840FFF716BFB9
:10DA4800503600207C360020F8B50446EFF31187E5
:10DA5800102383F31288BFF36F8F037C49B203F05E
:10DA68001F02002A0CBF0126002639D103F07F03CC
:10DA78002D4D03742BF056FE2A46037C817363F008
:10DA88007F03037452F8183F934227D1E869C4E929
:10DA980000200460EC610FE09842F8D01B68002B6E
:10DAA800F5D093F90EC06145F6D08C45F4DD596880
:10DAB800C4E900310C605C60AC69944200D004B9E0
:10DAC800EC68AB689C4202D0204600F049FA6C61D1
:10DAD80087F31188BFF36F8F3046F8BDE869DEE73A
:10DAE8009B071ED585682BF01DFE81732B689D4210
:10DAF80009D16B68C4E900531C606C60E8E76A6888
:10DB08009342F6D01B68002BF3D093F90E20914274
:10DB1800F5D08A42F3DD5A68C4E9003214605C60CB
:10DB2800D6E78173D4E700BF5036002049B9EFF338
:10DB3800058030B9054B5A699B689A4201D0FFF7B6
:10DB480095BE81F31188BFF36F8F70475036002060
:10DB5800034648B9EFF3058232B9064A516992681B
:10DB6800914201D0FFF782BE83F31188BFF36F8F14
:10DB7800704700BF50360020EFF31181102383F364
:10DB88001288BFF36F8F054B9A68D37B013BD37321
:10DB980081F31188BFF36F8F704700BF50360020A4
:10DBA80070B5EFF31186102383F31288BFF36F8FDC
:10DBB800144DAB68DA7B0132DA732A4652F8184FF3
:10DBC800944200D004B9EC681A7CD20604D1DA89F0
:10DBD8007F2A01D9A2692AB1A34202D0204600F0C7
:10DBE800BFF923466B6186F31188BFF36F8FEFF39C
:10DBF8001180102383F31288BFF36F8FBDE8704044
:10DC0800FFF7A6BF50360020024B03F11802C3E904
:10DC1800062270475036002008B5FFF715FF70B18F
:10DC2800074B9B68DB7B53B9EFF31180102383F319
:10DC38001288BFF36F8FBDE80840FFF789BF08BDA2
:10DC48005036002070B5EFF31186102383F3128845
:10DC5800BFF36F8F1B4CA168E0690B68814214BF4A
:10DC68001A46002249680B605960A368E1692AB91D
:10DC7800154AC3E900210B60E3610CE093F90E003B
:10DC880092F90E50A84218D0854216DD5168C3E9B2
:10DC980000210B605360A5690B4B9D4200D005B96C
:10DCA800E568A3689D4202D0284600F059F96561ED
:10DCB8003046BDE87040FFF7D9BD8A42D8D0126817
:10DCC800D5E700BF5036002068360020F8B550EA86
:10DCD800010306460C4603D1FFF7B4FF0020F8BD48
:10DCE800EFF31187102383F31288BFF36F8F124D60
:10DCF800124BA8681860FFF715FEA868234632463D
:10DD08000F49183000F0CAF9AA680446137C38464F
:10DD180043F004031374FFF7A9FDAB68D3E90A23A2
:10DD2800B3F1004F08BF002AD8D12BF05BFE201AB0
:10DD380020EAE070D3E700BF503600207C36002090
:10DD48000998030838B50446EFF31185102383F3C7
:10DD58001288BFF36F8F037C5B070FD518302BF049
:10DD680019FE237C204623F004032374FFF798FD53
:10DD78002946BDE838400448FFF7D8BE85F3118826
:10DD8800BFF36F8F38BD00BF133E0020014B98686A
:10DD9800704700BF503600202DE9F84304468789B4
:10DDA800EFF31185102383F31288BFF36F8F037C81
:10DDB800190705D585F31188BFF36F8FBDE8F88380
:10DDC800D90943F0080260D10274A36813B1204650
:10DDD8002BF0B0FC04F118002BF0DCFDA66D04F16B
:10DDE8005808B04511D04FF0000976B130462BF0F5
:10DDF800A1FC06F118002BF0CDFD3046C6F898902E
:10DE0800FFF74EFDA66DB045EFD1DFF8C480D8F816
:10DE180008309C4241D1EFF30589B9F1000918BFD8
:10DE28004FF00109D8F818602A4A964200D00EB976
:10DE3800D8F80C60B34202D0304600F091F8204682
:10DE4800C8F8146027F004FF204600F0DBF8B9F1A9
:10DE5800000F02D02048FFF7FBFCD8F808309C429E
:10DE680031D1EFF3058373BBA289D20718D42846B2
:10DE7800FFF7FCFCFB07A1D5002383F31188BFF350
:10DE88006F8F0423184602DF98E703F07F0343F0FF
:10DE9800080303742BF046FC97E74FF00009C1E72D
:10DEA80085F31188BFF36F8F83F31188BFF36F8FEA
:10DEB8000423184602DFEFF31180102383F312883E
:10DEC800BFF36F8FD4E785F31188BFF36F8FD1E766
:10DED800503600206836002000220020D3B5DDE946
:10DEE8000667089CCDE90067FFF78CFD1CB1034B62
:10DEF8009B685B69236002B0D0BD00BF503600202C
:10DF0800027C034612F01F0210D10A4988420DD044
:10DF18000949086868B1D9897F2909D893F90E2079
:10DF2800064B1B689A42B8BF002070470020704714
:10DF380010467047C0200020D00600208036002000
:10DF48000122044BC01A044BC0105843034B1A5407
:10DF5800704700BFA0220020ABAAAAAA133E002047
:10DF680070B50D4B0D4D1E7CFFF7CAFF06EB46033F
:10DF780005EBC305044628462BF00CFD0022084B90
:10DF88009A553CB1621E2846BDE870400549D31732
:10DF980000F084B870BD00BF50360020A0220020D9
:10DFA800133E002049DF000838B5EFF31185102330
:10DFB80083F31288BFF36F8F0F4B104A9C68106869
:10DFC800A04206D1FFF7CCFF85F31188BFF36F8F0E
:10DFD80038BD00211B7C1160094AD35C002BF3D0AB
:10DFE8002046FFF78DFF0028EED0237CDB0601D109
:10DFF800FFF7D0FC2046E5E7503600207C360020AD
:10E00800133E0020EFF31181102383F31288BFF32E
:10E018006F8F0A4A136A834207D1DB6F136281F359
:10E028001188BFF36F8F70471346002BF7D0DA6F54
:10E038008242F9D1C26FDA67F1E700BF503600209B
:10E04800024B1868984208BF00207047D406002089
:10E05800034B1B680BB9FCF71DBE0020704700BFBF
:10E068008436002030B570B10B4B5B6898420AD0FB
:10E07800036843B1D3E90421D0E90445121941EBFF
:10E088000501C3E90421D0E9003213605A60002376
:10E09800C0E9003330BD00BFD4060020B3F1FF3F14
:10E0A80008BFB2F1FF3F2DE9F84F044699461546DF
:10E0B8001F467AD08160EFF31188102383F312880A
:10E0C800BFF36F8FB9F1000FDFF8E4A020DBFFF793
:10E0D800BFFFDAE90027013549F100092D1849EB9E
:10E0E800E07306464FF00109C4E90453AD1843EB49
:10E0F8000707FFF7A5FF0346DFF8B8E0DEF804A03E
:10E10800EBB9C4E900EACAF80040CEF8044028E0B8
:10E118006FF00103DAE900125B1A4FF0FF3161EB8F
:10E1280002025B1B62EB0902012B72F10001BCBF0A
:10E13800012300224FF00009C0E90432D9E7D3E9EE
:10E14800041CD4E904208A4270EB0C0B24DA891AE7
:10E158005A686CEB0000C3E90410C4E9003214608B
:10E168005C60FFF76DFF84420ED1134B1B685BB9EF
:10E17800B9F1000F02D1FFF76BFF064630462BF0CE
:10E18800F2FB0021FCF718FD88F31188BFF36F8FAD
:10E1980028463946BDE8F88F521A60EB0C009A45BC
:10E1A800C4E90420ADD01B68AAE700252F46EFE795
:10E1B800B8220020D4060020843600202DE9F0473C
:10E1C800EFF31185102383F31288BFF36F8FDFF805
:10E1D800A0900026C9F800000027FFF731FFDFF8FC
:10E1E8009480D9F80030D8E900ECD91750B1D0E9BB
:10E1F8000442A34271EB020A1BDAE41A62EB010241
:10E20800C0E90442002413EB0E034CEB0101204645
:10E21800C8E90031C9F800402BF0A5FB2146FCF7FE
:10E22800CBFC85F31188BFF36F8FBDE8F047FFF78C
:10E23800BBBE14EB0E024CEBE473C0E90467C8E9FB
:10E248000023FFF70FFF85F31188BFF36F8F8368F3
:10E258009847EFF31185102383F31288BFF36F8F6C
:10E26800D9F800301B1BC9F80030FFF7E9FEB8E702
:10E2780084360020B822002010B5EFF31184102353
:10E2880083F31288BFF36F8FFFF7E2FE0346054A58
:10E29800D2E90001181841EBE37184F31188BFF348
:10E2A8006F8F10BDB8220020F8B50646EFF311872E
:10E2B800102383F31288BFF36F8F026822B187F3AC
:10E2C8001188BFF36F8FF8BDD0E90A54691C44F177
:10E2D8000003022973F1000334D3013D44F1FF34F4
:10E2E800002CBCBF15462C462BF080FB013041F1B9
:10E2F8000001401944EB0101012871F100014ADBDA
:10E308002BF074FB6FF00203013041F1000140195A
:10E3180044EB010183426FF000438B4140DB2BF05B
:10E3280065FB6FF001024FF0FF33013041F100014E
:10E33800401944EB0104121A63EB040330461A49EE
:10E34800FFF7ACFE336B01333363336A6BB187F38A
:10E358001188BFF36F8F3046336A9847EFF3118700
:10E36800102383F31288BFF36F8F334653F8184F87
:10E378009C42A4D0002CA2D020462BF01CFA0023EB
:10E38800C4F8983087F31188BFF36F8F2046BDE833
:10E39800F8402BF001BA6FF001024FF0FF33CDE7E0
:10E3A80000224FF00043C9E7B1E200082DE9F0412F
:10E3B80005461C4690461F46EFF31186102383F34B
:10E3C8001288BFF36F8FB4F1FF3F08BFB2F1FF3F70
:10E3D80005D186F31188BFF36F8FBDE8F081002C5B
:10E3E80009DB012A74F10003BCBF0122002412F1E9
:10E3F800FF3844F1FF3728462BF0CCFADDE9060157
:10E408000023C5E90A012B6342463B4628460249D8
:10E41800FFF744FEDDE700BFB1E2000838B5034668
:10E42800EFF31185102282F31288BFF36F8FC1605A
:10E43800012181600068834206D185F31188BFF30A
:10E448006F8F0024204638BDD0E9003213605A602F
:10E458000023C0E900332BF039FB29460446024863
:10E46800FFF764FBEEE700BF143E0020F8B507464F
:10E478000C4616462BF04BF908B10020F8BD0E4BA0
:10E488009B68D3F88C50002DF7D0221DF5D2EFF3FE
:10E498001184102383F31288BFF36F8F284647F047
:10E4A8000401B04784F31188BFF36F8F0028E4D0CC
:10E4B80040F8045BE2E700BF503600200146024AFC
:10E4C8000020FFF7D3BF00BF114F0308014826F013
:10E4D80082BE00BFA172050807B5074B4FF48062E2
:10E4E800009306494FF0FF330548FFF78BF80020EB
:10E4F80003B05DF804FB00BFECB80408A8B800201E
:10E50800C0220020F0B5042804468BB02BD0344D2F
:10E51800286818B113F00EF800232B601CB3314B98
:10E528009C4220D0002601AB02932F4B214602A823
:10E53800039301962FF0AFFC01983146013012F099
:10E54800D9FF0246286070B106AF3846019931F00C
:10E5580015FF264B214604A8059304972FF09BFC32
:10E568002A68019BD65402F0D9FC32F08BF82BF0C4
:10E5780045FC01F059FC00221D4D1E4BD5F8F0401A
:10E588001A7084B1204611F0CBFF30B3A06804F0B4
:10E5980093FBD5F8F040002CF4D1D5F8F0301C46A8
:10E5A800DB68002BFBD1C5F8EC400025124C02F0CB
:10E5B80061F804F039FC12F0A5F8206812F0BAFFEF
:10E5C80025600E4C206812F0B5FF25602BF01CFB6F
:10E5D8000BB0BDE8F0402BF09CBBE468DBE700BF64
:10E5E800E037002074380020C19B0308FD020408AE
:10E5F800FC370020143E0020C4360020C03600201E
:10E60800002270B50446154B00EB8105C3E90022D2
:10E618009A60264630682DF090F9022804F1040427
:10E6280018D130680E4C206098B10E482BF0C7FD09
:10E6380020682BF011FB0C4802F018F901F03AFCA5
:10E64800064920682BF003FB0023236001F032FC0D
:10E65800012070BDA542DCD10020E3E78C36002004
:10E66800BC360020347405089FC6050810B504465A
:10E6780008482BF0F1FA01F077FD40B1064802F0A6
:10E68800F5F834B1BDE81040044802F0EFB804488A
:10E69800F5E710BD347405088EC4050871BF050878
:10E6A800BBC4050873B506462BF033FB0CF024FFFA
:10E6B80012F01EFE054612F027FE0446641B0025D4
:10E6C8000CF022FFA4F580600CF024FF01F0ACFBF5
:10E6D80000F05CFC6B464FF4006230461F49009521
:10E6E8002BF06EFA01461E4B1E4C1860009B194415
:10E6F80005F030F84FF4005201AB30461A49019545
:10E708002BF05EFA0146194B1860019B194411F071
:10E71800D9FE06F027FC2946D4F8E8000DF078FE6B
:10E728001621D4F8E8002FF0ECFF6621D4F8E800B1
:10E738002FF0E7FF40F6B651D4F8E8002FF0E1FFDC
:10E74800294604F1D8000DF063FE094804F02AF8C0
:10E758000122084B1A7002B070BD00BFD8720508BC
:10E76800C0360020FC370020EF720508C4360020B0
:10E7780087550508143E00202DE9F047092804466E
:10E78800A4B000F08F8001F069FB00287FD0002C36
:10E798007DD1464BD3F8F030002B78D0204602AD1F
:10E7A800DFF80C81FFF77EFF2BF013FD01F0ECFB87
:10E7B8004FF40071284631F0C6FDC8F8005001F04A
:10E7C80055FB0121064600F180072BF0D0FA394BA2
:10E7D800394A3A493A482FF0BAFC06A800F040FBFB
:10E7E800384937482FF0D8FCDFF8DCA0DFF8D090A4
:10E7F80006AD5146484615F8012B01342FF0CCFCE4
:10E80800202CF6D131492E482FF0A1FC31F03BFFE6
:10E8180002212F48FFF7F4FE0023C8F8003001F06A
:10E82800B9FB012338462B4A0EA932F0C4FEA0B921
:10E8380002982DF022F9039A0446014601AB0132F1
:10E848000EA832F0DDFF40B9039A019B9A4204D129
:10E85800214604983CF0AEF8A0B14FF47A702BF042
:10E86800E2FC0A231B4A0EA9384632F0A4FEDDE971
:10E87800032101AB0EA833F075F80EA833F0DBF9CD
:10E8880001F0D2FA002130462BF071FA04E020465C
:10E89800FFF708FF2BF09DFC0F4C6068FFF732FE76
:10E8A8000023636024B0BDE8F08700BFFC37002078
:10E8B80088360020097305081C7305087573050858
:10E8C80028E0040861BE05088DC6050814B10508CE
:10E8D80028B90408857305088C3600202DE9F04F07
:10E8E80089B007462BF044FC804640B1B1482BF074
:10E8F80066FC3846FFF7BAFE384601F037F9DFF80C
:10E90800B892CDF80880002F40D0D9F80030B3F580
:10E91800007F40F0D780002520262C464FF00209C2
:10E928004FF4401B2BF07BFC4FF4C87303FB09F337
:10E93800049303F59C53083303900093002C40F094
:10E948007681A2464FF0010901F062FE01F030FC29
:10E9580005460190002800F0BD8046F0100601F041
:10E96800DBFB964C206828B103781E4002D112F0D8
:10E97800E1FD2660BAF1000F04D0002001F028FB69
:10E9880001F020FB284609B0BDE8F08F01F04CFAF1
:10E9980001F02CFC0546002840F08680874EFFF7E2
:10E9A80081FE2BF018FC3368002B5CD01A7822F01B
:10E9B80020021A7033689A681C78127892B15868E5
:10E9C80008B103F0EFFE336801219B6807A807939D
:10E9D800FFF716FE98B9336898682BF0F0FB784873
:10E9E80001F044FF04217748FFF70AFE38B90821EF
:10E9F8007548FFF705FE10B1744801F037FFD9F8E4
:10EA080000301B0531D501F00DF801282DD17048D3
:10EA18004FF0000A01F02AFF6E4BD9F8040083F882
:10EA280000A0FFF76FFD3268C9F804A02AB1137877
:10EA3800980644BF43F020031370D9F80030190535
:10EA480015D500F0EFFF441E18BF01243026D9F871
:10EA58000030DA051BD5B3F5007F4FF001043FF411
:10EA68005DAFA1462BE03C46BCE75B48D0E71BB94D
:10EA7800242604F00104EAE714F0020418BF83F422
:10EA880080634FF0280618BFC3F38024DFE7B3F58F
:10EA9800007F254615BF4FF001094FF002094FF4DA
:10EAA800405B4FF4401B3DE7D9F80030B3F5007FD9
:10EAB8003FF431AF3D463C4620264FF001094FF464
:10EAC800405B2FE7002520262C464FF00309DFF88E
:10EAD8000CB127E72BF04CFB059080B12BF067FBBE
:10EAE80068B101F083FB054648B92BF04EFB0428BA
:10EAF8007FF437AF032000F09BFF059D31E7CCB9C9
:10EB08002BF036FB0546A8B101F070FB90B9B8F1BF
:10EB1800000F02D13846FFF7A9FD029B13B938460A
:10EB280001F024F82C4623482BF049FB2C4801F02F
:10EB38009DFE02952BF01CFB0546002814BF454698
:10EB48002C46B9F1000F05D001F050FB10B902F0C6
:10EB580035FF81462BF063FB039B049AC31A9A4244
:10EB680080463FD94FF4C871B3FBF1F201FB12386C
:10EB7800B8F1630F11D9BAF1000F04D0002001F0E9
:10EB880027FA01F01FFAC8F5C870B9F1000F47D18C
:10EB980012F0DEFB12F026FC2CE0BAF1000F04D1D3
:10EBA80001F030FA584601F013FA0123C8F1640065
:10EBB8000193EAE7AF7405088C360020DC370020A3
:10EBC800A5C6050818B90408F8B8040892BD0508D0
:10EBD80006BD0508143E00201FBD050800303000A2
:10EBE800F2BF0508009A9A4208D22BF018FBCDF81C
:10EBF80004A00390A846DDF804A0A5E6BAF1000F2A
:10EC080004D0002001F0E4F901F0DCF9009B039A3C
:10EC18001344A3EB0800B9F1000F05D00028E9D090
:10EC2800484528BF4846B3E70028E3D0B0E74FF08F
:10EC3800000A96E607B5114A114B1068596820B1C9
:10EC480003B05DF804EB2BF0BABA1A6892050ED53A
:10EC58009A68002A0BDD51B109680C33C988094844
:10EC6800009109492FF073FA03B05DF804FB0748D7
:10EC780003B05DF804EB01F0F9BD00BFBC3600201D
:10EC88008C36002028E004089373050827C305087C
:10EC98002DE9F74312F010FB00F0D6FE2AF0B4FF7E
:10ECA80012F0C2FB2BF0A6F801F048FC53482AF0FA
:10ECB800D3FF00F0C3FE18B900F0CCFE00F0C4FE8C
:10ECC8002BF09DF801F070F900F0B8FEB0FA80F072
:10ECD8000021400900F0DCFF10B9082000F0B4FE64
:10ECE80031F0D0FC2BF08AF82BF087F802F050FABC
:10ECF80042482AF0B1FF002000F09AFE00F09EFE84
:10ED080008B901F00FFA0125012001F0A1F801204E
:10ED180001F098F800F092FEFFF72EFD2AF0FAFFB6
:10ED2800012001F0BBF84FF480742846344E354F6B
:10ED3800DFF8D48014F4106957D015B9384601F0BB
:10ED480095FD3578002D3ED100F078FEFFF7C6FD21
:10ED58000028EFD100F072FE044601F065F8204665
:10ED6800FFF7A0FC2BF037FA012001F0EDF900F0D5
:10ED780065FE28B9254B012101A80193FFF740FC46
:10ED880001F040F9404601F023F901F01BF933780E
:10ED9800012B1AD101F0F8F800F0C0FC044601F08C
:10EDA800F9F80420FFF7AEFB01F02CF9002001F080
:10EDB8000FF901F007F9012001F0CEF9032000F066
:10EDC80037FE0020B6E70025C4E7114BDFF8449072
:10EDD800C9F8003001F06EF800F030FD0023044659
:10EDE800C9F8003001F066F8DBE7002CB0D02DF050
:10EDF80052FC484603B0BDE8F08300BF34740508F0
:10EE0800153E00204FB50508303030009C730508CA
:10EE1800A4730508BC36002008B511F091FB00F07A
:10EE280037FB0421064831F0ACFB2BF046FA01F021
:10EE380055FC02F0EFF8BDE8084011F095BB00BFA3
:10EE4800EC380020014B1878704700BF143E0020B2
:10EE5800004870470048E801004870473333534082
:10EE680038B505462021FAF759FB041E11DA214668
:10EE7800094826F0B0F9002421462022074826F048
:10EE8800AAF9C4F1200228190021BDE838403BF056
:10EE980089BD1F2CF0DD38BD3D7405085774050881
:10EEA8000428034607B506D801460F4803B05DF8A5
:10EEB80004EB01F06DBC062168460C4A23F000FC07
:10EEC800011E0DDD052901DD26F0FBFE442201F1BE
:10EED80008036B446846013103F8082C01F058FC1C
:10EEE80003B05DF804FB00BF7E7405088374050851
:10EEF800F8B5244DAB7DDB0732D52E687068012844
:10EF08002ED9B168431ECA5C0A2A29D14A1E002B91
:10EF180001DC1A4608E0D45C0A2CFAD0013BF6E77B
:10EF28008C5C202C02D101329042F9D8002B0CDDE8
:10EF3800541CA04209D15C1E0C44A14205D014F80F
:10EF4800017D0A2F0CD0202FF7D00144D21A11F8D6
:10EF5800023C94083A2B0C4F08BF0134013C00D204
:10EF6800F8BD04223946304631F0C4F90421384648
:10EF780001F00EFC2B6904332B61AB7D43F00203D7
:10EF8800AB75EBE7C836002019C905082022002117
:10EF980001483BF007BD00BFB4380020002238B557
:10EFA8000B4C0546A26062754FF0FF326B6808464D
:10EFB800C4E9032363602560A1612AF04DFE6B68F4
:10EFC8000BB90123A375BDE83840FFF791BF00BF17
:10EFD800C8360020F8B503780446DBB10E4FD7F8E1
:10EFE800B80018B12146F2F74BF998B12046F2F76C
:10EFF80059F9461C30462CF043FD054650B13246BF
:10F0080021463BF0A8FC05491C22081D3BF0B0FC3A
:10F01800C7F8B850F8BD00BFFC370020B43800204E
:10F028002DE9F347AC4C06462368D3E901102DF0CF
:10F0380074F8A5680746002D40F03A81731E042B2A
:10F048001AD8D4E900325B689A4279D0012E15D1DA
:10F05800236865689868D4F8108000EB0801284494
:10F06800A8EB050800252AF0DAFDA8450646A560A4
:10F0780040F3BC80A946AAE00D2E13DC022E40F313
:10F08800B580F31E0A2B00F29180DFE813F05900D7
:10F098008F00CF018F008F0060008F008F008F00DE
:10F0A8003E004E001B2E4FD07F2E50D0A37D9907D7
:10F0B80000F181801F2E40F39980206821698368C0
:10F0C8005A5C06F0C003802B0CBF237DF2B202F11C
:10F0D800400508BF0133EDB214BF0023DBB2372D62
:10F0E80097BFE5250025D20802F0060298BF154112
:10F0F80019443246237598BF05F0030531F0E4F949
:10F10800237DAB4272D1013597E074482AF0A4FD03
:10F11800A0692AF0A1FD2268636821699068C91A6C
:10F12800184401F035FB002587E06D482AF094FD6E
:10F13800206831F058F9636800261844FFF74AFF41
:10F14800304602B0BDE8F0870123A3604EE0226993
:10F1580061688A424AD900232068561AD0F808E024
:10F16800B34203EB010C18D1032BCCBF04260126B4
:10F17800961B33461EF803C019460CF0C00CBCF1B0
:10F18800800F03F1FF33F5D0A2EB01084246761A4F
:10F1980031F0A7F94FF0010919E01EF80CC0BCF1D5
:10F1A800200F01D10133DBE70126E1E7A37D9A07B0
:10F1B80023D5092E18D0202E7FF47CAF00260321FA
:10F1C8002068A675B14631F085F94FF00308A8EB21
:10F1D8000600FFF765FE2369A3EB08032361B9F175
:10F1E800000F00F0298128E00023A375A37D4FF0CC
:10F1F800FF3623F00203A375A2E7092E7FF45AAF66
:10F2080022682169D2E90123002A40D00B4413F86F
:10F21800010C04F0E9FA002839D00425314B019398
:10F228000026019B21695A1C019231441A782068F2
:10F23800013631F043F9B542F3D12368D3E901101F
:10F248002CF06BFFB84203D20321274801F0A0FA43
:10F2580023682769D3F80880D3F80490781908EB55
:10F26800090140442AF0DBFC0646A9EB070108EB3C
:10F27800070001F08DFA236822695B689B1A5B1B03
:10F28800981BFFF70DFE23692B442361AEE7236823
:10F2980060689D682169154A091A01AB284410F075
:10F2A800C9FC05460028A1D0431C3FF431AFB7E79D
:10F2B800013D032D00F2E880DFE815F004001A0094
:10F2C800A000E1004F2E04D05B2E40F0DD80022329
:10F2D8003BE7042339E700BFC836002088740508D7
:10F2E800AF74050819C905089174050828E00408D1
:10F2F800A6F13003092B03D803236675A36075E7CD
:10F308000023412EA3602ED1E368062B3FF76EAF92
:10F318005E4D03F1010A2D3305EB8305AB68002B25
:10F328003FF464AFD4F80080D4F80490D8F808000B
:10F338002169014448442AF072FC06464046C8F850
:10F348000490A968C4F80CA031F0ABF8636822698E
:10F35800A2EB03082268B8F1000F5568A5EB030576
:10F368007FF76BAF16E7423E062E3FF63FAF01A38D
:10F3780053F826F099F30008DFF30008EFF30008CC
:10F38800F5F1000835F40008F5F1000859F0000817
:10F39800E568002DFFF62AAFD4F80080D4F8049071
:10F3A800D8F808002169013D014448442AF037FC97
:10F3B800D8F804100646A1EB09014046E56031F093
:10F3C80089F8E268002AC1DB304B206803EB82032E
:10F3D800D3F8B810B8E7236822695B689A42BFF48B
:10F3E80005AF01252BE0226963689A427FF6FEAEDD
:10F3F80000254FF00108A9462E46E8E67E2E43D1A7
:10F40800637D312B3FF424AE333B052B3CD801A25E
:10F4180052F823F057F4000835F4000891F4000876
:10F4280091F4000859F0000835F4000823685D6875
:10F438002369ED1A0023A360002D7FF7D7AE236858
:10F44800294698682369184401F0A2F91BE7206847
:10F4580021694368994217D2012285685B1A0D44D5
:10F4680015F8016F06F0C006802E01D19A4204D12A
:10F4780031F037F80023A36055E60132F0E7462E55
:10F48800D4D0482E3FF4E4AD00235EE6FC370020DC
:10F498002DE9F04F8BB068460A4BCDE90045196855
:10F4A800CDE90267091A8908CDE90489CDE906ABD7
:10F4B800CDF820C0CDF824D031F063F80BB0BDE80A
:10F4C800F08F00BFFC37002070B5067804461EB1E7
:10F4D8004FF0FF35284670BD2AF0F0FEC31E012B01
:10F4E80005460CD801210C48217001F051F9032D73
:10F4F800EED10A48836E60309E6010F02FFAA38820
:10F50800013B9BB2A380002BE4D10121044801F008
:10F518003FF96388A380DDE795740508FC37002070
:10F52800B37405082DE9F0431D46002391B0044645
:10F5380003A817460493884610F0FCF907F0010663
:10F54800034600285BD1F90641D5D4E90121DC2026
:10F558002EF035FC0446B8F1010FD4F8009007D11D
:10F568004FEA091140F28D2041F0060105F062FDD5
:10F578002146424601A80DF085FD4946C7F38002A1
:10F5880001A808F07DFFB8F1010F044601D1FFF78B
:10F5980043FC380602D4032000F0FCF914B12046DD
:10F5A8002DF0B1F84FF0FF3000F0F4F9012004F02D
:10F5B800B7F809F0FFFEEEB9CDB900241EB101215C
:10F5C800474801F0E5F8204611B0BDE8F0837A0617
:10F5D80005D594E80E00DC202EF0A9FBBAE7BB069F
:10F5E800B9D520462CF0F7F92EF0F7FBB2E7002347
:10F5F8002B60E2E701213A4801F0CAF8DCE74FF056
:10F60800FF3000F0C7F9022004F08AF8790602D525
:10F61800A368206898471EB10121314801F0B8F865
:10F62800049C20460AF0A8FA2E4905F035FA00286D
:10F6380041D004982EF027FE0E283AD0C20705D4F0
:10F6480083072BD10268284B9A4227D12CF05FFE02
:10F6580040F48074002DB1D04FF0FF33049F2C602C
:10F6680038466F60AB602EF0F9FD0028A6D06946D9
:10F67800384601AA2EF021FE019B002B9ED05A6825
:10F68800AA60002285F82C2018682CF0C4F92022E2
:10F69800014605F10C003BF0BCF98FE7014600225A
:10F6A80012480AF085FA124910482EF0CCFC0120C5
:10F6B800CEE70020CCE70F4B9C420DD004990B48B5
:10F6C8002EF0E9FB049B0C49186805F0E5F908B130
:10F6D8008224BFE70124BDE74FF40064BAE700BF06
:10F6E80095740508F8E4040804DF040828E0040811
:10F6F80014B1050874380020D4E4040808B5037868
:10F708004BB901210170044801F042F82AF0D6FDF6
:10F7180003380128FAD808BD957405082DE9F04387
:10F728008BB0202106A830F00EFE0026DFF8E88016
:10F738003A4F40462AF090FA384607962AF08CFA53
:10F748002AF0BCFD0128044635D107990229F0D1D9
:10F75800089B1A78052AECD193F80190B9F1410F6A
:10F7680006D02F4801F014F800232C480793E5E74A
:10F7780080252C4801F00CF803216846ADF80050AC
:10F788008DF8024001F004F8002301AA0392264AEA
:10F7980021460492254A03A805924A468DF804306A
:10F7A800ADF80650ADF80850FFF7BCFEC305DBD531
:10F7B8000BB0BDE8F083022809D11D482AF04CFAA5
:10F7C80006A830F0E2FD00201A4B1870F0E7032875
:10F7D80002D100230793B3E7042804D0C1B206A8D6
:10F7E80030F010FEACE714482AF036FA079B43B90C
:10F7F8000F482AF031FA06A830F0C7FD4FF48070A0
:10F80800D6E700231122012106A8FFF78BFE10F48A
:10F81800106F91D0CCE700BF977405080EAF0508AC
:10F82800E8B10408B2740508D1F4000805F7000827
:10F83800AF740508153E0020B57405082DE9F041A0
:10F8480092B0202101A830F07EFD494EDFF82481D6
:10F8580030462AF001FA48482AF0FEF930462AF0E4
:10F86800FBF9464FBA8A002302B1BB8205A802936E
:10F87800069310F05FF8044690B9414901A82AF0B0
:10F88800DCF9012805462CD139482AF0E5F901A808
:10F8980030F07BFD20463B4B1D7012B0BDE8F08177
:10F8A800022003F03DFF30462AF0D6F90699364883
:10F8B8002EF0F1FA029B002BD4D001A830F093FD72
:10F8C80010F0F4F858B10A2101A830F09BFD414628
:10F8D80001A82AF0B2F903280BD00428EDD10021A1
:10F8E8002CE0022803D122482AF0B6F9B0E7032811
:10F8F80001D1304619E0042808D11D482AF0ACF996
:10F9080001A830F042FD4FF48070C6E70528D1D138
:10F918001E482AF0A1F902941D4C2AF0CFFCC1B26E
:10F9280003298DF8031003D111482AF095F999E7B6
:10F9380004290CD10E482AF08FF901210023162240
:10F9480001A8FFF7EFFD10F4106F8BD0A5E701A811
:10F9580030F058FD9DF803300D2B03D120462AF0D6
:10F968007BF9DAE701210DF1030000F011FFD4E77C
:10F97800AF740508F47405081C730508FC370020EB
:10F98800B8740508153E002028E00408BD74050871
:10F99800ED740508014B1860704700BFDC060020B5
:10F9A800024B986A003818BF01207047FC370020C6
:10F9B8002DE9F04106460D4600270DB9BDE8F08156
:10F9C80033780A2B16D1AFB90121104800F0E0FEB8
:10F9D800012406EB040843461FB998F800200A2AB8
:10F9E80001D0A54208D13046214600F0D1FE464656
:10F9F8002D1BE2E70024ECE71F7808F10108A7F1C6
:10FA08000D035F425F410134E5E700BFF974050863
:10FA1800024B034819782EF079B800BF163E002033
:10FA2800A0C20408014B1878704700BF163E00209A
:10FA3800014B1870704700BF163E0020014B187824
:10FA4800704700BF173E0020014B1870704700BF79
:10FA5800173E00202DE9F04130F017FE294B0446EF
:10FA680020F47F0020F47F409842274E0AD114F4F6
:10FA78007F4FC4F3072505D030F006FE35702846C1
:10FA8800BDE8F081002333702AF0C7F828B10628B2
:10FA980033D85423C340DB072FD51C4830F0F4FD7E
:10FAA80000F0B0FA2AF0ACFB064600200F460146EB
:10FAB800DFF85C80FA220023F1F788FB7D2A73F1D6
:10FAC800000334BF4046002000F082FA2AF0F3FB1E
:10FAD800054648B92AF094FB801B61EB0701B0F595
:10FAE8007A7F71F10003E5D3002000F071FA00F08D
:10FAF80069FA25B9204630F0C7FD0025BFE7112572
:10FB0800BDE700BFAF0000AD173E0020AF1100AD4C
:10FB180000303000024B43EA002030F0B5BD00BF92
:10FB2800AF0000AD0D4D08B52B780446012B0FD959
:10FB380001280DD90A4825F04EFB2146094825F031
:10FB48004AFB2978084825F046FB26F08BF8FCE7A5
:10FB58002046FFF7DFFF30F091FD00BF173E002081
:10FB6800FB740508117505081D75050810B50446D0
:10FB7800002838D01C4800F079FE631E112B12D8DB
:10FB8800DFE803F02D1111111111112B1129111199
:10FB980027212523091F154800F068FEBDE81040FD
:10FBA800134800F063BE023C1248E4B200F05EFE67
:10FBB8000A2C16D8104B53F8240000F057FE0F48B3
:10FBC800EAE70F48E8E70F48E6E70F48E4E70F4899
:10FBD800E2E70F48E0E70F48DEE70F48DCE70F48A9
:10FBE800DAE70F48E9E710BDB1BC050839BD0508DB
:10FBF800C5BC05089DC3050898BA0408D6BC050805
:10FC0800F9C1050859C4050831BE050847BE0508ED
:10FC180032BF050815BF0508FCC3050813C0050851
:10FC2800EEBD050800B597B002460A2369460448A8
:10FC380031F0C1FC684631F0FEFF17B05DF804FBF7
:10FC48000012002010B5064C23783BB14FF47A72AD
:10FC5800044B1A6000F01CFA0023237010BD00BF8B
:10FC6800183E0020E0060020074B1A685AB11A68AF
:10FC7800012A09BF05491A680A704FF47A7218BF39
:10FC880002F1FF321A607047E0060020183E00209B
:10FC98002DE9F0414FF00008514EADF5287D07469B
:10FCA800504C30460D46A6F8048000F0FFF906F1E6
:10FCB8008000C4F8048031F07AFC0D2806D147B9D9
:10FCC8003DB900200DF5287DBDE8F081002D00F03C
:10FCD80084804FF40073002200930721424828AB28
:10FCE80012F05CFD0028ECD100F0D2F93F493E4803
:10FCF80012F06EFC0028E4D13D493B4832F04AFB43
:10FD08000028DED13B48FFF78DFF3B48FFF78AFF0D
:10FD18003A48FFF787FF3A48FFF784FF39493248E6
:10FD280032F038FB384B03AA03F138071546186838
:10FD38005968083303C5BB422A46F7D11B88334AA2
:10FD48002B80392312A9029327480A2331F033FC68
:10FD5800029A02AB03A912A831F004FE12A831F0EE
:10FD68006AFF2B48FFF75EFF2A4B03AA03F110072F
:10FD7800154618685968083303C5BB422A46F7D1A7
:10FD8800186899889B792860AB711623A980224A44
:10FD9800029312A90A23144831F00DFC02AB03A9FF
:10FDA8001A6812A831F0DEFD12A831F044FF1B4991
:10FDB8000D4832F0EFFA002883D100F069F9184BAA
:10FDC800012523600023E360164BC4E90156C3E90B
:10FDD8003B442BF018F9284674E70028EFD070E769
:10FDE80080110020E436002000120020CB80050896
:10FDF8003475050840750508537505086A750508C2
:10FE08007475050881750508B675050885750508B2
:10FE180099750508F0750508A8750508B1750508F0
:10FE280087550508FC3700204FF47A7208B5044B53
:10FE38001A6000F02DF9BDE8084011F0EFB800BFD6
:10FE4800E00600200146014829F06BBF8011002020
:10FE58000146014829F081BF80110020024B5868F3
:10FE6800003818BF01207047E4360020034B0448CF
:10FE78005B68002B08BF0020704700BFE4360020F5
:10FE880080110020034B1B7813B903482AF097B957
:10FE9800704700BF193E00200776050810B10122FF
:10FEA800024B1A70024800F08FBB00BF1A3E0020B8
:10FEB800F4360020F8B5254B1D7825B1BDE8F8408B
:10FEC8000120FFF7EBBF224B22481D702BF0E1F910
:10FED80020482BF0C4F958B91E482BF0D2F980F00D
:10FEE8000104012000F060FB01270546E4B20AE0A6
:10FEF8002AF03EF90028EFD016482BF0C2F92F4619
:10FF080080F00104E4B2F4B1012000F055FB06468C
:10FF180011482AF054F911482AF051F9FEF78AFEDF
:10FF28000F482AF04CF90F482AF049F90E482AF0F0
:10FF380046F917B1284600F037FB34B13046BDE822
:10FF4800F84000F039BB2646E2E7F8BD193E00202C
:10FF58001A3E0020A00700200E7605081376050833
:10FF6800187605081C7605080B760508044B1B78DF
:10FF780023B9044B1B780BB1FFF79CBF704700BF38
:10FF8800193E00201A3E00200122014B1A707047CA
:10FF9800193E00200022024B02481A7000F014BBE0
:10FFA800193E0020F4360020034B044A04481A6026
:10FFB80000225A602BF067B9F436002075FF00085C
:10FFC800A007002001482AF0C3B900BF0837002065
:10FFD80038B5094D04462B6883420CD0074B197875
:10FFE80029F0F1FEB0FA80F12C6005484909BDE816
:08FFF800384000F0D3BE38BD13
:020000040801F1
:10000000043700206B0B00200837002038B50B4D5B
:100010002C7894B901230A490A482B7000F0A6FEF7
:100020002246214607482AF0BFF94FF08072064B5E
:1000300018681A60FFF7D0FF2C7038BD1B3E0020F7
:10004000A40505080837002004370020014B18706C
:10005000704700BF6B0B0020014B1878704700BF42
:100060006B0B0020F8B50E461C4615466AB1094FC9
:100070003B781BB900F06AFB01233B7022463046F7
:10008000691EBDE8F84011F057B8012B94BF00205D
:100090000120F8BD1C3E002010B5054C10F0AAFF51
:1000A00023780BB100F064FB0023237010BD00BF68
:1000B0001C3E002010B50F4B04460360838843F0BC
:1000C0000503838030F0D2FA01230E220A4984F816
:1000D0008430231DC4E90823C4E90D232361616131
:1000E000064B0749A060C4F88040E260A162E36368
:1000F00010BD00BFC0F404080D9E03086B9F0308E9
:100100006500010808B5FFF797FC044B03F178027E
:100110009A62BDE8084011F0E9B800BFFC37002042
:100120000022014B1A607047143700200122034B54
:100130001A700022024B1A60704700BF1D3E00205B
:10014000143700200022014B1A7070471D3E00201A
:10015000024A136803431360704700BF183700203A
:10016000024A136823EA000313607047183700201F
:10017000014B1878704700BF1D3E002038B50B4B6F
:100180001B7893B10A4B1B687BB90A4C25682AF08F
:100190004AF82060236813B923680133236025B926
:1001A000BDE838400120FFF7ADBF38BD1D3E00203F
:1001B000183700201437002010B50C4C206890B17F
:1001C0000B4B1B6883B92AF02EF8236883422368FF
:1001D000A0EB030040F2EE2388BF00F1FF3098420D
:1001E00094BF0020012010BD0020FCE71437002040
:1001F00018370020024B1868003818BF01207047DC
:1002000014370020012910B502460C4617D90429DD
:1002100015D00B490B482DF0C3FF022C03D0052C41
:100220000BD0094900E0094906482DF0B9FFBDE8A7
:100230001040074903482DF08EBF0649F4E710BD72
:10024000C7C4050828E004080AC20508BAC10508A1
:1002500014B10508C5C105082DE9F04F9DB000AFE8
:1002600080460C469246FFF705FE28B90125284630
:100270007437BD46BDE8F08F01239F4A07F118018E
:10028000803031F09CF90028F0D1D7E91402D7E989
:100290000A139A4208BF884200F02B8197F8493030
:1002A000002B40F0268107F1180029F08DFE5B2815
:1002B000064606D1D7E90A2307F1180031F094FD6C
:1002C000E3E7002EF6D008F1FF3919F8015F2DBBE6
:1002D000304603F08DFA20B107F1180029F074FEC2
:1002E00006463D2E1CD107F1180029F06DFE22288C
:1002F0000CBF012300238AF8003040F0CA8007F1C8
:10030000180029F052FE22282AD016D830B30A2825
:1003100024D0C1B2204629F06FFEF0E7B54206D0E6
:100320000A2EB2D007F1180029F05DFEADE707F103
:10033000180029F03AFE0646C7E75C28E9D107F124
:10034000180029F032FE7628E3D861281DD80A2843
:1003500004D0552800F089800028DAD1052509E06D
:1003600007F1180029F030FE0A2803D0232807D00F
:100370000028F3D1EDB207F1180031F060FC76E708
:1003800007F1180029F02FFEF4E7A0F16203142B07
:10039000BFD801A252F823F08F040108130301080B
:1003A0001303010813030108FD03010813030108E7
:1003B00013030108130301081303010813030108C1
:1003C0001303010813030108F103010813030108D3
:1003D0001303010813030108ED03010813030108C7
:1003E000F503010801040108F90301080D2090E755
:1003F0000A208EE709208CE70B208AE70C2088E78B
:100400003B1D6E469B464FF00409D84609EB0B0A8C
:1004100007F1180029F0C9FD08F8010BD045F7D104
:10042000002339460BF809301022584622F0ECF927
:100430003B680146434528D1B0F5881F22D27F286A
:100440001AD9B0F5006F19D3B0F5803F34BF03233C
:100450000423227B22B16268134422689A420FD996
:1004600020462FF0DAFFB54649E707F10C036E4648
:100470009B464FF00809C8E70123EAE70223E8E7B3
:100480006360F0E70225B54674E7B54666E70820E5
:100490003FE70A283FF462AF00283FF45FAF002532
:1004A0000D281CD009DC092819D00A2800D040B931
:1004B00063685B1B636000255CE720280FD023285E
:1004C00005D0C1B2204629F097FD00250CE06368F5
:1004D00007F118005B1B636029F085FDEBE7C1B2F3
:1004E000204629F089FD013507F1180029F05DFD4E
:1004F000D6E704253FE700BF9975050870B586B0BB
:100500000E4610220DF1070302A929F080FD0446D2
:1005100048B99DF807507DB9084902A8F0F7B4FE24
:1005200020B901253570204606B070BD044902A8E7
:10053000F0F7AAFE0028F5D00524F4E72376050895
:100540002876050810B5054C23782BB929F004FE50
:1005500030F0C4F80123237010BD00BF1E3E002000
:1005600073B505460C46C1B10E4B1B78C3B90A469C
:1005700001AB01460C482AF0A3FF06460B4B1B7843
:1005800053B902F0D7FA40B12146284629F0ECFDD4
:100590002146284611F08AF83446204602B070BD44
:1005A0000E46EBE71F3E0020E8070020203E00201B
:1005B000024B1A7818701046704700BF203E00208A
:1005C000024B1A7818701046704700BF1F3E00207B
:1005D00010B5044601F03EFFE3681BB90C4A1168F0
:1005E000A14203D1BDE8104001F04EBFA360094B0A
:1005F0001968E160196809B119688C60116801B95E
:1006000014601C6001F040FF10F070FE10BD00BFD0
:1006100024370020203700202DE9F041144E32F01D
:100620001CFD33680BB3134D01F014FF2C681CB193
:10063000BDE8F04101F028BF01230F4A2B60336869
:10064000346014601BB92B68013B2B60F0E79F6896
:10065000C3E90244D3E9006801F016FF0EB1404639
:10066000B04701F0F7FE3B46ECE7BDE8F08100BF84
:10067000243700201C370020203700202DE9F743C5
:100680000025A846144E019501F0E4FE346801AF40
:1006900054B9019B3360114B1D60114B1C6003B0BA
:1006A000BDE8F04301F0F0BED4F808902046C4F84D
:1006B00008800FF039FF18B10023E3604C46E7E7EC
:1006C00060680FF031FF0028F6D12B463C602546CC
:1006D00004F10807F1E700BF24370020203700208D
:1006E0001C37002010B5044B1C6804B910BD6068AD
:1006F0002FF07FFFA468F8E72437002008B532F018
:10070000A9FC29F082FB00F087FBFFF79FFA32F08B
:10071000A3FC29F07AFB00202FF0BDFF034BC3E9B7
:100720000001BDE8084032F096BC00BF80230020E5
:1007300008B5FFF79DFABDE80840002201490248CC
:1007400029F04EBDFD0601082C37002010B5074CDE
:1007500001F080FE23680BB910F0EAFD2368013335
:100760002360BDE8104001F08FBE00BF2837002095
:1007700008B501F06FFE074B1A6812B11A68013A0A
:100780001A601B680BB910F0E1FDBDE8084001F0EC
:100790007BBE00BF283700202DE9F843DFF87C80BE
:1007A00000AF05460E4629F02BFBD8F8003043B3C6
:1007B0001B4829F0A0FDC0F500720446D8F80000DF
:1007C00043689919914223D90734D21A294624F053
:1007D00007042FF093FDE946ADEB040D6946104880
:1007E000D8F8004000F050F8014620462FF05DFE9A
:1007F0000A21D8F800002FF009FE0023C8F80030C5
:10080000CD4631462846FFF7ABFEBD46BDE8F8832E
:10081000324629462FF072FDF3E700BF88360020EC
:100820002CBD0508A1F18003532B70B5064618D8DE
:10083000194602230D480E4C10F8012B914205DA9F
:1008400003FB0144E518A54205D870BD03FB024433
:10085000891A0133F0E7304614F8011BFFF7E2FF75
:10086000F1E7BDE870402FF0D8BD00BF3176050834
:100870003B7605080246024902482DF06CBC00BFD9
:100880002E76050850E604082DE9FF410546802430
:100890000A4615F8011B684601312FF073FD009ED2
:1008A000254FDFF89880013E019B9E4205D868469F
:1008B0002FF09DFD04B0BDE8F081002318461946D5
:1008C0001A4695F800C0520014EA0C0F14BF4FF0FE
:1008D000010C4FF0000C64084CEA020204BF8024B3
:1008E000013501318242C9B205D317F801C00CEBC2
:1008F00040006344E5E71B1A4244D15C012917D14B
:100900000B2300202A784000144214BF0122002249
:10091000640804BF80240135013B40EA0200F1D1A4
:1009200001302BF07CF8014668462FF0BEFDBBE796
:100930006846FFF777FFB7E777780508CD770508B2
:1009400008B5024824F04BFC002008BD8478050857
:1009500038B5FFF78FFA044620B90D4824F03FFC64
:10096000022038BD29F0F4F920B90A4824F037FCF8
:100970000420F6E7084D2B782BB9204629F01EFA03
:1009800008B90648F2E7012300202B70E9E700BF11
:1009900097780508A9780508223E0020BC7805084C
:1009A000F8B514460E461F46FFF764FA05460420C4
:1009B000FFF7CEFB3B4622463146284631F073FF17
:1009C000D5F8CC30A34207D134B14FF40072314690
:1009D00005F5807039F0C3FFD5F8BC300020A34284
:1009E0009EBF0122014B1A70F8BD00BF213E0020BE
:1009F00038B50C461546FFF73DFA022C03D0052CFE
:100A000007D0012C15D12A46214612F0A9FC00205E
:100A100038BD2A4600210A4C12F0A2FC0420FFF740
:100A20009FFB2378002BF2D0FFF7A8FB0023237055
:100A3000EDE70448214624F0D2FB6FF08500E7E79C
:100A4000213E0020CC78050808B5F3F759FE30B1F7
:100A5000BDE808400121024A024824F086BF08BDD3
:100A6000E9780508A0B0040838B504460D4625F01D
:100A700009FA90B12B7843B92046F3F7FBFD20B17A
:100A80000121064A064824F070FF2B78012B04D17F
:100A90002046BDE83840FFF7D7BF38BD0A790508C2
:100AA000A0B0040837B5844824F099FB834824F0AB
:100AB00096FB8349834825F045FA034638B1824ABC
:100AC0000121824803B0BDE8304024F057BF80497F
:100AD0007C4825F037FA034608B17E4AF0E77E49A4
:100AE000784825F02FFA034608B17C4AE8E702F07F
:100AF00021F898B90E2002F06FF802F021F8D8B969
:100B00000E2002F077F87648F2F71EFD014608B392
:100B1000744803B0BDE8304024F061BB012180205F
:100B200010F0ECFC03460028E4D080226E496F48A8
:100B300002F022F86D48DEE70121802010F0DEFC93
:100B400003460028DCD0802269496A4802F014F884
:100B50006848D6E75B4825F055F90128044640D19E
:100B6000654824F03CFB2146644A5648F4F792FF5E
:100B700038B1634A0121554803B0BDE8304024F044
:100B8000F4BE604824F02BFB01F0D4FF48B15E496D
:100B9000234622464B48F5F7ADF8014608B15B48BD
:100BA000B7E701F0CDFF40B1012359491A46454846
:100BB000F5F7A0F801460028F1D1012355491A465E
:100BC0004048F5F797F8014608B15348A1E7534864
:100BD00024F005FB01210223EF223A48009125F081
:100BE00018F94F4824F0FBFA00214E4A3548F4F733
:100BF00051FF044608B14C4ABCE701F09BFF78B1B5
:100C00004A4824F0ECFA012322463F492D48F5F7E3
:100C100071F828B1464803B0BDE8304024F0DFBA8F
:100C200001F08EFF50B1414824F0D9FA012300228F
:100C300037492448F5F75EF80028EBD1012300225C
:100C400034492048F5F756F8044608B10146BCE798
:100C500001250223EF22014600951A4825F0D9F814
:100C6000344824F0BCFA2146164825F0F6F83248FC
:100C700024F0B5FA3149134825F0E2FB08B1304AB7
:100C800078E7304824F0ABFA0E48F3F7B5FC08B12A
:100C90002D4A6FE72D4824F0A2FA0A4825F0F2F811
:100CA00038B90848F3F7E6FC08B1294A62E7294851
:100CB000B1E703B030BD00BF2A7905083C790508CB
:100CC000840700203810002058790508A0B00408D7
:100CD0006C0700208679050854070020B8790508BC
:100CE000E4060020E579050828AE0408D823002092
:100CF0000CAE040888230020087A0508FC060020B2
:100D0000297A0508507A0508B7630508767A050838
:100D1000976305084F640508997A0508BE7A0508A7
:100D2000E37A050810070020047B05082B7B0508E3
:100D3000517B0508717B0508877B0508690A010856
:100D40009D7B0508C17B0508CC7B0508F07B050869
:100D50000A790508017C050808B501F0EBFE0028BA
:100D6000014808BF002008BDD823002038B50C4634
:100D70000546084628F050FF6C60606828F042FA8B
:100D800020B9074824F02BFA012038BD4FF48032F7
:100D9000217A606829F0CFFA0028F5D12872F4E7AB
:100DA000847C050838B50C4601214368054658681F
:100DB0001B7A994003691B6819420CBF234684F0D3
:100DC00001034BB18368DB689847014610B10448C2
:100DD00024F005FA6C7238BD83681B69F4E700BF24
:100DE0009B7C050838B543680129094A04460D462D
:100DF00018BF4FF40032197A586829F09CFA01465E
:100E000020B1044824F0EBF9012038BDA572FCE7BD
:100E100006000200B37C050808B5FEF7C5FD10B951
:100E2000FFF7CAF970B108BD0D4A934203D1BDE87E
:100E3000084029F0E7BE0B4A9342F4D1BDE80840D0
:100E400000F058BD08480368002BECD0074A9342D5
:100E5000E9D0074A9342E7D1BDE8084032F02CBC04
:100E600014BE0408ECBB04082824002060EC04082D
:100E7000701605084FF0FF3370B5204E204C3360DC
:100E800023682BB93368E3B9BDE8704013F0F2BDB5
:100E90001C4DAB42F6D01C4A934204D1204632F09E
:100EA00024FC2560EEE7194A934203D1204600F066
:100EB00051FDF6E7164A9342F3D1204601F0ACF813
:100EC000EFE7144C2368002BDED00E4DAB42DBD095
:100ED000114A934204D1204629F071FB2560D3E7E3
:100EE0000E4A934203D1204601F010FAF6E70C4A6D
:100EF0009342F3D1204601F019FDEFE79C07002053
:100F00002824002060EC040870160508ECBB0408D7
:100F100014BE04083C3700208CBD040890BF0408B0
:100F2000E0C10408F8B5334C334E23680BB1B3422B
:100F30000DD1266031480368002B59D0B34257D0F9
:100F40002F4A934246D1BDE8F84015F075B82D4AB6
:100F5000934216D16568A54203D304F198039D42DC
:100F6000E8D928460FF0E0FA0028E3D0264B6C229F
:100F70002946184639F0F3FC6060284632F033FC0D
:100F8000D8E7224A93421ED16568A54203D304F1F3
:100F900098039D42CED928460FF0C6FA0028C9D042
:100FA000194A2B46944605F1200E174618685968D1
:100FB000083303C773453A46F7D12846C4F804C03E
:100FC00032F052FDB6E7124A9342B3D120462AF0DE
:100FD000A0F8AFE70F4A934203D1BDE8F84000F014
:100FE000E5BC0D4A934203D1BDE8F84001F026B8B4
:100FF000F8BD00BF3C37002060EC04082824002026
:10100000701605088CBD04084437002090BF040802
:10101000E0C10408ECBB040814BE040808B5144879
:1010200003681BB9134803684BB908BD124A9342C1
:10103000F8D0124A9342F5D12AF0FEF8F2E70E4AB0
:101040009342F2D00E4A934203D1BDE8084032F0F9
:101050005BBB0C4A934203D1BDE8084029F0EBBDCD
:10106000094A9342E1D1BDE8084029F03EBA00BFE9
:101070003C3700202824002060EC0408E0C104086C
:101080007016050814BE0408ECBB040810B5084B24
:10109000084C1B68A34200D043B9074BB42200217F
:1010A000184639F083FC40F8044D10BD0020FCE7E1
:1010B0002824002060EC04082C24002008B5FFF749
:1010C000E5FF10B9014804F0DFF808BD7FBE050850
:1010D00010B5084B084C1B680BB1A34208D1074B55
:1010E00094220021184639F061FC40F8044D10BDEF
:1010F0000020FCE73C37002060EC0408403700206B
:1011000008B5FFF7E5FF10B9014804F0BDF808BDC8
:1011100085BE0508094B1B685A1C0DD0002B0BDC43
:10112000B8225343064A9818D358064A934203D02C
:10113000002B08BF0E2070470E2070479C07002030
:101140002824002060EC04080E2807B513D00E4AAE
:101150009042136803D10D4A934200D093B908F02E
:101160000FFDC388E82200934FF48A7140F25513B3
:10117000074804F0C5F84FF0FF33064A136003B088
:101180005DF804FB0023F8E72824002060EC040845
:101190002DC605089C070020074A1368013304D1B7
:1011A000064B07491B688B4200D17047002BFCD0CF
:1011B00000231360704700BF9C07002028240020F4
:1011C00060EC04082DE9F04F04461F464FF000087C
:1011D00085B0CDE9021200F15009B84502D305B03F
:1011E000BDE8F08F039B03EB080694F8B5307578E3
:1011F00096F901B0002B37D0B57806F1030A4846BE
:1012000017F07EF8A8B3012300930021334694F829
:10121000B620206DD4F860C0E04700955346012108
:1012200094F8B620206DD4F860C0E047484633F00B
:1012300054FCBBF1000F23DB00202AF0CEFA029B06
:101240003BB1D4F88430164A934202D0204629F0AC
:10125000DBF8FEF7A9FB0028C1D194F8B53045446E
:10126000DBB905F10208B8E706F1020A05F07F05CF
:10127000C5E7FEF799FB0028C5D1FFF7CDF9BEE71A
:101280006B1C94F8B520DDB256FA83F313445878FA
:10129000FF2808BF4FF4FA70CFE705F103089CE779
:1012A00060EC0408F0B54B6B05460C468BB0002B88
:1012B00000F0C980012380F84030486B32F04EFFC7
:1012C00085F83C00636B002B00F0C080A36B002B03
:1012D00000F0BC804FF48073A5F84030A06B32F072
:1012E0003DFF85F83D00B4F85630002B14BF0123B4
:1012F000002385F8B43094F8573018BF042185F8DE
:10130000423094F8563085F8433094F855600CBF5D
:1013100001230026626B0CBF194633460AB9A26B43
:1013200032B1228EB2F5807F02BF00260221334601
:1013300001220027CDE90422CDE90222CDE90013E4
:1013400005F10800638C228BE18A33F0DEFA94F811
:1013500059300897099394F8543005F15000CDE9BD
:101360000673638D0593238D0493E38C0393A38C01
:101370000293B4F920300193B4F91E300093628BCC
:10138000A38B216816F034FFA38D3249A5F8AA304B
:1013900094F82E3085F8B030238EA5F8AC3094F850
:1013A000323085F8B130606CEFF7A2FCEFF7A2FEA7
:1013B000A5F8A80094F84C3085F8B27085F8AF30E5
:1013C000206D2449EFF794FCEFF794FEC5F89000E8
:1013D00094F8543085F8B36085F8B63063681D49D9
:1013E000C5F894302389A5F8A030E068EFF780FCB9
:1013F000EFF780FEA5F8A6002369C5F89830A38A08
:10140000A5F8A230E36BC5F89C30B4F84030A5F8DD
:10141000A430114BC5F8843094F8583085F8B530B5
:10142000A36C4BB128460D4B40F8843FA16CFFF7ED
:101430009DFCA06C28F0EEFB284609490BB0BDE8E6
:10144000F04029F026B880F840303BE7002385F8CB
:10145000413048E700007A4460EC0408C81B0508E6
:10146000E809002010B50B680446C0F894304B68BA
:101470000549A0F8A0301046EFF73AFCEFF73AFE26
:10148000C4F8900010BD00BF00007A4410B5038F6F
:1014900004465A2B02D0B3F5877F19D15A2902D0BE
:1014A000B1F5877F19D104F1080033F0EDF90E4B47
:1014B0009C4205D113F0DEFAE18EA08E13F07CF988
:1014C000A06878B104F11801BDE8104032F0FBBC0F
:1014D0005A2902D0B1F5877FE5D1A38EE28EE3864B
:1014E000A286E0E710BD00BF282400202DE9F04FC0
:1014F00097B090F8B230044602AFE3B1D0F8842040
:10150000B14B9A4217D1843028F031FF94F8AF30B4
:10151000834204D100205437BD46BDE8F08FFFF769
:1015200027F900212046B4F8A230D4F8982084F896
:10153000B210FFF747FEA368002B00F0BF812046E2
:1015400028F0B0FF0028E5D104F1500A504633F0EE
:10155000B9FA0028DED094F84810002900F09A80EB
:101560000023236304F12803FB6294F8B430002BBA
:1015700040F0A180FEF718FA78610028CAD1204611
:1015800028F054FF04F1080B5846F96A07F13802B5
:10159000C7F810D033F057FA002800F0848107F123
:1015A000380033F081FC202594F83A30064607F1E4
:1015B0003800B5FBF3F533F07CFC814607F13800C9
:1015C00033F077FCB0EBC51F4FEAC51800F2CA80B4
:1015D00001233B6280231FFA89F09B004009BB6115
:1015E0000130073323F007037863ADEB030D7B6B0A
:1015F0000DF108089B00073323F00703ADEB030D43
:1016000002ABBB62B4F8AC300025B3F5807F14BFE9
:1016100002230123BB60BB694344FB6007F1380030
:1016200033F042FCB4F87A307862B3F5807F05D0AD
:101630005946504607F1380233F052FAB4F8AA304E
:1016400087F833301DB1B4F8AC3087F833305046EA
:1016500016F056FE002800F02681012394F8B620EB
:101660000093002107F13303206DD4F860C0E047F8
:10167000504633F032FA00239946FB61BB8B3A6A3D
:101680009A4200F2A380BA686B1C9A424FF001059F
:10169000C4D808E1A068002800F0108115F0C6FF4A
:1016A000F862002800F00A81B4F87A30B3F5807F40
:1016B0007FF45BAF54E7204604F1080628F0B6FE3D
:1016C0003046C7F828D033F083F90546304633F06A
:1016D00081F9C5F34F05EB1D23F00703ADEB030DB7
:1016E0000DF108092A4677218046484639F05EF90F
:1016F000B4F8AA30504687F8443016F001FE83460D
:1017000088B12046D7F828D028F0AFFE94F8B23040
:10171000002B3FF42FAFFEF747F900287FF42AAFE4
:10172000FEF77AFFF2E70123014694F8B620009312
:10173000266E07F14403206DB047504633F0CDF9D3
:101740001FFA8BF39845DCD9504616F0D9FD0BF102
:10175000010B0028D5D094F8B62000954B46012106
:10176000266EE8E707F1380033F099FBB8FBF0F09C
:10177000002808BF012086B207F1380033F094FB3F
:10178000B0FBF6F083B207F138003B6233F08CFB1C
:10179000B0FBF6F303FB160080B218B13B6A0133CD
:1017A0009BB23B6207F1380033F079FB16FB00F087
:1017B00080B2B0FBF5F293B205FB1202002A3FF4AF
:1017C0000CAF01339BB208E7C81B05087B69786A38
:1017D0007A8FFB643B8F8642A7F8443002EB090303
:1017E00088BF7A6A9BB298BF9219A7F8463095BF16
:1017F0004A449B1813B21BB2A7F84A307B6AB7F968
:101800003C109B1B9BB2A7F8481007F144007B6279
:1018100033F04FFB082294F83A300021B2FBF3F387
:10182000B0FBF3F37A6BB86A92007B6039F0BEF8D4
:1018300000214046BA6939F0B9F894F8B43013B9C8
:1018400040F20713E387D5B194F8B33063B10623B0
:1018500084F83E3043465846BA6A07F1440133F0F3
:10186000E5F894F8B13013E094F8402012B184F810
:101870003F30EFE7B4F84230002BF2D0EAE74346BE
:101880005846BA6A07F1440133F0D0F894F8B03002
:10189000B3B9504616F034FDFB69B1440133FB6126
:1018A0001FFA89F9A8B9FB6AD7F810D09B68FB62C8
:1018B000002B7FF467AE204628F0D7FD01202AE6F2
:1018C0004346FA689342E4D01A68D24343F8042BA3
:1018D000F7E7BB8894F8B620009301214346206DBA
:1018E000D4F860C0E047504633F0F7F8FEF794FEB6
:1018F000C4E600BF10B590F8B23004463BB3D0F850
:101900008420134B9A4214D1843028F030FD94F88F
:10191000AF3083421BD0FEF72BFF002184F8B210BA
:101920002046B4F8A230D4F89820BDE81040FFF764
:1019300049BC28F069FCD4E90432C01AB4F8A830D4
:1019400061EB020183424FF000038B41E3D310BDF2
:10195000C81B050810B590F8B230044693B1D0F812
:101960008420104B9A4201D028F04EFDFEF700FF74
:1019700000212046B4F8A230D4F8982084F8B210A0
:10198000FFF720FC04F1080033F044F8D4F8842079
:10199000054B9A4205D104F18400BDE8104028F0BF
:1019A000DBBC10BD60EC0408C81B050810B5044979
:1019B0000446083032F0DEFF012384F8483010BDC1
:1019C000E809002010B50B4C0B4B22689A420ED14F
:1019D000A2680A4B9A420AD1204628F063FD28B932
:1019E0002046FFF783FD80F00100C0B210BD00204B
:1019F000FCE700BF28240020ECBB0408E809002015
:101A000008B5014803F038FCF6C4050810B50449D0
:101A10002AF082FD044603F025F8204610BD00BFE1
:101A2000ECBB0408F0B50C4689B0064654F8040B2C
:101A30001746FFF7EBFF03AB01930C4B05463A4605
:101A400021460093701E022307F060FB05A90522C2
:101A5000039808F041FC049808F044FA05A90246EE
:101A60002846FFF7FFFC0E2009B0F0BDDCBB0408E0
:101A700008B5FFF7CBFFFFF739FD10B9024803F0B7
:101A800003FC0E2008BD00BFA7BF050810B5FFF777
:101A9000BDFF28F007FDA0B16430EEF7B7FC0022CF
:101AA0000A4BEEF757FEEEF7C5FF01460446EFF787
:101AB000E5FA40B924F0030040F00200A0F1FF4035
:101AC00010BD0348FCE70348FAE700BF00408F4021
:101AD00002008080020040002DE9F04FCBB00846A4
:101AE00011461A462AAB01936A4B009320232CF02F
:101AF0006DF82A9B05220AA92B98039308F0ECFBAA
:101B000005220DA92C9808F0E7FB40F2D621409859
:101B100029F094F95A22339F049097FBF2F302FBC9
:101B2000137313B15C4803F091FBFFF7C7FA054646
:101B30003F9808F0D7F98346429808F0D3F98246D7
:101B4000489808F0CFF93C9B80463A9805933D9B16
:101B50000E28069300F08C802CF0A4F906463E9CDB
:101B600009A920469DF81C9108F03EF9002800F0D4
:101B70008280032029F08DFF099B04460370002317
:101B80004370837009F10203444A00212A600DF179
:101B900056005222079338F009FF0A9A039B1492C9
:101BA0000B9A1393ADF854200D9ACDF858801792E4
:101BB0000E9AADF86E70ADF860202D9A2846ADF8FB
:101BC00062202E9A13A9ADF864202F9AADF86620F2
:101BD000309AADF86820319AADF86A20329AADF8A3
:101BE0006C20349AADF87020359AADF87220369A90
:101BF000ADF87420379AADF87620389A059BADF889
